:020000040800F2
:10000000304F002091D00008693400086B3400089C
:100010008134000897340008AD3400080000000067
:10002000000000000000000000000000C3340008D1
:10003000C534000800000000C7340008C9340008B7
:10004000ABD00008ABD00008ABD00008ABD00008A4
:10005000ABD00008ABD00008ABD00008ABD0000894
:10006000ABD00008ABD00008ABD00008ABD0000884
:10007000ABD00008ABD000081F140008B113000873
:10008000ABD00008ABD00008ABD00008ABD0000864
:10009000D1820008ABD00008ABD00008D5340008EE
:1000A000ABD00008ABD00008ABD00008ABD0000844
:1000B000E5340008ABD00008ABD00008ABD0000896
:1000C000ABD00008ABD00008ABD00008ABD0000824
:1000D000ABD00008ABD00008732A0008ABD00008F2
:1000E000ABD00008ABD00008D5820008DFF810D0F4
:1000F0000DF0C2FF0048004741340008AFF3008014
:10010000304F0020F0B507460020059E0446054606
:10011000A9B184469EB1761E8C4212D2B04210D252
:1001200017F804E0964508D1A54205D03D4443F8B0
:10013000205007F804C0401C651C641CECE700203C
:10014000F0BD8D4203D2791943F82010401C43F8CA
:1001500020C0F0BD2DE9F04F0024A1B08B468246AF
:100160004FF0FF364FF02009A0462746802101A816
:100170000DF079F82CA150460DF080F8B0B32B4D5E
:100180000FE050460DF07AF8040009D055F837001A
:100190000DF086F80444A4EB0A001FFA80F804E08E
:1001A0007F1C55F837100029EBD120783F2804D068
:1001B0000D2810D03D281AD034E060780D2831D1B8
:1001C000A0780A282ED105EBC700436873B101AAB5
:1001D000494601201BE060780A2823D105EBC700BF
:1001E00043681BB101AA4946022010E01AE0601CD6
:1001F000ABEB080101AB2C22CDF80090FFF782FF9A
:10020000014605EBC700436863B101AA0320984784
:100210000646401C06D006A002F080FB21B0304606
:10022000BDE8F08F04A0F7E741540000CC010108BD
:100230000D0A4F4B0D0A00000D0A4552520D0A00DF
:1002400000B591B0402168460DF00DF8F9A2FBA170
:1002500068460EF0A7F968460DF022F881B26846AC
:1002600001F08BF8002011B000BD00F0C4FEF9A031
:1002700002F054FB642002F09FFA00F00BFE00F045
:10028000A8FE00F0B8FEF3A002F048FB642002F0E4
:1002900093FA00F0FFFDEFA002F040FB00F0FAFD42
:1002A0002DE9F043C3B01746894603282AD14FF4FD
:1002B000807103A80CF0D7FF38680DF040F884B2C5
:1002C00078680DF03CF81FFA80F8B8680DF037F840
:1002D00086B2F8680DF033F885B238690DF02FF862
:1002E00081B2B8F1000F02D0B8F1010F08D10EB100
:1002F000012E05D10DB1012D02D1B9F1050F04D0A8
:100300004FF0FF3043B0BDE8F083D44808F0FF035E
:1003100080F82830A0F829101EB3052280F87C2030
:10032000012D20D05FF0000280F88220012B1CD02C
:10033000642C14D8C4840096CDE901512246C8A18A
:1003400003A80EF02FF903A80CF0AAFF81B203A8AE
:1003500001F013F8BFA002F0E1FA04F012FD002052
:10036000D0E70922DAE70122DEE7082CF7D8C484B7
:100370000096CDE901512246B9A103A80EF012F969
:1003800003A80CF08DFF81B203A800F0F6FFB1A026
:1003900002F0C4FA03F068FEE1E730B5C3B000250F
:1003A0002C464FF4807103A80CF05DFFAB4890F829
:1003B0007C10092900D0012590F88210012900D174
:1003C0000124B0F829100095CDE9014190F82830BA
:1003D000C28CB0A103A80EF0E5F803A80CF060FFF2
:1003E00081B203A800F0C9FF43B0002030BD30B592
:1003F00091B00C461546402168460CF034FF286841
:100400000CF09DFF10F0FF0001D0012801D1012C5C
:1004100003D04FF0FF3011B030BD904C012884F86C
:100420002B0001D107F09EFA94F82B20A6A1684674
:100430000EF0B8F868460CF033FF81B2684600F061
:100440009CFF00F0D8FD83A002F068FA642002F05F
:10045000B3F900F01FFD00B591B0402168460CF0E3
:1004600002FF7E4898A190F82B2068460EF09AF87B
:1004700068460CF015FF81B2684600F07EFF002050
:10048000F1E62DE9F04FCDB08B4614464FF4807164
:100490000CA80CF0E8FE20680CF051FF00F0FF0AF9
:1004A000A0680CF04CFF00F0FF09E0690CF047FF7A
:1004B000206A0CF044FFE0680FF000F80DF006FB36
:1004C000054620690EF0FAFF0DF000FB0646606954
:1004D0000EF0F4FF0DF0FAFA8046A0690EF0EEFF80
:1004E0000DF0F4FA074660680CF029FFBBF1090F24
:1004F00004D04FF0FF304DB0BDE8F08F77490A6867
:10050000A2F81AA010800A68CA4650800C683846C3
:10051000A4F81890E5612662A946C4F824804546EF
:10052000A7620DF090FA8346284600910DF08BFAF1
:1005300007460D4630460DF086FA06468846484680
:100540000DF081FA024600200A900B460B900099AC
:100550000DF1080CCDF800A08CE84C01CDE908B1F4
:10056000CDE906752388628B5D490CA80EF01AF858
:100570000CA80CF095FE81B20CA800F0FEFE002045
:10058000B9E72DE9F047CCB04FF480710CA80CF01E
:100590006AFE52480468A06A0DF055FA81468A4600
:1005A000606A0DF050FA07468846206A0DF04BFA53
:1005B00005460E46E0690DF046FA0A4600210A910A
:1005C00002AB0B9183E8E507208B00902388628BB8
:1005D00044490CA80DF0E6FF0CA80CF061FE81B2B6
:1005E0000CA800F0CAFE4CB00020BDE8F087002047
:1005F000704700B591B000201090402168460CF083
:1006000032FE10A809F0F9F910B14FF0FF302AE6D8
:1006100010980DF018FA02460B4633A168460DF00B
:10062000C1FF68460CF03CFE81B2684600F0A5FEB2
:10063000002018E656312E302E3100000D0A676575
:100640007476657220736F6674776172653A25738C
:100650000D0A00000D0A4F4B0D0A00008C0B002004
:100660000D0A7365746366672049443A25642C203B
:10067000526F6C653A25642C2043483A25642C203F
:10068000526174653A25642C2047726F75703A2563
:10069000640D0A000D0A6765746366672049443A71
:1006A00025642C20526F6C653A25642C2043483A0F
:1006B00025642C20526174653A25642047726F7559
:1006C000703A25640D0A00000D0A776F726B6D6F2A
:1006D00064653A2025640D0A0000000034100020F3
:1006E000F40F01086C0F01080D0A616E676C653A22
:1006F0002025660D0A00000030B591B00C46154665
:10070000402168460CF0AFFD28680CF018FE10F090
:10071000FF0001D0012809D1012C07D1F94C012893
:1007200006D000202070C0B201F0A8FF002072E6C1
:1007300000220121104601F081FF0120F2E701466D
:1007400006E00D2A03D00A2A01D000F8012B491C2B
:100750000A78002AF5D100210170704710B51446BF
:100760000B461068FFF7EBFF012B07D107F0FAF8F3
:10077000022303211320226807F00CF9002010BD8A
:1007800000B591B0402168460CF06DFDDE48006870
:100790000DF059F902460B46DCA168460DF002FF48
:1007A00068460CF07DFD81B2684600F0E6FD002051
:1007B00059E530B5C1B04FF4807168460CF053FD77
:1007C00045F65A22D6A168460DF0ECFE054668466D
:1007D0000CF066FD6C462044D3A10DF0E3FE6846A4
:1007E0000CF05EFD2044D3A10DF0DCFE68460CF059
:1007F00057FD2044AFF2C412D4A10DF0D3FE6846D9
:100800000CF04EFD2044D6A3D8A2DBA10DF0CAFE09
:1008100068460CF045FD2044DCA2E7A10DF0C2FEC5
:1008200068460CF03DFD421BE7A1A01C0DF0BAFE8E
:100830007B20605568460CF033FD2044D2A10DF0BA
:10084000B1FE68460CF02CFD81B2684600F095FDC3
:1008500041B0002030BDF0B5A9B00AF081FB0746D9
:100860000AF076FB0546A02101A80CF0FCFC0D2245
:100870001DB10A20152101FB0502A9A101A80DF057
:1008800091FE01AEA0213046D1A20DF071FE0446CA
:1008900015E038680090C4F1A0013019CFA27B6840
:1008A0000DF066FE0444012D06D9C4F1A0013019F3
:1008B000A5A20DF05DFE04446D1EADB20837002DFB
:1008C000E7D1C4F1A0013019C8A20DF051FE2044B7
:1008D00081B201A800F051FD0AF058FB002029B0B8
:1008E000F0BDF0B5A9B0A02168460CF0BCFC0AF040
:1008F0007BFA06460AF07CFA071E4FF00C020ADD6E
:100900003146684600F0D3FA68460CF0C9FC09216C
:10091000C01C00FB071282A168460DF043FE6D4625
:10092000A0212846B2A20DF023FE0446308888B1EB
:1009300031462819064600F0BAFA30460CF0B0FCF1
:100940000444012F06DDC4F1A00128197EA20DF098
:100950000FFE0444C4F1A0012819A4A20DF008FE62
:10096000204481B2684600F008FD0020B7E72DE979
:10097000F047A8B08A461746A02168460CF073FCE1
:100980001022002138680CF0D8FC0446884610225A
:10099000002178680CF098FC8146B8680CF0CFFC18
:1009A0000646F8680CF0CBFC054638690CF0C7FC2D
:1009B00007461EB115B1BAF1050F03D04FF0FF3055
:1009C00028B012E61FFA89F2204641460AF06EFA74
:1009D000040037D0A681E581278245F65A2250A12E
:1009E00068460DF0DFFD064668460CF059FC6D4682
:1009F000284482A10DF0D6FD68460CF051FC284435
:100A0000214600F054FA68460CF04AFC28447FA1C5
:100A10000DF0C8FD68460CF043FC821B6AA1A81CBF
:100A20000DF0C0FD7B20A85568460CF039FC284429
:100A300055A10DF0B7FD68460CF032FC81B2684656
:100A400000F09BFC0020BBE7F0B5A9B00E461446B1
:100A5000A02168460CF007FC1022002120680CF051
:100A60006CFC04460D46012E02D04FF0FF3036E7F5
:100A70004FF6FF710020091BA84104D220462946E9
:100A80000AF05BFA02E0A0B20AF04CFA45F65A22EC
:100A900023A168460DF086FD074668460CF000FC71
:100AA0006E46304422462B4659A10DF07BFD684628
:100AB0000CF0F6FBC21B44A1B01C0DF073FD7B20B3
:100AC000F05568460CF0ECFB30442FA10DF06AFDA8
:100AD00068460CF0E5FB81B2684600F04EFC00F081
:100AE0008AFA0020FBE610B5012902D04FF0FF3052
:100AF00010BD10680CF023FC4C49096848860020A2
:100B000010BD000004000020000000200D0A6469F0
:100B10007374616E63653A2025660D0A000000005B
:100B20004A532530345800007B22496E666F223AC2
:100B30007B0D0A0022446576696365223A2250449F
:100B40004F41204E6F6465222C0D0A0022566572BB
:100B500073696F6E223A222573222C0D0A00000061
:100B600031373A33353A3038000000005365702091
:100B70002032203230323600224275696C64223ACB
:100B8000222573202573222C0D0A00004457333090
:100B900030302043302044657669636520447269B3
:100BA0007665722056657273696F6E2030342E3010
:100BB000302E3030000000002244726976657222C7
:100BC0003A222573227D7D00253034580000000034
:100BD0007B22444C697374223A5B20002225303812
:100BE0006C582530386C5822000000005D7D0000F4
:100BF0007B224B4C697374223A5B00007B22546168
:100C0000674164646564223A200000007D000000B2
:100C10007B2254616744656C65746564223A2022C6
:100C20002531366C6C78227D0000000034100020E5
:100C300010B5012902D04FF0FF3010BD10680CF044
:100C40007EFBA44909688886002010BD10B50129E3
:100C500002D04FF0FF3010BD10680CF070FB9D49C2
:100C60000968A1F84400002010BD2DE9F04FC7B07D
:100C70008B4617464FF4807107A80CF0F4FA3868D9
:100C80000CF05DFB1FFA80FA78680CF058FB1FFA35
:100C900080F9B8680CF053FB86B2F8680CF04FFB93
:100CA00084B238690CF04BFB1FFA80F878690CF0BD
:100CB00046FB85B2B8690CF042FB81B2BBF1070F6D
:100CC0002DD1BAF1010F2AD8B9F1010F27D8012C83
:100CD00025D8804808F0FF02006820F82E4F468093
:100CE0000277C5820183B0F90630B0F9047000962E
:100CF000CDE90573CDE90351CDE90142C37E827E82
:100D0000754907A80DF04EFC07A80CF0C9FA81B28E
:100D100007A800F032FB002047B0BDE8F08F4FF08D
:100D2000FF30F9E710B5C8B04FF4807107A80CF098
:100D30009AFA68480DF10C0C0068B0F84410B0F94C
:100D40003440B0F93230B0F846208CE81E0090F8FC
:100D50004A3030F82E2F41888DE80E00C37E827E07
:100D60005D4907A80DF01EFC07A80CF099FA81B2A6
:100D700007A800F002FB48B0002010BD10B5012903
:100D800002D04FF0FF3010BD10680CF0D8FA514976
:100D9000096881F84A00002010BD10B5012902D071
:100DA0004FF0FF3010BD10680CF0C9FA49490968CE
:100DB000A1F84600002010BD30B591B00C46154694
:100DC000402168460CF04FFA28680CF0B8FA10F091
:100DD000FF0001D0012801D1012C02D04FF0FF30DB
:100DE000A5E43E4981F82C0068460CF059FA81B21E
:100DF000684600F0C2FA002099E400B591B04021A5
:100E000068460CF030FA354835A190F82C20684639
:100E10000DF0C8FB68460CF043FA81B2684600F05A
:100E2000ACFA002005E430B591B00C4615464021DF
:100E300068460CF018FA28680CF081FA10F0FF00F0
:100E400001D0012801D1012C02D04FF0FF306EE417
:100E5000224981F82D0068460CF022FA81B26846DA
:100E600000F08BFA002062E400B591B040216846A2
:100E70000CF0F9F9194820A190F82D2068460DF0E2
:100E800091FB68460CF00CFA81B2684600F075FAE6
:100E900000208DE4BFF34F8F1C4801681C4A01F409
:100EA000E06111430160BFF34F8F00BFFDE730B534
:100EB00085B04A880DF1040C0D8ACC898B898CE8A9
:100EC0003C004A6800928B680A8812490DF06AFB60
:100ED00005B030BD341000207C1001088C0B0020C0
:100EE0000D0A7477725F70646F615F6D6F64653A4D
:100EF0002025640D0A0000000D0A6D63755F6D6F9B
:100F000064653A2025640D0A000000000CED00E045
:100F10000400FA05E41001082DE9F04788B081A02B
:100F200001F0FCFC8EA291A193A001F0F7FC9AA124
:100F30009BA001F0F3FC6420A14C00900822638E7A
:100F4000E18DA04801F0EAFC9FA0216801F0E6FCD9
:100F5000A5A0616801F0E2FCD4F8A0106069CDE9B9
:100F6000000104F10801A8480EC901F0D7FC206C6B
:100F70000CF069FD81468A46E06B0CF064FD074683
:100F80008846A06B0CF05FFD05460E46606B0CF0CA
:100F90005AFD0246208B0B46CDE905A08DE8E00303
:100FA000218E9A4801F0BAFC84A001F0B7FC08B089
:100FB0005CA0BDE8F04701F0B1BC10B503460022CB
:100FC000104603E010CB521C2044D2B28A42F9D31F
:100FD00010BD7B484AF6AA218522016000214160AC
:100FE0008160C16001614161C0F8A010A0F5386165
:100FF00018300CF01FB910B5854C02E0642001F0E8
:10100000DBFB2A226E49204601F0F7FD0028F5D0CF
:1010100010BD2A226A497E4801F020BE10B5FFF7B4
:10102000F8FF674C2068A0F52A41AA3913D079A0AF
:1010300001F074FCFFF7CDFFFFF7DDFFBFF34F8F2B
:1010400078480168784A01F4E06111430160BFF318
:101050004F8F00BFFDE760680021401C606073484F
:101060000AF072FC94F82B00012817D15449A822E9
:1010700001F1A8000CF0DEF851490020A831644CC1
:1010800081F82B0002E0642001F096FB4C492A22F3
:10109000A831204601F0B1FD0028F4D010BD10B5F4
:1010A00000F0C8F84FF4FA7001F086FBFFF7B6FFC6
:1010B000BDE8104030E770B5414EF08CA0F57F419F
:1010C000FF3901D0022400E0012400F0DCF800F038
:1010D0000AF95748D0F8F40A18B10021084600F080
:1010E0004CF9534D903D686884420FD06C6096F87F
:1010F0002B0058B9012C02D0022C07D101E00A22A2
:1011000000E002220221002001F098FA287800284D
:1011100004D0BDE87040012001F0B0BA70BD0120DC
:10112000704700002A2A2A2A2A2A2A2A2A2A2A2A10
:101130002A2A2A2A2A2A2A555742204D6F64756C7A
:101140006520CFB5CDB3B2CECAFD2A2A2A2A2A2AD3
:101150002A2A2A2A2A2A2A2A2A2A2A2A2A0D0A0056
:1011600053657020203220323032360031373A3326
:10117000353A303800000000202020555742204DDD
:101180006F64756C6520B1E0D2EBCAB1BCE4202578
:10119000732025730A00000056312E302E310000D6
:1011A000202020555742204D6F64756C6520C8ED96
:1011B000BCFEB0E6B1BEBAC5A3BA25730D0A0000E5
:1011C0008C0B002084110108202020555742204D0F
:1011D0006F64756C6520B1EAD6BECEBBA3BA25306C
:1011E00032580D0A00000000202020555742204DA3
:1011F0006F64756C6520BFAABBFAB4CECAFDA3BAF2
:1012000025640D0A0000000038110108CC11010806
:1012100000380108C9E8B1B8CAD7B4CEC9CFB5E71C
:101220000A0000000CED00E00400FA0500043000A4
:101230009400002010B54021B9480CF014F8B848CB
:10124000402140300CF00FF8B5480521803001F006
:101250002DFF10BD30B503460C880020250411D4A5
:10126000C4F30D0413550A88521C92B20A803F2A17
:1012700001D900220A800A2B04D190B240F4004028
:101280000880012030BD2DE9F043A1B04FF00009E6
:10129000802168460BF0E7FF8021684601F001FFDE
:1012A00005001CD000246E462746DFF8788214E043
:1012B0009B4A9C49305D4032891CFFF7CBFF58B1F7
:1012C000974829464030FEF745FF9548A8F8027038
:1012D000402140300BF0C7FF641CAC42E8DB21B07A
:1012E0004846BDE8F08300B58D4891B0694680302E
:1012F00001F064FF00280AD08B4890F82B100DF104
:10130000020001299DF8011003D0FEF723FF11B060
:1013100000BD01F031F9FAE72DE9F041834C0F46A9
:101320000146D4F8F40A0026C21904F5AF65B2F5F7
:10133000AF6F08D228443A460BF07CFFD4F8F40A89
:101340003844C4F8F40AD4F8F00A012812D1D4F8C9
:10135000F42A7AB1294675480BF06CFFB4F8F40A08
:10136000002281B2714804F52F6401F0AFFA002029
:10137000206060603046BDE8F08170B50C460546DF
:10138000FFF7CAFF21462846BDE8704001F08BBE3A
:1013900001F089BE01F057BB30B50446002003467A
:1013A00003E0CD18655D68405B1C9342F9DB30BDFE
:1013B00070B54FF40036A0B0304609F010FF40B3CE
:1013C0005B48574A57490078FFF744FF08B3442168
:1013D0000EA80BF048FF534D00248DF838402A78B2
:1013E0008DF839204E490DF13A000BF023FF3622DB
:1013F00011A968460BF01EFF0DF1380C48489CE817
:101400000E00803001F0A6FE2C80402144480BF0F5
:101410002AFF20B03046BDE8704009F0EEBE10B59E
:101420004FF40054204609F0C2FE002808D03F497E
:101430000120C1F8F00A2046BDE8104009F0C5BE01
:1014400010BD0FB430B50B9C9DF80C0020709DF8BA
:101450000D5065709DF80E00A070BDF80F00E07093
:10146000000A20719DF811006071BDF811002A4634
:10147000000AA071DDF81100000CE071DDF8110028
:10148000000E20729DF815006072BDF81500000A6C
:10149000A072DDF81500000CE072DDF81500000EFA
:1014A0002073BDF819006073000AA073DDF81B00FB
:1014B000E073DDF81B00000A2074DDF81B00000C4F
:1014C0006074DDF81B00000EA074DDF81F00E074EE
:1014D000DDF81F00000A2075DDF81F00000C6075A4
:1014E000DDF81F00000EA075BDF82300E075000AAE
:1014F0002076BDF825006076000AA076BDF82700AA
:10150000E076000A207702212046FFF745FF60774A
:101510009DF82A00A077281D30BC5DF814FB000060
:101520000C140020DC0C00208C0B00209400002008
:101530000410002010B5F9A001F0F0F9002010BD52
:1015400010B5022801D0002010BDF8A001F0E6F986
:10155000BFF34F8FF7480168F74A01F4E061114388
:101560000160BFF34F8F00BFFDE70088704701881F
:10157000408801EB0040704710B5002306E000BF33
:1015800030F8134021F813405B1C9BB29342F7D311
:1015900010BD2DE9F0414FF0006516460F46044698
:1015A000A8421DD3E54904EB4600884218D209F051
:1015B000C0FEA4F10060C00A05EBC02009F0F4FEF3
:1015C000002507E037F8151004EB450009F0AFFFE0
:1015D0006D1CADB2B542F5D3BDE8F04109F0B5BE22
:1015E000BDE8F081F0B500242546D3074FF0FF3762
:1015F00034D12FE0035DA3F13006092E01D8F6B2F5
:101600000BE0A3F14106052E01D8373B04E0A3F11E
:101610006106052E22D8573BDEB203195B78A3F191
:10162000300CBCF1090F02D80CF0FF030DE0A3F160
:10163000410CBCF1050F01D8373B05E0A3F1610C6B
:10164000BCF1050F0AD8573BDBB243EA06134B55F2
:10165000A41C6D1C9442CDDB0020F0BD3846F0BDCB
:1016600030B5002414E0035DA3F13005092D01D845
:101670000D550BE0A3F14105052D01D8373B04E0E2
:10168000A3F16105052D01D8573B0B55641CE4B24D
:101690009442E8D30023184609E05B1CDBB2CC5C23
:1016A0005B1C44EA04140C54401CDBB2C0B29342ED
:1016B000F3D900220A5430BDF0B5ADF2044D0D4609
:1016C00006464FF480671446394668460BF0CBFD5A
:1016D000394668460BF0C7FD30460BF0E1FD024687
:1016E000A04203DB2246314668460AE000206946F4
:1016F000A31A01E00D54401C8342FBDC0819801A38
:1017000031460BF097FD68460DF2044DF0BD2DE912
:10171000F84F0E46002859D0012857D0DFF820A2F4
:10172000032307270125874C4FF0100C0AF104080A
:101730004FF4A02202281CD0032847D1272E45D2DF
:1017400054F82600002841D00078012858D00228FB
:101750003CD100219146104603F0FDFC54F82610C0
:10176000C968072901EB41015DD305FA01F2024383
:101770005CE0272E2AD254F82600002826D00078D4
:10178000012811D0022821D100219146104603F0F2
:10179000E2FC54F82610C968072901EB410117D370
:1017A00005FA01F2024316E054F821006946048963
:1017B0004568ADF800408DF803C08DF8023028462A
:1017C0000AF033F8214628460AF09FF8BDE8F88F62
:1017D0008F4020EA07020021484603F0DAFC00228D
:1017E0001146504603F0D5FC00214746404603F021
:1017F000B2FC54F82610097B8D4020EA050229E04E
:1018000054F82100694604894568ADF800408DF818
:1018100003C08DF8023028460AF007F82146284612
:101820000AF071F8D2E78F4020EA0702002148460B
:1018300003F0AFFC00221146504603F0AAFC002141
:101840004746404603F087FC54F82610097B05FA0A
:1018500001F202433846BDE8F84F002103F099BC7D
:101860002DE9FF411C4615460ECB37A001F056F876
:101870000020019002900390032D05D029463BA043
:1018800001F04CF8BDE8FF8120680BF009FD082845
:10189000206804D208223021FFF70EFF20600BF0F1
:1018A000FFFC024601A92068FFF79CFE20680BF0B0
:1018B000F7FC024631A0216801F030F89DF80700DE
:1018C00000909DF806309DF805209DF804102FA08B
:1018D00001F024F860680BF0E3FC0828606804D28B
:1018E00008223021FFF7E8FE60600BF0D9FC0246C9
:1018F00002A96068FFF776FE60680BF0D1FC024633
:1019000029A0616801F00AF89DF80B0000909DF88D
:101910000A309DF809209DF808104DE044573330F7
:1019200030302D3030310D0A000000000D0A4F4BD1
:101930000D0A00000CED00E00400FA0500000808A4
:1019400008000500F80E0020617267765B305D3A92
:1019500025732C617267765B315D3A25732C617259
:1019600067765B325D3A25730D0A00006572726F0F
:101970007220617267633A25640D0A0061726776AE
:101980005B305D3A25732C25640D0A006770696F22
:101990005374617465313A25782C25782C25782C80
:1019A00025780D0A00000000617267765B315D3AB0
:1019B00025732C25640D0A00FCA000F0AFFFA06881
:1019C0000BF06EFC0828A06804D208223021FFF733
:1019D00073FEA060082203A9FFF704FEA0680BF0C5
:1019E0005FFC0246F8A0A16800F098FF9DF80F0088
:1019F00000909DF80E309DF80D209DF80C10F6A07B
:101A000000F08CFF0425002401AFC4F10306385D0B
:101A10006E4300F00300F1B2FFF779FE385D711CF0
:101A2000C0F38100C9B2FFF772FE385DB11CC0F38C
:101A30000110C9B2FFF76BFE385DF61C8009F1B2E8
:101A4000FFF765FE641CE4B2042CDED3002402AF71
:101A5000C4F10306385D6E4306F1100100F0030087
:101A6000C9B2FFF754FE385D06F11101C0F38100E1
:101A7000C9B2FFF74CFE385D06F11201C0F3011048
:101A8000C9B2FFF744FE385D13368009F1B2FFF7A3
:101A90003EFE641CE4B2042CDAD3002403AFC4F18C
:101AA0000306385D6E4306F1200100F00300C9B261
:101AB000FFF72DFE385D06F12101C0F38100C9B2A8
:101AC000FFF725FE385D06F12201C0F30110C9B20F
:101AD000FFF71DFE385D23368009F1B2FFF717FED0
:101AE000641CE4B2042CDAD3CCE670B514460D467F
:101AF00002280FD003280DD1012108460AF031FA3F
:101B00000121BC4809F020FF002123462A4608464F
:101B1000FFF7A6FE002070BD2DE9F04FA1B002F046
:101B200016FCB5A000F0FAFE002402F047FB02F01C
:101B3000F9FA022002F0EBFA4FF0FF3B4FF47A760D
:101B400007E0022002F0E3FA641CB44201DDAFA01A
:101B5000A6E004F0D8FF0028F3D0B0A000F0DEFE2D
:101B6000002003F0D2FB401C0ED0AFA000F0D6FE48
:101B7000032005F0DBF8B1A000F0D0FEB34803F07D
:101B800095FF18B1B2A08BE0B6A089E0BAA000F032
:101B9000C5FE05F0ADFADFF8B482A8F1A408454609
:101BA00088F8000003F03FFC0446024695F9001057
:101BB000B5A000F0B3FE1CB1BCA000F0AFFE80E009
:101BC0000024A146EA46002049465246641C1154AE
:101BD000401C7F28FBDB002005F07CF9B9A000F059
:101BE0009DFE0025BB4F07E0022002F090FA6D1C1D
:101BF000B54201DDB8A053E00021442003F0ABFA68
:101C00003842F1D0400465D5B7A000F087FE00212E
:101C10004C2003F0A0FAC0F309017F2908D8002264
:101C2000684604F052F99DF80110B6A000F076FE67
:101C300004F0B0F90BF027FE6FF019020BF0E8FD8D
:101C40000022B64B0BF003FD0BF040FF05460BF0F6
:101C5000FAFE02460B46B2A000F060FEB5F17E5FD0
:101C600002DC15F1814F21D9B54928460BF0CCFB98
:101C70000746454698F900000BF0E1FD39460BF0A8
:101C8000BDFB0BF03EFE00F03F00287005F027FA88
:101C900095F90010ABA000F041FEC82C13DDB5A0F3
:101CA00000F03CFE584621B0BDE8F08F1E214446AE
:101CB00098F9000003F065FC94F90010B3A000F05F
:101CC0002DFE0020EFE74FF480420021442003F076
:101CD00060FA78E7B8A000F021FEBD4AF5E710B53C
:101CE000022804D1FFF718FF08B1012010BD002021
:101CF00010BD2DE9F05F002402F060FA02F012FA44
:101D0000022002F004FA4FF0FF3B4FF47A7807E02C
:101D1000022002F0FCF9641C444501DD3BA03FE0D9
:101D200004F0F1FE0028F3D0002003F0EEFA401C8E
:101D300005D0464803F0BAFE18B145A030E0A5A092
:101D40002EE0012005F057F9012004F03CFE3F4C45
:101D50000125DFF88CA24FF00009A43C01E0A1A00E
:101D60001EE00020524649461154401C7F28FBDBF0
:101D70009F4A00201154401C2528FBDB9C487421FD
:101D800074380BF070FA002005F0A4F80026514FCB
:101D900030E1022002F0BBF9761C464505DD4EA07D
:101DA00000F0BCFD5846BDE8F09F23E16770696F05
:101DB0005374617465323A25782C25782C25782C5B
:101DC00025780D0A00000000617267765B325D3A8B
:101DD00025732C25640D0A006770696F5374617454
:101DE00065333A25782C25782C25782C25780D0A12
:101DF000000000000004300072785F776974685F4B
:101E00007874616C5F7472696D0D0A0049444C45C9
:101E10005F5243206572726F720D0A0049444C454F
:101E20005F52430D0A0000006477745F696E697445
:101E300069616C6973650D0A000000006477745F66
:101E40007365746C6564730D0A000000940F0020C4
:101E5000434F4E464947204641494C4544202020A7
:101E600020200000494E4954204641494C45442019
:101E700020202020000000006477745F636F6E668E
:101E800069677572650D0A007543757272656E74C7
:101E90005472696D5F76616C3A25642C587472696E
:101EA0006D466C673A25640D0A000000616C72652E
:101EB0006164792063616C6962726174696F6E0D2F
:101EC0000A0000006477745F7278656E61626C6509
:101ED0000D0A000000D0052472785F74696D6520DA
:101EE0006F75740D0A0000005359535F53544154E9
:101EF00055535F52584643475F4249545F4D4153E3
:101F00004B0D0A004672616D652052656365697606
:101F10006564207365713A25640A000080842E414F
:101F200061646A757374696E6720207874616C4FA0
:101F300066667365745F70706D3A25660D0A000001
:101F40007BC7543F61646A757374696E67206477F8
:101F5000745F7365747874616C7472696D20754315
:101F6000757272656E745472696D5F76616C3A2534
:101F7000640D0A0061646A757374696E6720636F2B
:101F8000756E74206F75740D0A000000656E642014
:101F90006477745F7365747874616C7472696D20B2
:101FA0007543757272656E745472696D5F76616C9B
:101FB0003A25640D0A0000005359535F53544154AD
:101FC00055535F414C4C5F52585F4552520D0A00C9
:101FD00000900524494E4954204641494C4544004F
:101FE000E4150020636F756E74206F75740D0A0020
:101FF000F01600200021442003F0ADF83842606064
:102000003FF4C7AEA088400455D54FF4804200216C
:10201000442003F0BEF800214C2003F09CF8C0F3EC
:10202000090161807F2903D80022F84803F04DFFA1
:10203000F648983004F01BF8F44C25219834B4F895
:1020400040008009801E82B204F17400303403F035
:1020500069FF608A0BF028FC00224FF080430DF0EE
:10206000A3FB064620880D4640050BF01DFC3246BA
:102070002B460BF05EFB0BF029FD0DF0BBFAE4499B
:102080000BF0C2F90BF0DFFCE24AE34B0BF0D9FA9C
:102090000BF01CFD0BF0D7FC02460B46DFA000F056
:1020A0003DFC218BE1A000F039FC218EE3A000F083
:1020B00035FC002077E6E54A0021442003F069F86A
:1020C000D248803004F0AAFF6D1CC82D7FF746AEC1
:1020D00045E610B5022804D1FFF70BFE08B1012038
:1020E00010BD002010BDF0B5002506462C4606E0C8
:1020F000355D202D01D0092D03D1641CA4B28C4282
:10210000F6D3002301202D2D1BD1801E17E0355D55
:10211000A5F13007092F03D803FB0253303B0EE033
:10212000A5F16107052F03D803FB0253573B06E0D7
:10213000A5F14107052F06D803FB0253373B641C6A
:10214000A4B28C42E3D35843F0BD7CB50D4606469D
:102150004FF0FF3402F032F801F0E4FF022001F00A
:10216000D6FF15B1012D06D01CE002223146002019
:1021700004F088FB16E000200090022269460190DE
:1021800004F080FB009808B9019808B1214606E0E8
:1021900002223146002003F003FA04460146ACA0B7
:1021A00000F0BCFB20467CBDF0B58BB01646022883
:1021B00004D00021032802D001286FD0A1E00591AE
:1021C00006910791002430680BF06AF80C2866D15C
:1021D00005AF012501E0052C20D2326812F8140069
:1021E000A0F13001092905D91139052902D9203971
:1021F000052954D805EB4403D15CA1F1300CBCF1A6
:10220000090F07D9A1F1410CBCF1050F02D96139C1
:10221000052979D88DF81C00D05C1EE0326812F8D0
:102220001400A0F13001092905D91139052902D975
:102230002039052968D805EB440C12F80C10A1F1DF
:102240003003092B05D9113B052B02D9613905292A
:102250005AD88DF81C0012F80C008DF81D001022C1
:10226000022107A8FFF73FFF3855641CE4B2062C93
:10227000B1D39DF8180001AC9DF81B309DF81A20D1
:102280009DF8191084E80F009DF8170000909DF844
:1022900016309DF815209DF8141001E01AE033E087
:1022A0006EA000F03BFB9DF81610BDF81400BDF8C1
:1022B000182061F31F409DF81710099240EA016051
:1022C000089001466EA000F029FB012108A8FFF745
:1022D0003CFF16E003910491002103A8FFF735FFAE
:1022E0009DF80F009DF811209DF810108DE8070053
:1022F0009DF80E309DF80D209DF80C1064A000F0A4
:102300000DFB00200BB0F0BD0120FBE770B590B0D5
:1023100016460D46022826D0664C032802D0012816
:1023200024D020E0402168460AF09DFF30680BF081
:1023300006F810F0FF0001D0012807D1012D05D1CA
:1023400084F82B00012801D105F00CFB94F82B2018
:1023500059A168460CF026F968460AF0A1FF81B23F
:102360006846FFF70AF810B0002070BD40216846AB
:102370000AF079FFEAE700B591B0402168460AF01B
:1023800072FF4C484CA190F82B2068460CF00AF9DB
:1023900068460AF085FF81B26846FEF7EEFF11B08D
:1023A000002000BD002070472DE9F04FADF57B7D8A
:1023B0008A4681464FF0FF364FF0FA0800244FF46A
:1023C0007A7168460AF04FFF40A148460AF056FF6E
:1023D000002818D03E4D00BF55F8341048460AF08A
:1023E0004DFF070078D055F834000AF059FF384403
:1023F000A0EB09018AB2092C05D201783F2970D0DF
:1024000011B13D297DD0ACE073E065E0E41500201A
:1024100000002041CDCCCCCCCC6C5E407369675FB2
:10242000706F7765723A25660D0A000073747350F9
:102430006F7765723A25640D0A0000007374733279
:10244000506F7765723A25640D0A000000900524EC
:102450006572723A25640D0A000000006D61635FC9
:10246000746D703A25782C25782C25782C25782CBD
:1024700025782C25782C25782C25780D0A0000004D
:1024800065756936343A25782C25780D0A000000E8
:102490005557424D41433A25303278253032782520
:1024A0003032782530327825303278253032780D48
:1024B0000A0000008C0B00200D0A776F726B6D6FA5
:1024C00064653A2025640D0A0000000041540000B4
:1024D000A40F002005E014E0641C092CFFF47CAF7D
:1024E0003FE005EBC4004368DBB36A464146012088
:1024F00034E005EBC40043689BB36A4641460220C2
:102500002CE0BAEB02074FF000024FF02C09EB462B
:10251000C2461346944600F1010003D00121E6466D
:10252000009013E0614613E010F80280C84503D123
:1025300000F802E0012308E03BB100EB02084BF891
:1025400021800023491C514502D2521CBA42EBD3D0
:1025500005EBC400436823B15A46032098470600A0
:1025600007D018A000F0DAF90DF57B7D3046BDE804
:10257000F08FAFF64840F5E72DE9F0410C460746ED
:102580003E194FF0FF3016F8021C0D2917D116F82E
:10259000011C0A2913D1042C11D3002504E0795D14
:1025A0000BA000F0BBF96D1CA542F8DB002006F87B
:1025B000020CA41EA1B23846BDE8F041F4E6BDE825
:1025C000F08100000D0A4552524F520D0A000000E2
:1025D000256300005B4A052818D2DFE800F0140FDD
:1025E0000F0F140002210BE001290FD1022102E09C
:1025F00001290BD10021104609F087B90029F7D134
:10260000104609F080B90029EED1EBE7704708B514
:102610000121042009F0A5FC0220ADF800001020E3
:102620008DF8030003208DF802006946454809F043
:10263000FCF801210420FFF7CDFF08BD10B5424B87
:1026400002290DD0042804D003F82010FFF7C2FFA0
:1026500010BD0022521C03F82010042AFADBF5E713
:1026600028B1012803D0022801D00328F0D102218B
:1026700003F8201003EB8000428010BD70B5334E8C
:102680004FF4A023351D48B32F4CA41E20780428F6
:1026900011D200221146184602F07BFD002211469D
:1026A000304602F076FD2078012282400021284643
:1026B00002F06FFD03E000210846FFF78BFFC82002
:1026C00000F07AF82078052801D2401C04E00121AE
:1026D0000020FFF77FFF0020207070BD0F22002137
:1026E000184602F056FD0F220021304602F051FD3F
:1026F00000221146284602F04CFDBDE870400A2237
:10270000022100209AE770B50F4D0646002400BF55
:1027100015F82400022811D105EB84004088B6FB8F
:10272000F0F100FB116149B9B6FBF0F0C007E0B26F
:1027300001D0002100E00121FFF74CFF641C042CB4
:10274000E6DB70BD00080140EE0F00200800050028
:1027500010B54FF4407008F023FC00F052F800F080
:102760004BFAFEF756FC134C94F82B00FF2801D0CF
:1027700018B104E0002084F82B00FFF748FF00F0B8
:102780008FF900F008FB94F82B00002811D100F01D
:102790007DFC94F82B0000280BD100F003FB94F88B
:1027A0002B00002805D100F03DFBBDE8104007F0EC
:1027B00056B810BD8C0B0020424908604FF0E02055
:1027C000026942F00102026108680028FCD17047EA
:1027D0003C480168002902D00168491E0160704729
:1027E00008B51C208DF800000B208DF8010000209A
:1027F0008DF8020001208DF80300684608F0D5FB33
:1028000008BDFEB530484FF47A710068B0FBF1F0B6
:10281000401EB0F1807F42D24FF0E0246061671724
:102820000F21384600F03EF80025A56107262661F5
:102830000521384600F036F80121084609F09AFBD8
:1028400040F2E730ADF8040041F61F40ADF800005B
:102850004FF08044ADF80650ADF80250694620466E
:1028600009F0A0FD0122114620460AF059F8012185
:1028700020460AF040F8FFF7B3FF40F2712445F21A
:10288000555009F045FA304609F045FA204609F05E
:1028900045FA09F046FABDE8FE4009F047BAFEE7FE
:1028A00009F03FBA0907090E002804DB00F1E02017
:1028B00080F80014704700F00F0000F1E02080F86D
:1028C000141D704700100020F41300202DE9F04182
:1028D0000E460746012A0FD0C14C0021204608F0C1
:1028E0004EFCBF484438866407650121204608F045
:1028F00046FC3046BDE8F0810025BA4C0BE021884B
:102900002046795D0AF029FB402120460AF086FB2B
:102910000028F9D06D1CB542F1DBEAE70FB44FF4A3
:10292000807110B503ABB048029A0BF04FFE81B234
:102930000122AD48FFF7CAFF10BC5DF814FB2DE97A
:10294000F04301218BB0084609F002FBDFF89082CA
:10295000404608F07DFBA34D00242D1D102080264D
:102960000095CDE9044647020290CDE90847069458
:102970000794694640460A9408F0D7FB01220221D9
:10298000404608F007FCDFF85C82012280214046C7
:102990000AF0AFFADFF8489209F11409484608F046
:1029A00057FB92480095CDE9010403A9012081E875
:1029B000510020200694CDE90740CDE9097469460D
:1029C000484608F0B2FB01220221484608F0E2FB2B
:1029D0000121484608F0D3FB0122402140460AF07D
:1029E00088FA0BB0BDE8F08308B50E208DF8000022
:1029F0000A208DF8010000208DF8020001208DF8DA
:102A00000300684608F0D1FA08BD08B50F208DF81C
:102A100000000A208DF8010000208DF8020001203E
:102A20008DF80300684608F0C0FA08BD10B5704C78
:102A3000014620460AF091FA802120460AF0EEFA7B
:102A40000028F9D010BD2DE9F0410E4607460024BC
:102A5000674D0BE0395D28460AF07FFA8021284651
:102A60000AF0DCFA0028F9D0641CE4B2B442F1D3D5
:102A700040E770B55E4C40F22555294620460AF0E5
:102A8000D7FA00280BD020460AF06BFAC0B2FFF745
:102A9000CDFF29462046BDE870400AF0E8BA70BD77
:102AA0001FB5012144F2040009F05BFA4FF40070F5
:102AB000ADF8000003208DF8020018204D4C8DF871
:102AC00003006946204608F0B0FE2015ADF800006E
:102AD00004208DF803006946204608F0A6FE4FF456
:102AE000E13000900020ADF80400ADF80600ADF82C
:102AF0000800ADF80C000C203A4CADF80A0069460D
:102B000020460AF061F9012240F2255120460AF0E0
:102B1000D8F9012120460AF0CAF9FFF710FFFFF7A4
:102B200063FFFFF772FFBDE81F40AFF3008070B591
:102B300086B00121042009F014FA0121480409F0AB
:102B400019FA0424ADF8104018208DF81300294E0E
:102B500003258DF8125004A9304608F066FE0820BF
:102B6000ADF810008DF813408DF8125004A93046CE
:102B700008F05BFE00244FF4E1300090ADF808400F
:102B80000C201B4DADF80440ADF80A00ADF806402E
:102B9000ADF80C40694628460AF016F9012128468E
:102BA0000AF085F9012240F2255128460AF089F9F8
:102BB000402128460AF039FA4FF4C06008F0F0F9D5
:102BC00026208DF814008DF815408DF81640012050
:102BD0008DF8170005A808F0E8F906B070BD0000F0
:102BE0004400024000380140151700200410002066
:102BF00000440040000801407047F8B50546042035
:102C000016460F4600248DF8000008F092FB352090
:102C100008F09DFD284608F0C7FB8DF800009DF8E0
:102C2000000004280AD015E057F82410284608F0C0
:102C30005AFC8DF80000641CE4B22D1DB44203D28E
:102C40009DF800000428EFD008F07FFB9DF80000FD
:102C5000042801D00020F8BD0120F8BD10B50023E4
:102C600004E010C841F823405B1CDBB29342F8D368
:102C700010BD000008B517208DF8000001208DF868
:102C8000010000208DF802008DF80300684608F06E
:102C90008CF908BD1CB50521012008F07EFE20201E
:102CA000009000208DF8040008208DF80500012018
:102CB0008DF80600684608F0BDFAFFF7DBFF1CBD83
:102CC00070B5354D86B0284609F09AF90121080300
:102CD00009F047F901210D2009F043F90021ADF871
:102CE00004104FF48270ADF80600ADF80C106815B2
:102CF000ADF80E00ADF80810ADF810100720ADF8D3
:102D00000A10ADF81210ADF8140001A9284609F018
:102D10009BF9A020ADF8000018208DF803001F4E8D
:102D200003248DF802406946304608F07EFD4020BD
:102D3000ADF8000048208DF803006946304608F0E1
:102D400074FD1021ADF800108DF803108DF80240CD
:102D50006946304608F069FD0021284609F029FA45
:102D60000121284609F0EDF91021304608F0CBFD8D
:102D70000121082009F0F5F82020ADF800002820F6
:102D80008DF803006946064808F04FFDFFF782FF03
:102D900006B0002070BD93E70030014000080140FC
:102DA000000C014010B5012186B0480509F0E2F899
:102DB0000121082009F0D5F8C020ADF8100003204B
:102DC0008DF812001C208DF8130004A9934808F018
:102DD0002CFD934C204608F007FE0020ADF80400BF
:102DE0004BF6FF70ADF806003020ADF80800201556
:102DF000ADF80A000001ADF80C008A4800900121EE
:102E0000204608F06BFE6946204608F000FE04F0FC
:102E100022FDFF2004F08AFD002004F087FD002041
:102E200006B010BD10B5012186B0880509F0A2F8E2
:102E30000121082009F095F84FF44060ADF810002A
:102E400003208DF812001C208DF8130004A973488C
:102E500008F0EBFC744C204608F0C6FD0020ADF8ED
:102E600004004BF6FF70ADF806003020ADF8080006
:102E70002015ADF80A000001ADF80C00694800907B
:102E80000121204608F02AFE6946204608F0BFFDD1
:102E90000020C5E710B590B0002004F047FD63485E
:102EA0000068007D40B110B002230121BDE8104050
:102EB0005FA2302004F06EBD5F4C4FF00203B4F807
:102EC000440001281CD05DA20221232004F062FDF1
:102ED00094F82800012817D0E28C5AA168460BF01C
:102EE00061FB022358A20621282004F053FD02238F
:102EF0006A4606215FF0400004F04CFD10B010BDA2
:102F0000022152A22720E1E7B4F829204DA108A808
:102F10000BF048FBE28C4FA168460BF043FB01230A
:102F20004FA20621162004F035FD012308AA062130
:102F3000232004F02FFD012306216A463B20DBE716
:102F400000B589B0002004F0F1FC3B483DA1C28CE3
:102F500068460BF027FB00221146102004F082FD8A
:102F600001220021202004F07DFD022200213020DA
:102F700004F078FD03220021402004F073FD0223B9
:102F800038A20021512004F005FD08220221202052
:102F900004F068FD09220221302004F063FD0223C1
:102FA00029A21946402004F0F5FC02236A4619467E
:102FB000582004F0EFFC09B000BD10B588B00446FD
:102FC00010F1FF4F27D2202168460AF04CF927481C
:102FD0002749844202DD2748844208DC20460AF063
:102FE00045FA0AF030FD0B46024623A10AE02448C8
:102FF0008442F3DC20460AF039FA0AF024FD0B463D
:10300000024620A168460BF0CDFA01236A4606214C
:103010004B2004F0BFFC08B010BD0000000C0140C4
:1030200000540040801A0600005800403410002070
:1030300050446F41000000008C0B0020785041206C
:10304000545752002564000049443A00504120542E
:10305000575200005425643A2D2D2D2D206D00006F
:10306000473A000020545752000000000000104171
:103070000000C84200C0794425302E3366000000AD
:10308000003C1C4625302E326600000010B504F0CE
:1030900063FD04F090FD04F0A5FDBDE8104005F0CF
:1030A000D3BE04F0CDBD04F0DDBD00000022C0F8A9
:1030B0004C21C0E95421704770B5D0F84C1104463A
:1030C000D0F850210D4685A0FFF728FC1BE02946CB
:1030D00088A0FFF723FC05EB451688A014F816100E
:1030E000FFF71CFC04EB460687A07178FFF716FC7F
:1030F00087A0FFF713FCB11C87A0FFF70FFC87A088
:10310000FFF70CFC6D1CD4F8540195FBF0F100FBAB
:103110001150D4F850118842D9D1BDE870407FA039
:10312000FFF7FCBB00F5A871D0F84C0106C9491C9B
:1031300091FBF2F302FB1311814201D10120704790
:1031400000207047D0E95310814201D1012070471F
:10315000002070470FB410B50446FFF7E3FF18B125
:10316000002010BC5DF814FBD4F850119DF80C0041
:1031700001EB411104F81100D4F850119DF80D0035
:1031800001EB411104EB41014870D4F850019DF866
:103190000D2000EB401004EB40000DF10E01801CEF
:1031A0000AF048F804F5A87003C8401C90FBF1F23F
:1031B00001FB1200C4F850010120D2E770B50D46A2
:1031C0000446FFF7BFFF08B1002070BDD4F84C01E2
:1031D000422200EB401004EB400128460AF02AF896
:1031E000D4F84C01422100EB401004EB40000AF0FF
:1031F0003AF8D4F84C01D4F85411401C90FBF1F289
:1032000001FB1200C4F84C016878402803D944A09F
:10321000FFF784FBD8E7012070BD30B5002288B0ED
:103220005FF00A03B0FBF3F403FB1404B0FBF3F00C
:1032300030348C54521C0028F4D1885410006B4652
:1032400004D40C5C151A401E5C55FAD5012004E02C
:103250001C5C0D18401C05F8014C9042F8DD08B0CC
:1032600030BD2DE9F04117468846064600241DE092
:10327000305D09F0D9FFC5B23019407809F0D4FFAC
:10328000C0B2392D01D9373D00E0303DE9B23928CF
:1032900001D9373800E03038C0B204EBD47240EACC
:1032A000011008EB6201A41C087024B2BC42DFDBF1
:1032B000BDE8F081F8B515460E46074600240AE041
:1032C0003A5D1CA168460BF06DF906EB4400BDF8B1
:1032D00000100180641CAC42F2DBF8BD512D3E664B
:1032E000726F6E74203A25642C726561723A2025E3
:1032F000640A000069203A2564000000666C61677A
:103300003A256420000000006C656E3A25642000B8
:103310006D7367203A000000257320000A0000004A
:103320006572726F72207175657565206D73670ABD
:1033300000000000253032580000000010B586B0B3
:1033400008F004FD4FF48034204608F018FD08F022
:1033500043FD28B3102007F0E3FF022007F0D0FF61
:10336000002008F071FD002008F07CFDA01108F09D
:1033700072FD601008F08BFD4FF4E011204608F05C
:103380004CFD012008F051FD392008F010FD002807
:10339000FAD0022008F04CFD08F051FD0828FBD1BE
:1033A000684608F095FD06B010BD10B509F0D2FED4
:1033B000FFF7C4FFFFF7CCF9BDE81040FDF76FBE83
:1033C00000F0E5FF204C94F82B0010B1FDF773FEE0
:1033D000FCE702231DA21946132004F0DBFA0223A6
:1033E0001DA20421132004F0D5FA1E4D4FF6FF76DE
:1033F00002E000BFFDF75FFE2868C089B042F9D047
:103400002868007D28B194F82800012812D0A0B1C6
:1034100015E02068A0F52A41AA3910D194F82800B7
:10342000012801D018B10AE000F01EFE07E001F00B
:10343000A8FC04E007F053F901E006F010FDFEE7F8
:10344000FFF7B3FFFFF7BCFF8C0B0020506C6561EA
:1034500073652053656E6400415420436F6D6D6148
:103460006E64000034100020704730A0FFF756FA59
:1034700033488168491C8160FDF7BDFD00F049F8C3
:1034800030A0FFF74BFA2E48C168491CC160FDF718
:10349000B2FD00F03EF830A0FFF740FA284801697D
:1034A000491C0161FDF7A7FD00F033F82FA0FFF7DD
:1034B00035FA23484169491C4161FDF79CFD00F044
:1034C00028F87047704770472D480168491C016013
:1034D000FFF77EB910B500F02EFFBDE810402020A8
:1034E00007F006BF10B501218C07204609F02DFC1E
:1034F00000280DD00121204609F033FC214908881D
:10350000421C0A80FFF7FFF8BDE81040FFF7C8B97A
:1035100010BDBFF34F8F1C4801681C4A01F4E061E5
:1035200011430160BFF34F8F00BFFDE74861726434
:103530004661756C745F48616E646C65720A000068
:103540008C0B00204D656D4D616E6167655F486154
:103550006E646C65720A00004275734661756C7426
:103560005F48616E646C65720A00000055736167A4
:10357000654661756C745F48616E646C65720A00C3
:1035800030100020061000200CED00E00400FA05C9
:103590002DE9F0418046FC48FC4CD0E90D15A068AF
:1035A00009F0DAFE0746294609F0D6FE01463846FC
:1035B00009F05CFF616806460D46404609F01EFFB3
:1035C000314609F021FF294609F0C6FE054631467D
:1035D0004FF07E5009F012FF394609F015FFC4E99B
:1035E00001502846BDE8F0812DE9F0470646E6483F
:1035F0008A46DFF89883D0E90D14D8F8180009F04E
:10360000ABFE8146214609F0A7FE0146484609F077
:103610002DFFDF4F0546504657F82640214609F05A
:10362000EDFE294609F0F0FE214609F095FE04461C
:1036300029464FF07E5009F0E1FE494609F0E4FECC
:10364000C8F8180047F826402046BDE8F0872DE965
:10365000F0430546CFA09BB0026800928088ADF889
:1036600004005B208DF806006868CDF80700288804
:10367000ADF80B00B1F8C001ADF80D00A8788DF8D9
:103680000F00287AC04F8DF8100000244FEA0D0873
:1036900005EB440008EB8406408900EB8000400005
:1036A000C6F81100398E79B10AF0C9F8DFF8EC924A
:1036B000494609F0DBFE01462046FFF795FF4946E3
:1036C00009F0A2FE0AF01DF9641CC6F83200082CAD
:1036D000DEDB388E00B101208DF8310000208DF83E
:1036E00052008DF854008DF853008DF85500CDF838
:1036F0005600CDF85A00CDF85E005B2206216846E0
:10370000FDF74AFE8DF86200A5A065210088ADF89E
:1037100063006846FDF73CFE1BB0BDE8F083F0B5E2
:103720008BB004462C21684609F09DFD002210460E
:10373000134694464FEA0D0104EB43058F18AE7A09
:10374000521C06EB86067600FE71D2B26E898F1887
:1037500006EB8606C6F3D716FE71521CD2B26D89EF
:103760008E1805EB8505C5F3CF35521CF571D2B225
:103770008D18521C5B1C85F807C0D2B2082B01DAE9
:10378000202AD9D3AA228DF8002029228DF80120E1
:1037900002228DF8022022788DF803202288120A56
:1037A0008DF804207F4A1268537C8DF80530B2F8FA
:1037B0001120120A8DF8062055228DF828200022AB
:1037C0008B5C521C1844C0B2272AF9DB8DF8270005
:1037D00029216846FDF7DEFD0BB0F0BD6C482030B6
:1037E00070472DE9F05FDFF8BCB107460D46DBF806
:1037F000000001F59474B1F8D281427DB1F8C001A6
:10380000411CA2B1614AA8B1012816D0022817D0E4
:10381000032818D04FF4EB73042818D0052816D0CD
:103820004FF4F073062812D0072810D010E0B5F836
:10383000CA010FE04FF4AA7007E04FF4D27004E021
:103840004FF4E17001E04FF4E670108000E0138067
:103850000846118897F885204843B5F8F81197F87D
:1038600086600844B5F810120844B5F812120844EE
:10387000110A0E4397F88410120642EA014246EA02
:10388000114697F8831042EA012246EA116617F8BA
:10389000821F42EA01090AF007F800F08BFE10EBE4
:1038A00009004FEA502944F288107141608094F871
:1038B0008400A61C2071401C84F88400B5F8C00167
:1038C000A4F80900A4F80780B5F8C201A4F805001F
:1038D0001B20E07201F0FF0AD7F80620B5F8C011EE
:1038E0004FEA492961B30020C6F80A0095F8D001D3
:1038F000B073DBF800002C49B0F81100A6F80F00F7
:1039000008EBC80005EB80000B36D0F86C0209F01C
:103910007BFD0AF00FF8F080152024F8680B0122D7
:10392000A2760020E076217F491C21774FEA1921F9
:10393000627741EA0A61C4E90910A085BDE8F09FF9
:10394000B5F8C81108F0FF00B2FBF1F301FB132238
:10395000B5F8C4315843801A4A0852428242C3DD46
:103960000844C1E770472DE9F04F0546B0F9000063
:1039700005278FB00C460D281AD0152818D07028AE
:1039800016D0102112E000008C0B0020081000203F
:1039900018180020436D644D3A34000000007A444A
:1039A0000D0A0000341000200000C842FCA006E010
:1039B0006888A0F58241883904D01021FDA0FDF768
:1039C000DCFC46E1E87A1A2804D01B28F9D01C2830
:1039D000F7D13EE0287B84F8D001B5F80900A4F8BF
:1039E000D201D5F88200C4F8D80195F8860084F891
:1039F000DC0121462846FFF7F4FE04F59475002704
:103A000003F042FA28880022A91C02F00BFA0022D7
:103A10002888114602F02DFAD5F88C0008B103F081
:103A2000C1F995F88500800707D5D5F8900003F017
:103A300047F8B5F8940003F091FA95F8850003F083
:103A4000B6F918B101271021DFA0B8E706202060E1
:103A5000FFE0E249B5F86E000968B1F8111088423C
:103A60007DD1B5F80990B4F8D2114945F8D195F84F
:103A70005D10B4F8C001C140C90770D0297B94F82B
:103A8000D0219142ECD1D5F88210C4F8E81195F814
:103A9000861084F8EC11D5F80DC0D5F8118005EB2F
:103AA000C000CDF8348050F815EF09EBC90140682B
:103AB00004EB81060590D5F85920D5F85510CDE9CD
:103AC0000A12D4E97810D4E976380893D4E97A3226
:103AD0008246C3460693DDF834800598BEEB0C039E
:103AE00060EB0800C0B2CDE90C30089B0B27CB1A65
:103AF0006AEB0B009B46069BC0B2591A62EB0A02A6
:103B00000990D0B28A46DDE90A2107900598B2EB08
:103B10000E0861EB0001C8B2059006F51476584610
:103B2000099909F09AFE02904046059909F095FE20
:103B3000029909F069FC02905046079909F08DFE40
:103B40000490DDE90C0109F088FE049909F05CFCA1
:103B5000029909F053FC02905846099900E077E079
:103B600009F07BFE83465046079909F076FE5946D8
:103B700009F0F2FB82464046059909F06EFE804648
:103B8000DDE90C0109F069FE414609F0E5FB01465B
:103B9000504609F0E1FB0146029809F067FC09F084
:103BA000B0FE09F04CFE09F04EFF8D4A8D4B09F036
:103BB0004EFD09F08BFFDFF830820490D8F840000A
:103BC00009F041FF82468B46D8F83C0009F03BFFE4
:103BD00080460391049809F036FF0022834B09F0D8
:103BE00036FD4246039B09F032FD52465B4609F022
:103BF00087FC09F06BFF7E4909F038FCF061FFF7A4
:103C0000C7FC3062A6F80090287BB07000F074FA10
:103C1000706095F85D003081102205F15E0106F1BB
:103C20000A0009F007FB21463046FFF710FD214648
:103C30003046FFF774FDB9F1000F0AD16D49F06904
:103C400009F0E2FBFFF7B9F96B49F069086000E0A1
:103C500006270FB03846BDE8F08F70B5674D05F503
:103C6000947495F8AA0101280BD104F1860002F0A2
:103C700008FDD4F88600C5F8E00194F88A0085F8BC
:103C8000E401012084F8830070BDF8B55B4D074660
:103C900095F82401D5F82061801BC043C00720D0CF
:103CA000684602F0A7F9C6EBC60000EB800005EB02
:103CB0008004083400F020FAC4F8880004F182007F
:103CC00002F016FDF8887F2800D37F20208081B283
:103CD0000022A01C02F0F9F80120B043C5F8200131
:103CE000F8BD47A0FEF71AFEF8BD10B5002003F09E
:103CF00035F9BDE81040002003F0ECB810B5002005
:103D000003F02CF9BDE81040002003F0E3B82DE9E2
:103D1000F041044600F038FB0546072621680020E4
:103D200039B1062974D00127072972D0082971D129
:103D3000AFE0E98AA4F8C211E989A4F8C011696862
:103D4000C4F8C411A968C4F8C811A989A4F8CC1191
:103D500095F86A1019B30A21A4F8C4114FF4C87178
:103D6000A4F8CA114FF49651A4F8CC116A8BA4F8A8
:103D7000C621B4F8C4115143A4F8C81184F8D00185
:103D8000FF20A4F8D201288802F041F8688802F0E8
:103D900044F80621002002F00EFDE88A3BE04AE0EC
:103DA00072656376206572726F72206D7367310A77
:103DB0000000000072656376206572726F72206D7C
:103DC0007367320A0000000073656E6420726573C9
:103DD00070206661756C740A0000000034100020C9
:103DE0001329AA153236733F8C0B002000408F40F8
:103DF00000007A440000C84200000020381800206B
:103E0000CAFDD7E9D2E7B3F620B4EDCEF30A00003D
:103E100028E034E058E002F0E7FCE88902F0E9FC31
:103E2000002002F04DFE002003F098F8A88D012834
:103E30000BD001200AE01421A4F8C4114FF44871FA
:103E4000A4F8CA114FF4FA518EE7002001F005FCE6
:103E5000A88D012804D0002001F008FC266033E082
:103E60000320F9E794F8AB11012906D184F8AB01DE
:103E700094F8AA11012900D12660606024E0002096
:103E8000676003F027F8002003F068F8082020603E
:103E90001AE094F82001D4F82451401B00F00100EE
:103EA000002810DDC5EBC50000EB800004EB8000AE
:103EB00021460830FFF757FD00B126606D1C05F064
:103EC0000100C4F8240167606068BDE8F08110B5A6
:103ED000694C002060602046FFF719FF0028FAD0E7
:103EE00010BD00BFFFF7F3FFFDF7E5F8FAE7F0B507
:103EF00087B0614E00F048FA04464FF483513046D3
:103F000009F0B1F9002504F16400356081790746B4
:103F1000B9B10121417085705FF04101A0F809102D
:103F2000817900914178019141790391C17804919F
:103F3000C17A11F00B0F09D0017B0820891C884041
:103F400005E00521417085708121E7E7002002909E
:103F50000D20059006F5F871684600F043FA15202B
:103F6000059006F50471684600F03CFA7020059053
:103F700006F50C71684600F035FA00F0E8F900F03B
:103F80001DF900F0CFF8022000F0C1F84FF4FA76E6
:103F900002F0B9FD0028FBD005E038A0FEF7BEFC1A
:103FA000304600F0B4F8002001F0AFF9401CF4D026
:103FB00084F8715084F86F5005E035A0FEF7AEFC30
:103FC000304600F0A4F8384601F070FD0028F4D126
:103FD00094F86400092819D0324800BF01F0D2FBE0
:103FE000032002F0A3FE0095AFF2EF23AFF20532FB
:103FF000AFF26931AFF29D30019502F073FD0122FD
:104000000021294802F0C4FF07B0F0BD2748E5E7CA
:1040100000B593B0402103A809F025F9244890F891
:104020008200012817D023A124480068B0F811208D
:1040300090F86430CDE900310292C38920A240217A
:1040400003A80AF095FA402803D281B203A8FDF72D
:1040500094F913B000BD26A1E6E710B5FFF747FFBE
:10406000BDE8104000F07EB9FEF714FFFFF7F5FF42
:10407000FFF7CEFFFFF735FF38180020494E4954AF
:10408000204641494C4544202020202000000000CB
:10409000434F4E464947204641494C454420202045
:1040A000202000003810002080D02304441000207D
:1040B0008C0B00203835306B0000000034100020DD
:1040C00049443A256420BDC7C9AB3ABBF9D5BE20E7
:1040D000D0C5B5C03A256420CBD9C2CAA3BA2573CE
:1040E00020206E6F6465D7E9A3BA25640D0A00002D
:1040F000362E384D000000009E48006870479D49EC
:104100000A6810440A68121A002AFBDD7047F6E7B5
:1041100000EB40008100002001E000BF401C88420D
:10412000FBD37047F8B50124ADF8004010208DF89E
:104130000300914E03258DF802506946304607F082
:1041400074FB0121304607F0E0FBADF80040002091
:104150008DF803008DF802506946304607F065FB84
:104160000220FFF7CCFFF8BD30B5844D044685B082
:10417000284607F045FF0021ADF800104FF482708B
:10418000ADF80200ADF808106815ADF80A00ADF8FA
:104190000410ADF80C400720ADF80610ADF80E1075
:1041A000ADF810006946284607F04EFF0121284669
:1041B00007F0C7FF05B030BD2020D5E70020D3E7CA
:1041C00010B56D4C1021204607F09FFB0120FFF732
:1041D00096FF1021204607F096FBBDE8104007200F
:1041E0008DE78CE76649024600200968114200D03D
:1041F000012070477FB5012500245F4A0826ADF8ED
:10420000085030B304208DF80B0002A9104607F0C7
:104210000CFB0021084607F0C0FB8DF804408DF828
:10422000056000958DF80650684607F003F84FF4D6
:10423000407006F0B5FE06208DF80C000F208DF8BA
:104240000D008DF80E408DF80F5003A806F0ADFE5E
:104250007FBD8DF80B4003208DF80A0002A910469F
:1042600007F0E3FA8DF804408DF8056000958DF8AD
:104270000640684606F0DEFF7FBD2DE9F041984616
:1042800015460F460646002400F085FE02463A48D1
:10429000102314300360394806E0395D81810189BB
:1042A000C907FCD08189641CB442F6DB002107E019
:1042B00018F8014084810489E407FCD08489491CF2
:1042C000A942F5D32C4810300360104600F074FE6C
:1042D0000020BDE8F0812DE9F0411D4616468846D4
:1042E0000746002400F057FE0246234810231430EE
:1042F0000360224809E000BF18F804108181018999
:10430000C907FCD081892970641CBC42F4DB002100
:104310000C4606E084810789FF07FCD087896F542B
:10432000491CB142F6D3144810300360104600F027
:1043300043FE0020CDE710B5124C01E002F0ECFB8B
:104340002021204607F0CBFA0028F7D110BD4FF00E
:10435000E0214FF40000C1F88001BFF34F8FBFF39D
:104360006F8F70474FF0E0214FF40000C1F800015B
:10437000704700003010002000080140003001406C
:1043800000040140000C01400E480068704738B539
:104390000C490D48A0F118040860B4F85E000090C4
:1043A000B4F85C3034F94A2F0848B4F90210FEF72B
:1043B000B5FAB4F84220B4F84010BDE8384004A083
:1043C000FEF7ACBA34100020A40B002080120108C4
:1043D000736C6F743A25642C616464723A253034CE
:1043E000580A00002DE9F04706460C464FF0000839
:1043F000406909F048FA032209F00AFA0F46054617
:104400000022604B09F095F909F060FB0BF06CF8A5
:1044100009F019FB00225C4B09F019F90B46024622
:104420002846394609F06CF809F050FB574F3168BF
:1044300011B101294BD101E0554900E0554908F07F
:10444000E3FF8146F06802280DD00820824670689C
:104450000E283CD2DFE800F03B1D11093B1A0F3B50
:104460003B170C3B3B141020F0E74FF08B4512E05C
:104470004FF08A450FE0484D0DE04FF089450AE0C6
:104480004FF0884507E04FF0874504E04FF0864540
:1044900001E04FF08545B06800280DDD09F0CFF947
:1044A00009F0D1FA3D4A3E4B09F0D1F8012209F05A
:1044B000AFF909F00BFB80463069092809DA50464C
:1044C00009F0BDF9294608F047FF36490AE0AFF385
:1044D0000080192809DA504609F0B1F9294608F098
:1044E0003BFF314908F090FF0546284609F022FAC3
:1044F0002080404609F01EFA60802C4E2C4809F0BE
:1045000019FAA0803146484608F0B0FF09F012FAC7
:10451000E0803946484608F01FFF314608F0A6FF04
:1045200009F008FA80B2208109F092F90646414666
:10453000284608F011FF314608F00EFF09F0FAF99D
:1045400080B2608109F0B0F900F054F809F025FA62
:10455000A081608909F0A8F900F02CF8C4E90401F1
:10456000227C2276020A42EA01626276020C42EA68
:104570000142000EA27640EA0120E076207D2077FD
:10458000BDE8F08700A0744000004840E144A84620
:104590007B348044C33500430000C0440D71AC8BB4
:1045A000DB68E03FEA5B7E3FB341823F00007A4434
:1045B000B94EAC4110B52C4A2C4B09F0BAF8002288
:1045C0002B4B09F0B6F8BDE8104009F024BA10B53D
:1045D00009F08BF9BDE81040234A244B09F037B8A5
:1045E00010B5214A214B09F0A4F809F014FA01F0A2
:1045F0000F0110BD1F4A204B09F09BB8417919B13A
:10460000012901D0022901D0092100E011214278BD
:104610000E2A16D2DFE802F015070C1515070C1547
:1046200015070C151507130940229A40114406E09E
:1046300013094FF400729A40114401F5007109B258
:1046400001E001F580518078012807D0022807D0C9
:10465000032801D0083904E0091F02E0103900E006
:10466000203908B270470000FA48CE3B1835B13DFA
:1046700080842E410D71AC8BDB68F03FF9487047A8
:104680002DE9F041044690F8D101401E40B284F873
:10469000D101002805DA002901D003202060BDE8FF
:1046A000F081D4E97856B4F8CA11C0F10800484343
:1046B00009F0E9F8FFF77EFF401941EB0607450ACC
:1046C000B4F86A02B4F848126D020844963009F052
:1046D000EBF8FFF78FFF09F060F986B2280A40EA8D
:1046E000076002F05FFB304602F038FC012002F068
:1046F000F1FB0820D2E770B50446002502F0C4FBA8
:1047000020880022A11C01F08DFB00222088114688
:1047100001F0AFFBD4F88C0008B102F043FB94F831
:104720008500800707D5D4F8900002F0C9F9B4F8E5
:10473000940002F013FCD4F88C0000B1012094F82E
:104740008510084302F033FB00B10125284670BDF7
:1047500070B5C44C04F5947504F5D77001F091FF61
:1047600095F8820088B9082084F8D101002084F8E7
:10477000D201D5F88600C4F8E00195F88A0084F8E3
:10478000E40100212046FFF77BFF012085F883002C
:1047900070BDF8B5B34D074695F82401D5F82061F2
:1047A000801BC043C00727D0684601F023FCC6EB3E
:1047B000C60000EB800005EB80040834FFF79CFC8A
:1047C000C4F8880004F1820001F092FFF8887F2885
:1047D00000D37F20208081B20022A01C01F075FB55
:1047E0000120B043C5F8200195F8AA01002803D1A3
:1047F00000212846FFF744FFF8BD9A4890F8AA1117
:10480000002901D101213BE77047F6E730B50446A6
:1048100095A09BB0016800918088ADF804005B20F2
:104820008DF80600FFF768FCCDF80700B4F8C0016A
:104830000021ADF80B00ADF80D1094F8D0018DF803
:104840000F0094F8D2018DF810000A464FEA0D05CA
:1048500004EB4200B0F8860100EB8000430005EB5A
:104860008200521CC0F81130C0F83230082AEFDB49
:104870008DF852108DF854108DF831108DF85310BA
:104880008DF85510CDF85610CDF85A10CDF85E10B1
:104890005B2206216846FCF77FFD8DF8620074A05C
:1048A00065210088ADF863006846FCF771FD65215D
:1048B0006846FCF76DFD1BB030BDF0B58BB004460B
:1048C0002C21684608F0CFFC00221046134694467F
:1048D0004FEA0D0104EB43058F1895F88661521CD1
:1048E00006EB86067600FE70D2B2B5F886618F18A8
:1048F00006EB8606C6F3D716FE70521CD2B2B5F888
:1049000086518E1805EB8505C5F3CF35521CF57021
:10491000D2B28D18521C5B1C85F803C0D2B2082B92
:1049200001DA202AD6D3AA228DF8002029228DF878
:10493000012002228DF8022055228DF82820002225
:104940008B5C521C1844C0B2272AF9DB8DF8270073
:1049500029216846FCF71EFD0BB0F0BD2DE9F0479C
:104960000446FFF711FD21680646052700254FF094
:10497000060904F594704FF001080A2960D2DFE8B7
:1049800001F005795FA85FF0CD5FF762F08AA4F8C7
:10499000C201F089A4F8C0017068C4F8C401B0680D
:1049A000C4F8C801B089A4F8CC0196F86A0080B3B5
:1049B0000A20A4F8C4014FF4C870A4F8CA014FF447
:1049C000965000BFA4F8CC01708BA4F8C601B4F8CF
:1049D000C4114143A4F8C81184F8D05184F8D151CE
:1049E00084F8D251C4F8D451308801F010FA70889C
:1049F00001F013FA0621002001F0DDFEF08A01F03B
:104A0000F3FEF08901F0F5FEB08D01280CD00120F5
:104A10000BE0FFE71420A4F8C4014FF44870A4F899
:104A2000CA014FF4FA50CDE7002000F016FEB08D19
:104A3000012806D05FF0000000F018FEC4F80080E6
:104A4000AEE00320F8E794F831020A2802D0C4F857
:104A50000480A5E084F8315284F83052C4E900851E
:104A60009EE0000098280020436D644D3A34000019
:104A70000D0A0000811C44F2881221F8012B90F8E5
:104A800084204A70B4F8C021CA804FF6FF728A8031
:104A9000B4F8C2214A801A220A7294F8D021521C1A
:104AA00084F8D0214A720D2120F8681B8576C576DE
:104AB000017F491C0177457745628562FD498585FF
:104AC00068380D804D80FFF716FE20B3FAA02760EE
:104AD0000CE094F8D21161B10546214600F059F975
:104AE0002846FFF708FEB0B1F7A02760FDF716FFD4
:104AF00056E04FF0E0264FF400052760C6F88051DD
:104B000006F5C076BFF34F8FBFF36F8F02F0BCF98D
:104B100046F8805C44E0C4F8009041E094F8AB01B2
:104B200001281AD184F8AB5194F8AA01082610B1D3
:104B3000022812D101E026600FE020462760FFF72F
:104B400065FE2046FFF7B9FE84F8D16184F8D251A2
:104B5000102104F5C37008F086FB656020E007E0D3
:104B6000FFE7092020600220606084F8308217E0AF
:104B700094F82001D4F82451401B00F001000028D3
:104B80000EDDC5EBC50000EB800004EB8000214684
:104B9000083000F054F96D1C05F00100C4F8240140
:104BA0006068BDE8F08770B5CB4C00256560204695
:104BB000FFF7D4FE0028FAD0022813D094F832026E
:104BC00001280ED1FFF798FAD4F83812884208D39A
:104BD00084F832520A2084F83102FFF78DFAC4F8C3
:104BE0003C0270BDFFF7D0FBB4F8C811D4F8D40173
:104BF0000844C4F83402D4F83C120844C4F838021B
:104C0000012084F83202C4F8D451DBE7FFF7CBFF70
:104C1000FCF751FAFAE7F0B587B0AF4FFFF7B4FBF6
:104C200005464FF42871384608F01DFB002605F1B3
:104C300064043E60A079E0B301216170A670412157
:104C4000A4F80910A0790090607801906079039031
:104C5000E0780490E07A10F00B0003D0217B08206C
:104C6000891C884002900D20059007F51071684658
:104C7000FFF7B8FB1520059007F518716846FFF798
:104C8000B1FB7020059007F520716846FFF7AAFB7D
:104C9000FFF75DFBFFF792FAFFF744FA0220FFF7F8
:104CA00036FA4FF4FA7700BF01F02DFF0028FBD051
:104CB0000BE0FFE705216170A6708121C0E787A0A6
:104CC000FDF72CFE3846FFF722FA002000F01DFB0E
:104CD000401CF4D085F86F6005E085A0FDF71EFE4E
:104CE0003846FFF714FA204600F0E0FE0028F4D121
:104CF00095F86400092819D0824800BF00F042FDF1
:104D0000032002F013F80096AFF20153AFF21552F0
:104D1000AFF28151AFF2C750019601F0E3FE0122DC
:104D20000021794802F034F907B0F0BD7748E5E793
:104D300000B593B0402102A808F095FA744890F8A5
:104D40008200012814D073A07449096891F8642086
:104D5000CDE90020CB8972A2402102A809F008FC0D
:104D6000402803D281B202A8FCF707FB13B000BDB4
:104D700074A0E9E710B5FFF74EFFBDE81040FFF75C
:104D8000F1BAFEF787F8FFF7F5FFFFF7D1FFFFF75E
:104D90003DFF2DE9F0410D460446D5E97878B1F89C
:104DA000CC0101F5E07508F07FFDFFF703FCC019A9
:104DB00041EB08064FEA5028A71C44F2881027F858
:104DC000020B94F8840007F8010B2888B8804FF68E
:104DD000FF707880688838801C20B871287CF87152
:104DE000D5E90801B860F9604FEA4828A889683415
:104DF00008F05AFDFFF7DEFB484A1268538800228C
:104E0000C018D5E9083C5141C01841EB0C01386588
:104E10007965A87C87F85800702024F8680C022077
:104E2000A076E276207F401C2077012060774FEA51
:104E3000182040EA0660C4E90902A2852FE4F0B513
:104E4000C27A1B2A35D10288152A32D1194B821C0D
:104E500001255C881CB9B2F80F401C805D80B2F857
:104E60000F401B889C4224D1B2F80530B1F8C041F4
:104E7000A3421ED1937B91F8D041A34219D1B2F83D
:104E8000076001F5947306F007043EB9D2F80A6092
:104E9000C1F8D461B2F80F60A1F8D86191F8D2617D
:104EA000A5402E4381F8D26101EBC40600F18005D4
:104EB0004CE065E05E100020B7A2CBCD706F6C6C4B
:104EC000CAA7B0DC0A000000B7A2CBCD66696E614C
:104ED0006CCAA7B0DC0A000098280020494E49544B
:104EE000204641494C45442020202020000000005D
:104EF000434F4E464947204641494C4544202020D7
:104F0000202000003810002080D02304441000200E
:104F10008C0B00203835306B00000000341000206E
:104F200049443A256420BDC7C9AB3AB1EAC7A920B4
:104F3000D0C5B5C03A256420CBD9C2CAA3BA25735F
:104F40000D0A0000362E384D0000000050F8827F18
:104F5000C6F8E871007986F8EC019B1C03EBC400ED
:104F6000D5F80260C0F81360AD79C57503EB440451
:104F7000B2F81100A4F85C00B2F80F00A3F86C00BE
:104F800091F9D101401C05D191F8AA01002801D165
:104F900003200860F0BD10B51720FFF723F90028A3
:104FA00009D04FF0E0224FF40001C2F88011BFF3A6
:104FB0004F8FBFF36F8F10BD002805D04FF0E02159
:104FC0004FF40000C1F80001704700004FF480204A
:104FD000704710B14FF0FF307047FF49FD4808603F
:104FE0000020704738B50024009400F018F838BD50
:104FF00008B589B26B460122FFF7F4FF9DF8000067
:1050000008BD30B5F34D00230446403503E0E05CB5
:1050100050405B1C2A5C8B42F9DB104630BD2DE909
:10502000F843064617463144C1F3044208989846AF
:1050300001F07F011F2A27D87F2925D8B7F5445FC3
:1050400022D24FF4004C48F2010360450AD048B127
:10505000984207D0A0F50044023C03D0A0F50044DC
:10506000033C11D1520242EA810240EA0204240ABE
:1050700000F003058DF8004015438DF801500FB185
:1050800051B10CE0604501D0AFF30080812141EACD
:1050900046018DF8001012E060450ED068B144F072
:1050A00040018DF800100224C11ACB4D98420DD05A
:1050B00007DC20B3604508D108E08DF800400124EA
:1050C000F2E7012902D0022900D0FEE72868007D1E
:1050D00070B1002221466846FFF793FF0246394629
:1050E0004046FFF78EFFBDA0FDF718FCBDE8F88332
:1050F00043463A4669462046FFF7BFF8F6E743467F
:105100003A4669462046FFF7E6F82868007D0228FF
:10511000ECD1182EEAD0002221466846FFF771FF35
:10512000024639464046FFF76CFF0446002118202E
:10513000FFF75EFF8442D9D02868406A0028D5D0A6
:105140008047D3E738B54FF400440094FFF767FF7A
:1051500038BDFFF735B838B5002489B26B46042254
:10516000FFF740FF03216846425C491E02EB04241E
:10517000FAD5204638BD08B589B26B460222FFF742
:1051800031FF9DF800009DF8011000EB012080B276
:1051900008BD38B500236C46E254120A5B1C042B90
:1051A000FADB89B223460422FFF7CCFF38BD08B5ED
:1051B00089B28DF80020120A8DF801206B46022278
:1051C000FFF7C0FF08BD07B589B202AB0122FFF7A8
:1051D000B9FF0EBD3EB5140A8DF804208DF80540C8
:1051E000140C8DF80640120E8DF807208DF808304B
:1051F0001A0A8DF809201A0C8DF80A201A0E8DF85B
:105200000B2048F20302009289B201AB0822FFF79B
:1052100006FF3EBD1CB589B28DF80420120A8DF838
:1052200005208DF806301A0A8DF8072048F2020290
:10523000009201AB0422FFF7F2FE1CBD1CB589B23F
:105240008DF8042048F201028DF80530009201AB80
:105250000222FFF7E4FE1CBD2DE9F0415E4D0E4633
:1052600004001FD04023FF2200211020FFF7E6FF9B
:10527000022C01D128684662564E00220723403690
:10528000D1B208200F0602D583EA410100E04900AF
:10529000401EC9B210F0FF00F4D1B154521CFF2AD5
:1052A000EEDD05E00023BF2219461020FFF7C6FF00
:1052B00028680475BDE8F08170B54F4D04460122A1
:1052C00000212846FFF773FF22460021281FFFF721
:1052D0006EFF022200212846FFF769FFBDE87040FB
:1052E00045480021083036E70021084633E710B56D
:1052F000FFF7FAFF4149884205D0404910398842FA
:1053000001D0881710BD002010BD2DE9F041324CAE
:105310000646002520680221C57301820575457582
:105320008572C5728562C56205634563C563856321
:10533000FFF7DDFF08B1681EBCE70420FFF7BCFFE4
:1053400080460520FFF7B8FF07460A20FFF7B4FFA5
:10535000C0F304412068B8F1000F017203D017B107
:1053600009B102F023F92020FFF7A6FF2449884263
:1053700003D121680120487201E020684572F006DF
:1053800004D40620FFF798FF21680860B00604D413
:105390000720FFF791FF21684860700604D50820B8
:1053A000FFF78AFF21688872300604D50920FFF7CD
:1053B00083FF2168C8722068C17A09B98521C1724A
:1053C000817A09B9742181721F20FFF775FF216866
:1053D000487317E0382B0020641000204E4F4E45D4
:1053E00020535049207772697465746F73706977C0
:1053F0006974686372630A0008000B001203CADE56
:10540000400200101E20FFF757FF10F07F012068B8
:10541000817301D12E218173CAB20021FE48FFF7AA
:10542000D2FE002046E710B51E20FFF745FF00F032
:105430007F0010BD40E770B5044680B240F40072B2
:105440004FF4302500212846FFF7B1FEA2B22846CE
:10545000BDE870400021AAE62DE9F047DFF8BC83E3
:105460000E46044600214046FFF775FE82464FF483
:1054700070434FF0FF3200214046FFF7ABFEDFF8EC
:10548000A093182200214846FFF791FE2520FFF740
:10549000D2FF0220FFF7CFFF4FF4FE70FFF7CBFFE4
:1054A000F0B240F48070FFF7C6FF4FF480763046CC
:1054B000FFF7C1FF0020FFF7BEFF0220FFF7BBFF91
:1054C0004FF4E070FFF7B7FF46EA146060F30F0592
:1054D000C4F3074040F48077C4F3072040F480769B
:1054E000E0B240F48070FFF7A6FF3046FFF7A3FF5D
:1054F0003846FFF7A0FF28B2FFF79DFF0020FFF717
:105500009AFF3A20FFF797FF40F2FF10FFF793FF53
:105510004FF48570FFF78FFF0020FFF78CFF3A20D4
:10552000FFF789FF40F20110FFF785FF4FF43024A9
:10553000022200212046FFF73AFE002211462046B3
:10554000FFF735FE0220FEF74CFE3A20FFF773FF0F
:105550004FF48170FFF76FFF022200212046FFF712
:1055600026FE002211462046FFF721FE00221146AA
:105570004846FFF71CFE52464046BDE8F047002172
:1055800007E670B50D460446FFF766FF2846FFF7AD
:1055900093FEA04201D1002070BD4FF0FF3070BDDE
:1055A0002DE9F041074615460E464FF0FF30002426
:1055B00008E0381981B256F82400FFF7E2FF00280E
:1055C00002D1641CAC42F4DB74E62DE9F041954C49
:1055D000012818D0271F25056FF48076022819D0DE
:1055E0000123FF2200213846FFF728FE2B463246D2
:1055F00000212046FFF7EEFD00237F2202212046F6
:10560000BDE8F0411AE6052001F0F7FF0123FF2273
:105610001946F4E70323FF2200213846FFF70EFE68
:105620002B46324600212046FFF7D4FD00237F227F
:1056300002212046FFF702FEBDE8F041052001F0FF
:10564000DCBF784800214FF480334FF0FF32001F59
:10565000C0E575480068407B7047724B083308B15D
:10566000724A00E0724A0221184692E570B504467B
:105670004FF4A02500212846FFF76DFD6D4900EA93
:105680000102E00701D042F48022A00701D542F4D4
:105690001042600701D542F012022846BDE8704072
:1056A000002176E55D4800212838A1E45E480068C5
:1056B000807A70475C480068C07A70475A48006832
:1056C0000068704758480068406870472DE9F0410D
:1056D000524F0D4606464FF0FF343F1D4FF0082352
:1056E000224600213846FFF775FD4FF06013224631
:1056F00000213846FFF76EFD4FF4E020052E0DD057
:105700004D4B22460021FFF765FD002D08D0BDE876
:10571000F04142480021494A30383AE5484BF0E729
:10572000C8E570B504460D46012001F066FF002172
:105730002846FFF7CBFF284601F08EFFC4F30B028B
:1057400000214048FFF733FD3E4C03230C3CFF2271
:1057500000212046FFF772FD00212046FFF748FC9C
:10576000C007F9D101F072FF002001F056FF0520BB
:1057700001F043FF294800212838FFF739FC00F0E9
:105780003F0070BD70B50446008990B10525002129
:105790002D48FFF72DFCC00700D009252089294698
:1057A000FFF7BFFF6268BDE8704027480021083856
:1057B000EFE41A48227800212838FFF704FDF1E7CA
:1057C00010B50446026800212048FFF7E2FC1F489C
:1057D0000021001D6268FFF7DCFC1C480021083036
:1057E000A268FFF7D6FC1948E2680021BDE8104026
:1057F0000C30CEE410B50446026814480021103085
:10580000FFF7C7FC1148002114306268FFF7C1FCA4
:105810000E48002118301BE0140009004400070066
:1058200008000B0008001100641000207488D204E6
:105830001000D200C00FE0FF001C000200110101A7
:10584000003C00021C000800140001000C000200D3
:10585000A268FFF79EFCE268BDE810400021FD4809
:1058600097E4FC480123FF2200212438E6E42DE9D7
:10587000F04705283FD0FB4EFA4D3F36F64ADFF899
:10588000DC93DFF8DC83F74F77352C460021F648B0
:10589000FFF77FFCF4484A460021001DFFF779FC22
:1058A000F148424600210830FFF773FCEE483A46C3
:1058B00000210C30FFF76DFCEB4832460021103020
:1058C000FFF767FCE8482A4600211430FFF761FC27
:1058D000E548224600211830FFF75BFCE248E34A26
:1058E00000211C38FFF755FCBDE8F047DE480021D9
:1058F000DF4A18384DE4E14FE14DE14CC0377F35C8
:10590000DC4ADFF87493DFF87483DD4EBF34BDE703
:1059100070B5DC4D05242868007A08B101F046FE18
:1059200014220121D848FFF74EFC18220021D74845
:10593000FFF72FFCD548E8220021001DFFF729FCC6
:1059400028686FF4C052007C00F0E001D0482029A4
:1059500002D0602908D102E04FF4806301E04FF4E7
:1059600040630021FFF736FC0021CA48FFF703FC23
:10597000F82101EAD00109390F290ED8C00700D05B
:1059800009242868407A0128204602D0BDE87040EA
:105990006DE7BDE8704001F01DBE70BD10B5044656
:1059A000B8486FF4304200210068447504F00B00E1
:1059B00003031020FFF70EFCE0438107B64805D033
:1059C000B64ABDE810400021FFF7E3BBB44AF8E750
:1059D0002DE9F0419F4AB34F0024273A214638462B
:1059E000FFF7D7FB1023FF2200213846FFF726FCE4
:1059F000DFF8B082002508F11408661E1420FEF7B7
:105A000087FB00214046FFF7F3FA012804D06D1C04
:105A1000EDB2032DF2D33446002211463846FFF78B
:105A2000D2FB012200214046FFF7CDFB0123FF22DC
:105A300002213846FFF702FC9A4800210830FFF7A0
:105A40008AFB6FF06045A84200D13446954800219A
:105A50001030FFF780FBA84200D13446204629E4ED
:105A60002DE9F041884D0446083D01280CD1002164
:105A70002846FFF780FB064640F205134FF6FF72FB
:105A800000212846FFF7C6FBFFF7A2FF0746012CBF
:105A900005D10023324619462846FFF7BBFB38469E
:105AA00008E4024601212820FFF78DBB2DE9F05FB5
:105AB000044690F800800079182802D8E078182869
:105AC00001D9012000E000208346E079012864D05C
:105AD000002082466078012863D004285FD0052822
:105AE00063D007285FD04FF48075DFF89891D9F81C
:105AF0000060308A20F0E0003082E0793073217B52
:105B00000120891C884087B2F80007F0A1FE664991
:105B100007F07AFC07F0F5FE7082E07A7075607B22
:105B2000E17A000401F00B0140EA0133207A2021E0
:105B300001EA4010034343EA0A035C4A00211020B3
:105B4000FFF748FB5FEA0B00594EDFF844B16FF4F2
:105B5000C05A2CD0D9F800004FF440635246018A55
:105B600041F06001018200215846FFF733FB40F20B
:105B700006320021B01FFFF70CFB00221146301F38
:105B8000FFF707FB4B4A00213046FFF702FB7D225F
:105B90000021301DFFF717FB38E0102099E7202582
:105BA000A3E74025A1E748259FE780259DE7E07A08
:105BB000A8B1607B404901281CD0D8B1207B0422C9
:105BC00031F81000102101F059FD00F07F0305EBC2
:105BD000C7054FF6807202213046FFF71BFBFF2DF1
:105BE0000DDDD9F800004FF48063018A41F02001F7
:105BF000018206E0207B032231F81000E2E74FF437
:105C0000A053524600215846FFF7E4FA4FF4C0254E
:105C1000A378FC2200212846FFF710FB7F1EFAB272
:105C200000214FF40030FFF7CEFA607807284DD0FE
:105C30005FF00000FFF735FFE07AC04381071648A8
:105C400046D0164A0021FFF7A4FA124E0021304632
:105C500034E0000028000200FEA8020036AC02007A
:105C6000FEA502003EAF0200380003004002001013
:105C700089A46D1BFDC001003EC40100BEC6010029
:105C800036CF010064100020500007000C001F00F8
:105C900008000B00140001000C0006004C585FAF18
:105CA000CC355FAF0C0004006666663FCF4FFCFF4B
:105CB00012000E000A5A0C00CC020108FFF74BFA42
:105CC0006FF30C00B8F1090F04D005E00820B1E72C
:105CD000F84AB7E740F0010021794FF4F85202EAA0
:105CE00001210143E0780622C00641EA1060617993
:105CF00002EA4102024300213046FFF74AFAA07946
:105D00006178800240EA01336FF47442002124205C
:105D1000FFF760FAB4F8090010B98120A4F809006F
:105D2000B4F8092002212846FFF741FAE2484FF46F
:105D30001025B8F1090F42D0E04A0021FFF729FAF7
:105D400041F63C7200212846FFF731FADA48142266
:105D500001213430FFF737FAD7480E220221001F05
:105D6000FFF731FA81220021D548FFF72CFA0222F1
:105D700000214420FFF727FA0120FFF726FC002529
:105D80000120FEF7C4F900214420FFF731F9800714
:105D900026D52079CB4C09380F282ED8D9F8000009
:105DA000407A012824D04046FFF761FD4FF4C843F4
:105DB00048F2FF1200212046FFF72CFA23E0C24AE6
:105DC0000021FFF7E6F940F63C7200212846FFF774
:105DD000EEF9B948BD4A00210C38FFF7DAF9B5E70A
:105DE0006D1CEDB2062DCBD34FF0FF30BDE8F09F18
:105DF0004FFA88F001F0EEFBD8E70023FE221946A7
:105E00002046FFF71BFABDE8F05F012028E60246B6
:105E100000214FF46020FFF7CAB902460021AC48C8
:105E2000FFF7C5B970B50546501914460E46B0F5D2
:105E3000806F1BD27F2C05D80B462A4621464FF493
:105E4000A0100FE014220021A248FFF7A2F9A148F8
:105E500022460021001DFFF79CF933462A46002107
:105E60004FF4E810FFF76EF9002070BD4FF0FF30DF
:105E700070BD10B5984C7F290AD840EA014040EA2D
:105E8000C22322460021BDE810402420FFF7A2B91A
:105E90004FF4000303EB0141014341EAC2232246D0
:105EA00000212420FFF796F9BDE8104000214FF4AF
:105EB0000020FFF79DB830B414460A462146034639
:105EC00030BC4FF4B010FFF78DB870B5064683486C
:105ED00014460D460068C07B03280BD04FF4901089
:105EE0006119B1F5806F1CD27F2C06D833462A4643
:105EF000214612E04FF49810F2E7020C0021754899
:105F0000FFF747F9734822460021001DFFF741F9CA
:105F100033462A4600214FF4E810BDE87040FFF7F1
:105F200061B870BD2DE9F0416D4E14460D4607462F
:105F300048F240034FF6FF7200213046FFF76AF93E
:105F4000601943F20101884222D87F2C05D83B46D4
:105F50002A4621464FF4A8100FE0152200215D4883
:105F6000FFF717F95B4822460021001DFFF711F9E2
:105F70003B462A4600214FF4E810FFF733F830463D
:105F8000BDE8F041002347F6BF721946FFF742B95A
:105F9000AFF30080514810B50068C07B012808D0DD
:105FA000032802D000214F4805E00C214FF4F010E7
:105FB00001E000214C48FFF7DEF8C0F30C00C104FB
:105FC00001D540F4604000B210BD38B500246B46E6
:105FD000032221464548FFF705F8022069460A5C7E
:105FE000401E02EB0424FAD5E00201D540480443E8
:105FF000204638BD10B5044600213E48FFF7BBF8E7
:10600000C0F30B01080501D541F4704108B23349D2
:1060100020800968B1F91210401A10BD70B5002532
:10602000044601290DD030484FF00C1220302B4986
:106030000968C97B01290ED0032907D00221104627
:106040000AE02948274A28300C3AF0E72A49014457
:106050004FF4F01000E00221FFF78DF8C009208016
:106060000004000C01D04FF0FF35284670BDF0B59C
:106070001A4E0446BBB030684FF4C0176D46C17B62
:1060800001297DD0807D032910D0C1074FF4402025
:1060900005F16C072B4674D06C220021FEF7A2FF9D
:1060A0006C223B4600214FF4502095E101074FF44C
:1060B000F01787E1CC355FAF1C0007003411071CD7
:1060C00008000900180003003400011C33A8B508BB
:1060D0000400010004001F0000F400FC6410002014
:1060E0000400110020000C000C001800290006001C
:1060F0000000F0FF080002000200E8FF2B46E82243
:1061000002E0382200E0202200213846FEF76AFF34
:10611000002029182218097C401C11770628F8DB7A
:10612000BDF80C00C0F30C00A084BDF81600C0F34D
:106130000D006084810402D540F440406084BDF8C5
:106140001C00C0F30B00A4F842003268907D800769
:106150007DD40020291811F8203F235423180E7AEB
:106160001E72097C401C99740528F3DB9DF82200FF
:106170006071BDF82100E0809DF82A00E08101E017
:106180001EE127E1BDF8290020829DF8320020831E
:10619000BDF831006083907D400758D49DF83800E9
:1061A0009DF83B109DF8392040EA01609DF83A10B7
:1061B000090441EA0221084320F0604044F8280F16
:1061C0009DF83C009DF83F109DF83D2040EA01609D
:1061D0009DF83E10090441EA0221084320F00040E6
:1061E00060609DF840009DF843109DF8412040EA12
:1061F00001609DF84210090441EA02210843C0F3FE
:106200001000A0609DF844009DF847109DF84520BF
:1062100040EA01609DF84610090441EA0221084362
:10622000C0F31500E0609DF848009DF84B109DF804
:10623000492040EA01609DF84A10090441EA022120
:106240000843C0F3150020619DF84C0000E0B5E064
:106250009DF84F109DF84D2040EA01609DF84E10CA
:10626000090441EA02210843C0F315006061BDF84A
:106270005C0020839DF86C009DF86F109DF86D20E8
:1062800040EA01609DF86E10090441EA02210843CA
:1062900020F04040E061BDF8700020849DF874005B
:1062A0009DF877109DF8752040EA01609DF8761002
:1062B000090441EA02210843C0F3150060629DF819
:1062C00078009DF87B109DF8792040EA01609DF8E8
:1062D0007A10090441EA02210843C0F31500A062C4
:1062E0009DF87C009DF87F109DF87D2040EA0160BC
:1062F0009DF87E10090441EA02210843C0F315000D
:10630000E062BDF88C00C0F30E002086BDF89C0052
:10631000C0F30B0060869DF8B4009DF8B7109DF89F
:10632000B52040EA01609DF8B610090441EA022157
:10633000084320F040406063BDF8B80020879DF816
:10634000BC009DF8BF1040EA01609DF8BE109DF8AA
:10635000BD20090441EA02210843C0F31500E063AF
:106360009DF8C0009DF8C3109DF8C12040EA01606F
:106370009DF8C210090441EA02210843C0F3150048
:1063800020649DF8C4009DF8C7109DF8C52040EA20
:1063900001609DF8C610090441EA02210843C0F3D8
:1063A00015006064BDF8D400C0F30E00A4F84800E6
:1063B000BDF8E400C0F30B00A4F84A003BB0F0BD08
:1063C000807D01070029FFF699AE40072B467FF537
:1063D0009AAE96E628220021FEF704FE002022183D
:1063E000295C21542918401C0B7A13720B7C93747E
:1063F000097E11770528F2DB9DF81D0084F8210045
:106400009DF807006071BDF80500E0809DF80F0061
:106410009DF80E100843C009E081BDF80D002082F0
:106420009DF817009DF80E100843C0092083BDF8A1
:1064300015006083BDF81E00C0F30D006084810468
:1064400002D540F440406084BDF82000C0F30C0049
:10645000A0849DF824009DF827109DF8252040EA8F
:1064600001609DF82610090441EA0221084320F04A
:106470006040A0623068807DC0079FD09DF82800F2
:106480009DF82B109DF8292040EA01609DF82A1004
:10649000090441EA0221084320F0004044F82C0F8F
:1064A0009DF82C009DF82F109DF82D2040EA0160EA
:1064B0009DF82E10090441EA02210843C0F31000A0
:1064C00060609DF830009DF833109DF8312040EA5F
:1064D00001609DF83210090441EA02210843C0F32B
:1064E0001500A0609DF834009DF837109DF8352008
:1064F00040EA01609DF83610090441EA0221084390
:10650000C0F31500E0609DF838009DF83B109DF841
:10651000392040EA01609DF83A10090441EA02215D
:106520000843C0F315002061BDF84800A082BDF803
:106530005800C0F30B00E0829DF85C009DF85F10EE
:106540009DF85D2040EA01609DF85E10090441EA73
:106550000221084320F04040A061BDF86000A08304
:106560009DF864009DF867109DF8652040EA016081
:106570009DF86610090441EA02210843C0F31500A2
:1065800020629DF868009DF86B109DF8692040EA34
:1065900001609DF86A10090441EA02210843C0F332
:1065A000150060629DF86C009DF86F109DF86D20DD
:1065B00040EA01609DF86E10090441EA0221084397
:1065C000C0F31500A062BDF87C00C0F30E00A085EA
:1065D000BDF88C00C0F30B00E0859DF8A4009DF889
:1065E000A7109DF8A52040EA01609DF8A6100904B7
:1065F00041EA0221084320F040402063BDF8A80092
:10660000A0869DF8AC009DF8AF109DF8AD2040EA43
:1066100001609DF8AE10090441EA02210843C0F36D
:106620001500A0639DF8B0009DF8B3109DF8B1204F
:1066300040EA01609DF8B210090441EA02210843D2
:10664000C0F31500E0639DF8B4009DF8B7109DF805
:10665000B52040EA01609DF8B610090441EA022124
:106660000843C0F315002064BDF8C400C0F30E0059
:10667000A4F84400BDF8D400C0F30B00A4F8460011
:106680009CE60346052200217420FEF7ABBC0121E5
:106690007420FEF760BD00217420FEF75CBDFE484B
:1066A00010B50068C07B012808D0032802D0022161
:1066B000FA4805E016214FF4F01001E00221F848F5
:1066C000FEF759FDC0F30D00810402D540F44040AF
:1066D00000B210BD10B504460346F0480622002162
:1066E000001FFEF77FFC607900F00100607110BDB3
:1066F000E9490968C97B01290BD0032903464FF0FA
:10670000050202D00021642008E004214FF4F010BB
:1067100004E00346E248052200211038FEF762BC7F
:1067200000210170431C04227020FEF75BBCDA4993
:106730000968C97B01290CD0032903464FF00502E3
:1067400003D000214FF4402008E020214FF4F01046
:1067500004E00346D248052200210C30FEF742BC7B
:10676000CD490968C97B01290CD0032903464FF0A4
:10677000050203D0C9480021143808E028214FF44D
:10678000F01004E00346C648052200211430FEF74D
:1067900029BC01216420FEF7DEBC00216420FEF745
:1067A000DABC00211C20FEF7D6BC034604220021DF
:1067B0001C20FEF717BC10B50C4602280CD0002395
:1067C000FE2219461020FEF739FD00220021BDE807
:1067D00010401420FEF7EBBC0123FF220021102003
:1067E000FEF72CFD2246F1E7024602210C20FEF7BF
:1067F000DEBC024600210C20FEF7D9BC034608226D
:1068000000210420FEF79EBC03460822002104203C
:10681000FEF7E8BB10B502460021A248FEF7C7FC10
:10682000A04C8822083C00212046FEF7CCFC002228
:1068300011462046FEF7C7FC0021201DBDE8104090
:10684000FEF7D6BB70B500240D46FF2800D92024E2
:10685000024600219348FEF7AAFC92482A460021EE
:10686000001DFEF7B0FC44F090028E4C0021083C65
:106870002046FEF7A8FC2046BDE8704000221146E5
:10688000FEF7A1BC2DE9F04115460E46074600244F
:1068900006E0381980B2FEF70FFD46F82400641CAC
:1068A000AC42F6DBBDE8F08110B5022805D100232B
:1068B000FE2201217C48FEF7C1FC7A4C0022083CF4
:1068C00011462046FEF77FFC20460222BDE810401C
:1068D0000021FEF778BC10B50446C1B24FF48170B8
:1068E000FFF7B0FF210ABDE8104040F20310A9E70E
:1068F00070B56E4D1023FF2200212846FEF79EFC46
:106900004FF4827600213046FFF79CFF0421304689
:10691000FFF798FF0220FDF764FC4FF48770FFF744
:1069200079FF044640F20F10FFF774FF44EA002499
:1069300000213046FFF786FF0023EF221946284644
:10694000FEF77CFC204670BD10B50C465249096824
:106950000A8A02430A8200214FF42020FEF727FC16
:10696000224650480021BDE810400830FEF72BBCFD
:1069700010B5002211464FF42020FEF718FC4948BC
:10698000002211460830FEF71EFC464C0022083C4F
:1069900011462046FEF717FC20460222BDE81040B3
:1069A0000021FEF710BC30B43F4C20B14FF400631F
:1069B0004FF6FF7202E000234FF2FF72204630BC18
:1069C0000021FEF727BC10B50446C1074FF4602034
:1069D00002D00023EF2201E01023FF220221FEF764
:1069E0002DFC620800213248FEF7EDFB2A480068C2
:1069F000847510BD10B502462D480C460321203881
:106A0000FEF7E1FB4CB10021BDE810404FF48123BB
:106A10004FF0FF321020FEF7DDBB0023BDE8104031
:106A20004FF2FF7219461020FEF7F4BB002310B599
:106A30001A4619461320FEF785FB17480068C17BEC
:106A4000032902D00321C17310BD0121FBE770B5FA
:106A50000E46114900256C1E0A6868B10825002001
:106A6000D0734EB324F480642B462246BDE87040B8
:106A700000211020FEF7AEBB0120D0736FF0080498
:106A8000182200210B48FEF784FB0A48E822002167
:106A9000001DFEF77EFBE4E7641000201C000C00E4
:106AA000140018000C000A0008001100480007003C
:106AB000280001000C001F00FFE745F48065D3E7C4
:106AC00070B5F94D044600212846FEF744FB6FF3EC
:106AD0001300C4F3130202432846BDE870400021AE
:106AE000FEF757BB70B5F14CDDE904562468283435
:106AF00084E86F0070BD10B500214420FEF778FADD
:106B000000F0010010BD10B502214420FEF733FB58
:106B10000004C0F3006010BD2DE9F04700214FF4E0
:106B2000F810FEF765FA064600214420FEF713FB35
:106B3000DE4C054620688561407DC043800703D157
:106B4000A80401D546F00806300628D500214820C3
:106B5000FEF711FB014620688183027D12B1007EA1
:106B6000400702D411F4606F0FD0042200214420AA
:106B7000FEF70FFB4FF4606200214820FEF717FB81
:106B80002068816B09B1183088472068808BC00568
:106B900005D54FF4807200214820FEF708FBF0076E
:106BA00009D0F82200214420FEF70DFB2068816AFD
:106BB00009B11830884770060AD52068C16B09B141
:106BC000183088474FF4C07202214420FEF7EFFAD4
:106BD00030077DD520680027DFF8CC9280F8207040
:106BE000C07BB84609F11C09A0B100214846FEF758
:106BF000FFF92168C97B032900D10009C10701D031
:106C000045F48045810701D545F40055400701D57D
:106C100045F4806520686903856108D590F82010E7
:106C20004FF4802741F0080180F8201007E0690543
:106C300005D590F8201041F0040180F82010E900FB
:106C400007D590F8201047F0805741F0100180F8E8
:106C50002010A90403D5417DC943890709D06904DF
:106C600031D5C07B012817D003280CD000214C203F
:106C70001AE010F8201F47F4004741F002010170AC
:106C800020F8028C1FE0F02200214846FEF79BFA14
:106C900000214FF4F01007E00F2200214846FEF7D4
:106CA00092FA00214FF4C010FEF765FA21680A7BC2
:106CB000B2B3C0F30902CA83000404D511F8200F4F
:106CC00040F001000870002147F4DE42442000E05B
:106CD0000BE0FEF75EFA2068C16A09B118308847F8
:106CE0002068C07B08B1FFF7A1FEF00609D5704A05
:106CF00000214420FEF74DFA2068416B09B118309D
:106D00008847B00610D5222202214420FEF75BFA04
:106D10002068016B002907D0BDE8F047183008470C
:106D2000FFE700F07F02C6E7BDE8F08770B50446D4
:106D3000C107604E6FF47C624FF4A0201FD04FF467
:106D400010730021FEF746FA5A484FF404034FF03F
:106D5000FF3200211238FEF73DFA3513A00700D5A7
:106D6000554D00212A463046FEF713FAA00713D5E9
:106D7000AAB23046BDE870400021FEF70ABA0023EF
:106D80001946FEF727FA3046BDE8704000234FF65B
:106D9000FF621946FEF73EBA70BD02460021302060
:106DA000FEF7F7B9024600212C20FEF7F2B970B5C4
:106DB000002410F0050F03D1010701D4C10648D506
:106DC000C10709D04FF0000380071A46194601D5C4
:106DD0000D2024E0032022E0010709D54FF0000335
:106DE00080071A46194601D50F2018E0072016E043
:106DF000C1064FEA807009D54FF0000300281A46FB
:106E0000194601DA0E200AE0052008E04FF00003E1
:106E100000281A46194601DA102000E00920FEF782
:106E200091F903214420FEF7E3F800074FF0FF3506
:106E300007D421480021E038FEF78DF9B0F5502F36
:106E400020D100231A4619461846FEF77BF92C4636
:106E500018E081064FEA807009D54FF00003002842
:106E60001A46194601DA11200AE00B2008E04FF01B
:106E7000000300281A46194601DA0C2000E0012020
:106E8000FEF760F9204670BD10B5FEF784F80023C8
:106E900004461A4619461846FEF754F92046BDE83E
:106EA0001040FEF789B800000800010064100020BF
:106EB000009005241600110010010F00FE4B20B1B8
:106EC00041EA022020F0F00200E0002200211846F2
:106ED000FEF76DB970B504000CD024F002004FF03D
:106EE000FF3501280DD0042810D008282AD01028FA
:106EF00026D12CE000231A4619460220FEF722F97B
:106F00002AE000231A461946042003E000231A460B
:106F100019460A20FEF716F903214420FEF768F807
:106F2000000719D500231A4619461846FEF70AF934
:106F3000A00705D400231A4619460220FEF702F9DD
:106F4000284670BD00231A4619460820E2E70023B0
:106F50001A4619460620DDE7002070BD10B548B17D
:106F6000024600213420FEF714F94FF400734FF667
:106F7000FF7202E000234FF6FF520021BDE81040EF
:106F80001020FEF747B902460021CC48FEF70FB9A2
:106F90002DE9F04116460C460546FDF7FCFF074675
:106FA000022E12D0012E1BD00023EA4319463C20AA
:106FB000FEF710F90023E24300214020FEF70AF912
:106FC0003846BDE8F041FDF7F7BF2A4600213C20D6
:106FD000FEF7DFF8224600214020FEF7DAF8EFE75F
:106FE0002B464FF0FF352A4600213C20FEF7F2F8F1
:106FF00023462A46E0E770B504464FF47025022286
:1070000000212846FEF7DFF8002C06D02846BDE810
:10701000704001220021FEF7D6B870BD10B50446BD
:107020000021A748FEF797F8C0F30B012180C0F3B9
:107030000B406080A2480021001DFEF78CF8C0F3D1
:107040000B01A180C0F30B40E0809D480021083077
:10705000FEF781F82072000C6072994800210C3014
:10706000FEF779F8C0F30B41A181C0F30B006081FA
:10707000934800211030FEF76EF8C0F30B412182D7
:10708000A0738F4800211430FEF765F8A074000C3F
:10709000E0748B4800211830FEF75DF8C0F30B0058
:1070A000A08210BD10B5FFF763FC0120FDF799F831
:1070B00081480323FF2200211638FEF7BFF8002283
:1070C00011464FF48810FEF77EF80120FDF789F88D
:1070D0007C4801210068C1730021018210BD00F0CD
:1070E0003F0278480021006882737748FEF76BB84A
:1070F00074480068807B704770B504460D460020D8
:10710000FEF7ABFA0F2D00DD0F25601E032800D31C
:1071100004241022E24000216C48FEF73AF8A00057
:10712000001F05FA00F2BDE8704000216848FEF734
:1071300030B810B5044662481023FF2200212030E9
:10714000FEF77CF8042C00D2042422460021BDE87E
:1071500010402C20FEF71DB810B504460121FEF7A3
:10716000B5FA204600F078FA012000F046FA0F2127
:10717000BDE810400120BFE770B50D46044601216F
:107180002846FEF7A3FA284600F066FA012000F030
:1071900034FA2046BDE87040CBE72DE9F0474B4C70
:1071A000002120342046FDF723FF81460223FF22E1
:1071B00000212046FEF742F8444E04220C360021FE
:1071C0003046FEF700F84FF4002801220021404627
:1071D000FDF7F9FF08F1040500212846FDF708FF37
:1071E000C007F9D000214FF00810FDF7C4FFC5B269
:1071F000070A002211464046FDF7E5FF002211462E
:107200003046FDF7E0FF4A4600212046FDF7DBFF50
:1072100045EA072088E52B4910B50968C97A401A64
:1072200006F00DFB2B4906F0EFF8BDE810402A49A7
:1072300006F092B8234910B50968897A401A06F019
:10724000FEFA264906F0E0F8042106F04DF924493B
:1072500006F00CF9BDE81040224906F07DB8012186
:107260004FF00810FDF7C4BE00214FF00810FDF7E5
:10727000BFBE70B504460D46012000F0BEF90021E6
:107280002846FEF723FA284600F0E6F90F4804F0F6
:107290003F0200210C38FDF796FF0D4C0123083CFE
:1072A000FF2200212046FDF7C9FF00212046FDF7FF
:1072B0009FFEC007F9D117E01A0011000400060074
:1072C00004000F00641000201400090028000700CB
:1072D000180008006666863F0000A041CDCCCC3E79
:1072E00000007F43000040400021EC48FDF743FFD1
:1072F000C0F30B0400F0AAF9002000F08EF905207D
:1073000000F07BF9204670BDC179827941EA4201E3
:10731000427941EAC201027941EA8211C27841EA26
:10732000C211827841EA02214278007841EAC22102
:1073300041EA003082B20021D948FDF738BF002170
:1073400018B1FF2101EB5000C1B20846704710B5DB
:1073500004460268D24800212430FDF71AFFD048C5
:10736000002128306268FDF714FFCD4800212C3041
:10737000A268FDF70EFFCA48E2680021BDE8104090
:107380003030FDF706BF2DE9FF470446C07CFF28DB
:107390004AD0C34E361DE9B32068E1896B46827A34
:1073A0008DF80020427A8DF80120027A8DF80220B3
:1073B000C2798DF8032082798DF8042042798DF806
:1073C000052002798DF80620C2788DF80720827892
:1073D0008DF8082042788DF8092002788DF80A206F
:1073E0008DF80C100022090A8DF80B208DF80D1075
:1073F000017B8DF80E10C07A8DF80F00102200214D
:107400003046FDF79FFE227BE089A17C13184FF4E4
:10741000B01600E00BE04FF4A01859B1012912D0CA
:107420006FF0010004B07FE46FF00200FAE70C2275
:107430002368E4E7207C18B14FF48060454608E0FB
:107440007F20354605E0607C10B140F2FF3000E05F
:107450007F20E77CC01B801E984202D24FF0FF3095
:10746000E0E751B9002128466368FDF76BFEE28929
:10747000217B2846A368FDF765FE207C894D012805
:1074800001D0022804D12868C07B032808D001203D
:10749000617C012906D0022904D004290AD00FE01A
:1074A0000220F5E72968C97B032901D0012107E003
:1074B000022105E0E289102A02D96FF00300B1E74A
:1074C00040EA4132764800211430FDF762FE207B0D
:1074D0006FF4FC0100F07F02E08901EAC010024372
:1074E0006F4800211830FDF754FE6D48012200213D
:1074F0001C30FDF768FEDFF8A89109F12009002192
:107500004846FDF775FD074610F0050FF7D03A46DF
:1075100000214846FDF757FE07F03F0727F03000EF
:10752000012825D1A07C012822D1607C012804D02B
:10753000022802D003280AD00AE02868C07B03286A
:1075400002D04FF4901603E04FF4981600E0464640
:1075500063682BB1227B1AB100213046FDF742FD52
:10756000A3682BB1E2891AB1217B3046FDF73AFDC1
:10757000384657E74A4B183B59B1012904D01B1D27
:10758000022906D0032907D1024602211846FDF739
:107590000EBE02460021F9E77047062101EA4003CA
:1075A000CA433F4800211C38FDF714BE10B54FF404
:1075B000C0734FF6FF7200213B48FDF72BFE3948A0
:1075C0004FF6E07200210068037ABDE810403748AA
:1075D000FDF720BE30B4344C6FF40052052808D0BB
:1075E000092808D14FF40153204630BC0021FDF793
:1075F000F1BD4023F8E730BC70472C4B1B3B012802
:1076000007D0052808D14FF4007200211846FDF775
:10761000CEBD41F62202F8E7704710B504460022BD
:1076200011462348FDF7B5FD002211464FF4E02036
:10763000FDF7AFFD002C08D01D480021BDE810402B
:107640004FF0E0523438FDF7A4BD10BD00221848B9
:1076500011464438FDF79DBD30B4154C4FF0FF3254
:10766000443C052807D00928C5D1124B204630BC20
:107670000021FDF7AFBD104BF8E7BCE74843032AF4
:1076800002D1B5214843C009C0F30A01C00A01F57F
:107690008061B1F5006F00D3401C704714000800F2
:1076A000300001006410002008000B001F001100D2
:1076B00048000700001C0002003C000210B5012138
:1076C00086B0480504F056FC0121082004F049FC6E
:1076D000C020ADF8100003208DF812001C208DF89A
:1076E000130004A9F84804F0A0F8F84C204604F070
:1076F0007BF90020ADF804004BF6FF70ADF80600F2
:107700003020ADF808002015ADF80A000001ADF8F2
:107710000C00EF4800900121204604F0DFF9694693
:10772000204604F074F906B010BD2DE9F05FEA4C74
:107730008B46824600272178E64DE4483E460029E4
:1077400071D04FF4003980464946404604F0ACFA07
:1077500050B17F1CAF4204DDE0A0FBF7DFF82670DC
:1077600002E020780028EFD100270121404604F0F4
:10777000D3F9DFF8789309E07F1CAF4204DDDCA089
:10778000FBF7CCF8267007E0207828B14946404640
:1077900004F077FA0028EFD000273A4678214046D7
:1077A00004F001FADFF8589309E07F1CAF4204DDD2
:1077B000D4A0FBF7B3F8267007E0207828B149463B
:1077C000404604F05EFA0028EFD051460027C2463A
:1077D000404604F0E3F9DFF82883A14608F10208E7
:1077E0000BE07F1CAF4205DDCAA0FBF797F889F8D4
:1077F000006008E099F8000028B14146504604F0C6
:1078000040FA0028EDD0002459465746504604F06F
:10781000C5F90CE0641CAC4206DDC2A0FBF77EF8A3
:1078200089F8006009E00EE099F8000028B14146AF
:10783000384604F026FA0028ECD03846BDE8F05F60
:10784000012104F073B9BDE8F09F014600206CE708
:107850000146402069E710B56420FAF7ADFFAE207D
:10786000FFF7F3FF2020FFF7F0FF1020FFF7EDFFF9
:10787000B020FFF7EAFFC820FFF7E7FF0020FFF77F
:10788000E4FF1020FFF7E1FF4020FFF7DEFF81203B
:10789000FFF7DBFFFF20FFF7D8FFA120FFF7D5FFA1
:1078A000A620FFF7D2FFA820FFF7CFFF3F20FFF76A
:1078B000CCFFA420FFF7C9FFD320FFF7C6FF0020AD
:1078C000FFF7C3FFD520FFF7C0FFF020FFF7BDFF94
:1078D000D920FFF7BAFF2220FFF7B7FFDA20FFF722
:1078E000B4FF1220FFF7B1FFDB20FFF7AEFF20202F
:1078F000FFF7ABFF8D20FFF7A8FF1420FFF7A5FFD0
:10790000BDE81040AF20A0E710B50446B031C8B2C2
:10791000FFF79BFF102040EA1410FFF796FF04F0DA
:107920000F00BDE8104040F001008EE770B506463C
:107930005FF0000404F1B000C0B2FFF786FF002042
:10794000FFF783FF1020FFF780FF00253046FFF789
:107950007FFF6D1CEDB2802DF8D3641CE4B2082CBF
:10796000E8D370BD0020E1E710B58D20FFF76DFF73
:107970001420FFF76AFFBDE81040AF2065E710B59F
:107980008D20FFF762FF1020FFF75FFFBDE810407A
:10799000AE205AE72DE9F047002591468A46044675
:1079A000012B22D0DFF88C81022B24D155E0203826
:1079B000C7B27E2C04D90AF10100002400F0FF0AAE
:1079C00051462046FFF7A0FF07EB4700002608EBD3
:1079D0004007B85DFFF73CFF761CF6B2062EF8D3E1
:1079E000A41D6D1CE4B2EDB201E0DFF84C8119F882
:1079F00005000028DBD1BDE8F0872038C7B2782C1D
:107A000004D90AF10100002400F0FF0A5146204683
:107A1000FFF77AFF5FF0000606EB071118F8010088
:107A2000FFF716FF761CF6B2082EF5D30AF1010017
:107A3000C1B22046FFF768FF5FF0000606EB0711B2
:107A400001EB0800007AFFF703FF761CF6B2082E60
:107A5000F4D308346D1CE4B2EDB219F80500002827
:107A6000CBD1C8E72DE9F0410F46804600255401EF
:107A7000FFF74AFF184E761C305DFFF7E9FE6D1CDC
:107A8000EDB2641C102DF7D37F1CF9B24046FFF70E
:107A90003BFF0025305DFFF7DBFE6D1CEDB2641C83
:107AA000102DF7D3BDE8F0812DE9F0479846174631
:107AB000824600260C46DDF820904AE021465046DA
:107AC000FFF722FF554640E0000C01400054004003
:107AD000801A060040420F006810002049494320E8
:107AE0004572726F7220310A00000000010003002D
:107AF000494943204572726F7220320A000000002B
:107B000082000700494943204572726F7220330A90
:107B100000000000494943204572726F7220340A08
:107B200000000000494943204572726F7220350AF7
:107B30000000000002050108DA02010819F8060039
:107B4000761CFFF785FE6D1CEDB2BD42F6D3641CBA
:107B5000E4B24445B2D34EE738B55E494FF4A06471
:107B60002246A1F1200000F0C5F85B492246A1F5AC
:107B7000A26000F0BFF80121082004F0F2F9022011
:107B8000ADF8000003208DF8020010208DF80300EE
:107B90006946524803F049FE4FF48024204603F022
:107BA000A7FB4F4908200C604871012088710846E6
:107BB00003F040FB38BD10B5002004F064F901214A
:107BC000BDE81040C80504F0D5B946490320086057
:107BD00070474548817A434809B1052100E00121F9
:107BE0000160704738B514208DF8000002208DF830
:107BF000010000248DF8024001208DF80300684642
:107C000003F0D3F92A208DF800008DF80140684672
:107C100003F0CBF938BD314A00284FF0020110467D
:107C200001D003F070BE03F070BE10B5FFF794FFF3
:107C3000FFF7C1FFFFF7D6FFBDE8104001F004B920
:107C40000A4601462348203800F072B80A46014629
:107C50002048203800F054B80A4601461D48103824
:107C600000F066B80A4601461A48103800F048B8D5
:107C7000F0B500230A24302537261F4611E000BF47
:107C8000B4EB107F02D905EB107C01E006EB107C11
:107C900001F813C001EB430C00015B1C8CF8017070
:107CA000DBB29342ECD3F0BD104810B50168001D63
:107CB0000468001D006808180AD008220C49FFF764
:107CC000D7FF0B4920460422BDE810401031CFE712
:107CD00010BD0000982C002098310020000C0140BD
:107CE0006C1100207C12002038370020E8F7FF1FBD
:107CF000761100200260C160416081600020704701
:107D000070B5002483680FE0C56806685B1C3544C5
:107D10009D4200D8C36845689D4207D011F8015BB9
:107D2000866835708360641C9442EDD3204670BD34
:107D300030B500230DE04468651C45602478CC54C0
:107D4000C46805682C4445685B1CAC4201D8C46813
:107D5000446045688468A54204D0934202D2046816
:107D60009C42E8D8184630BD10B50021426807E0B3
:107D7000C3680468491C2344521C934200D8C2685B
:107D80008368934202D003688B42F1D8084610BD45
:107D9000F0B54468059E05680AE027788F420CD04C
:107DA000C768D0F800C0641C6744A74200D8C46804
:107DB0008768A74201D06D1EEFD28168A14228D00A
:107DC000691C26D0C768D0F800C0611C674409E070
:107DD000C16809E00F7897420BD0C768D0F800C09F
:107DE000491C67448F42F3D987688F4201D06D1ECA
:107DF000F0D282688A420CD06A1C0AD0C268076836
:107E000017444A1C974200D8C26801684D1B0021E4
:107E10000DE00020F0BD00BF14F8017B5F54C7687F
:107E2000D0F800C0491C6744A74200D8C4689442F7
:107E300006D0B14204D207688F4201D96D1EEBD241
:107E400042600846F0BDF0B54468066809E0257850
:107E50008D420BD0C5680768641C3D44A54200D81C
:107E6000C4688568A54201D0761EF0D28568A54217
:107E700027D0751C25D0C56807682F44651C09E00C
:107E8000C56809E02F788F420BD0C768D0F800C0D2
:107E90006D1C6744AF42F3D98768AF4201D0761EAC
:107EA000F0D28168A9420CD0711C0AD0C168076861
:107EB0006D1C3944A94200D8C56801688E1B002199
:107EC0000DE00020F0BD00BF14F8017B5754C768D7
:107ED000D0F800C0491C6744A74200D8C468AC422F
:107EE00006D0994204D207688F4201D9761EEBD2A0
:107EF000022908DCC2680021641E944203D2C268D1
:107F00000368D418641E44600846F0BDF0B54468A8
:107F1000056809E026788E420BD0C6680768641CA5
:107F20003E44A64200D8C4688668A64201D06D1EB1
:107F3000F0D28168A1420CD06D1C0AD0C1680568DE
:107F4000641C2944A14200D8C46841680668002521
:107F50000DE00020F0BD00BF11F8017B5755C76848
:107F6000D0F800C06D1C67448F4200D8C168A142A0
:107F700003D09D4201D2761EEED241602846F0BD6C
:107F8000F0B54468059E002705680EE0B94202D1AD
:107F9000277897420FD014F8017BD0F80CC0D0F8A6
:107FA00000E0F444A44500D8C468D0F808C0A44553
:107FB00001D06D1EEAD28168A1420CD06D1C0AD09E
:107FC000C1680268641C1144A14200D8C4684168B9
:107FD000056800220DE00020F0BD00BF11F8017B14
:107FE0009F54C768D0F800C0521C67448F4200D825
:107FF000C168A14203D0B24201D26D1EEED24160EF
:108000001046F0BD0360B2FBF3F242600161002153
:108010008160C160084670472DE9F041C568174688
:1080200088460446002614E060686D1C854200D333
:108030000025A068A8420ED02069E168226801FBF3
:1080400002002268414605F0F5F82168E5608844A1
:10805000761CBE42E8D33046BDE8F0812DE9F04100
:10806000002590460E4604462F4612E02069A1687E
:10807000226801FB02012268304605F0DBF8206827
:108080000644A068401CA06061686D1C884200D353
:10809000A760A068E168884204D06068A84201D95E
:1080A0004545E3D32846D7E70021826805E04368C9
:1080B000491C521C9A4200D30022C368934202D04A
:1080C00043688B42F3D808467047000070B5294DCD
:1080D0002878012815D140212748FFF7BDFD040469
:1080E000240C4FF000060DD02246C021224800F09B
:1080F000A1FF2146012001F086F9012001F05CF882
:108100006E6070BD2E7070BD1B4910B540310320EC
:1081100001F02BFB81B218484030FFF797FDBDE816
:108120001040032001F058B870B5144800680528C5
:108130001FD1104C207800281BD16068411C616061
:10814000052816D10020606040210B48FFF784FD10
:1081500005042D0C0DD02A46C021074800F06AFF07
:108160002946012001F04FF9012001F025F80120F6
:10817000207070BD9C110020983600207C120020D9
:108180002DE9F0414C4E88B0002430684B4D68809A
:1081900068884B4F39880840800507D54FF6FF5057
:1081A00030602878401C2870FFF7BEFF6888398847
:1081B0000840000401D500F05BFE688839884FF65E
:1081C000FF380840400504D5C6F800803D484068A7
:1081D0008047698838880140890402D54DF6FF71CF
:1081E000316069880140C80405D54EF6FF703060E3
:1081F000002000F0F0F968883988084000050BD5A8
:108200003148007810B100F082F902E0022000F05D
:10821000E2F94FF2FF703060688839880840C00585
:1082200046D54FF6FF6030602348001D00684FF0D0
:108230000002000438D56868401C6860686803283C
:1082400033D91D48001F016809072ED4016889B27F
:10825000A9601E494FEA0D0301EB8407D7F8007CA3
:10826000BFB243F82470641C082CF5D3AC6844F00A
:108270000104AC60AC68A4B20460AC6824F00104F2
:10828000AC60AC68A4B2046030684005FCD5C6F8A8
:108290000080002053F8204001EB8006A4B2C6F80D
:1082A000004C401C0828F5D36A60072000F093F9C1
:1082B00008B0BDE8F0810000445C0040A41100203B
:1082C000A012002004120020801200200050004064
:1082D000FFF756BF4FF4802003F00AB810B5FFF740
:1082E000E3FC764800240068847200F0F1F801F0A5
:1082F0001DFA7348046010BD704810B50068714ADB
:1083000000218172D2794272C172084600F0D4FE17
:108310004FF40071002000F0E7FE1021002000F073
:10832000F8FE4021002001F04AF88021002001F0F1
:108330003AF8002000F07CFF634890F82C100020F1
:1083400001F07FF8002000F047FF0021012000F03D
:10835000CBFEC021012001F026F82021012000F0F1
:10836000D8FE0021012000F0EAFE4FF4C061022097
:1083700000F0BAFE4FF48071022001F014F80021E1
:10838000022000F0DCFE2021022000F0C2FE0021CD
:10839000032000F0A9FE4FF48871032001F00FF8CC
:1083A0004021032001F04DF84FF44051032000F02C
:1083B000C6FE0021032000F0ACFE002000F084FC8B
:1083C0003F490120086010BD4048807A002802D053
:1083D0003B49052008607047394904200860704710
:1083E00039481C380178202901D1002101707047DB
:1083F000704710B134481838704730490820096870
:1084000008820020704710B12F48183870472B4958
:1084100008200968088200207047284A10B500210A
:108420001268212802D0202808D019E0107800F026
:108430007F00212814D1AFF231010AE0107800F05A
:108440007F00212801D1AFF255011F4B20201C3B9A
:10845000187029B10020916150828847002010BD1A
:10846000022010BD15490968097801F07F01212912
:1084700003D1022803D0222801D002207047002017
:1084800070471149103900F049BA0F49083900F016
:1084900045BA0A490968C978042901D900207047FA
:1084A000094A303202EBC10100F038BA09B901289B
:1084B00001D902207047002070470000941200206C
:1084C0007C120020040B0108041200203837002021
:1084D00010B50120FFF79FFB6248012101600021D8
:1084E000614A0160031D19604FF4E0511180016081
:1084F000002010BD10B55B4C01202060211D002024
:108500000860FFF788FB03202060002010BDF8B54D
:108510005449002000900A68544B554C92B200BF59
:1085200003EB8005D5F8005CADB244F82050401C48
:108530000828F5D342F48060086040F0010008602C
:1085400020F001050D60474A121D10684005FCD55A
:108550004FF6FF301060002054F8206003EB8007D6
:10856000B6B2C7F8006C401C0828F5D345F00800E7
:108570000860086880B240F0040008603D4B18684D
:108580000090186820F0030040F0010018603A489D
:10859000046844F0040404601468E40409D54EF649
:1085A000FF7414600A6892B222F008020A6000990F
:1085B0001960016821F004010160F8BD10B5294C73
:1085C000206880B220F004002060FFF702FB4FF427
:1085D0003F40206010BD2DE9F041284C072800D015
:1085E00020702278254D0627052104261D48062ADD
:1085F0000BD2DFE802F0030C11161E27686810B1D9
:108600002170BDE8F081FFF7D9FF2770F9E7FFF788
:10861000D5FF2670012022E0022060700320207028
:10862000EFE76078401E607060780028E9D126701E
:10863000E7E7026892B242F01002026021700A205D
:108640006070DEE76178491E617061780029D8D1D9
:10865000016889B221F01001016027700020686074
:10866000CFE70000405C0040A01200200050004016
:10867000183700200070004010ED00E08412002048
:1086800010B5FB4C30B1FB4800680068804720689B
:108690000A3010BD216801200882002010BDF44876
:1086A00010B50068F44AC1785278914203D88278B4
:1086B0000AB982880AB1022010BD8172ED480068B3
:1086C00040688047002010BD10B5E94C30B1E94842
:1086D00000688068804720680C3010BD2168012048
:1086E0000882002010BD10B5E14CE44A20681268F1
:1086F000C17892694079904721688A7A22B118B985
:10870000087908B9887808B1022010BDD9480068F6
:10871000C068804720684179C172C1780173002028
:1087200010BDD34910B5096860B1D5480022028058
:108730000A7853060AD002F07F02012A16D0022AD4
:1087400016D001E002200882002010BD497A8A0676
:10875000027802D542F0020201E002F0FD02490671
:108760000270D1B211D401F0FE0110E0C44810BD76
:108770004A7911071306C34A02EB9161D1F8001C34
:1087800007D5C1F3011106E0017841F00101017044
:1087900003E0C1F301310129F6D0B6480068006951
:1087A0008047E3E72DE9F041B1480068017811F016
:1087B0007F0102D0022905D066E0417A01F0DF0195
:1087C00041724EE0418800295ED10179F1BB4179C7
:1087D000AC4D21F080040A0605EB8402A64BD2F8CA
:1087E000002C03D5C2F30112120102E0C2F30132E0
:1087F00012031E782346A64246D93AB3807A28B39C
:1088000008064FEA84000ED52844D0F8000CC0F3C7
:108810000110012821D1184600F09CFD204630218E
:1088200000F077FC19E04619D6F8000CC0F30130CF
:10883000012812D14BF68F7748F28008A4B1184670
:1088400000F076FDD6F8000C384000E01CE080F423
:10885000405040EA0800C6F8000C864800684069AD
:1088600080470020BDE8F081874890F82C10002058
:1088700000F0E7FDD5F8000C384080F4405040EAA5
:108880000800C5F8000CE8E70220EBE770B578486F
:108890007C4D0368597921F0800005EB80000C06BF
:1088A000D0F8004C21F0800203D5C4F30114240158
:1088B00002E0C4F3013424036F4D2D78954210D9A2
:1088C0005A8872B96CB19A7A5AB10906D0F8001C6C
:1088D00048F2800207D548F6BF73194081F01001B5
:1088E00006E0022070BD4BF68F73194081F4805171
:1088F0001143C0F8001C5F48006880698047002071
:1089000070BD5B4810B50068417A41F020014172AA
:1089100058480068C0698047002010BD544A136859
:108920005A8A10B10868104470478888801A1882E3
:10893000002070472DE9F047DFF83481534F4FF0A6
:108940003009D8F8001001F11005088A0E7A08B92C
:10895000042E04D0AC88A04216D8042615E048485E
:10896000801E0178012903D00726102038802BE0D3
:10897000474A00211268474B120403EBD232516080
:10898000A7F8009001701FE00226844200D9044637
:10899000A968204688478246002000F01DFD014658
:1089A0002246504600F046FB2146002000F02BFDF9
:1089B0002888001B2880688820446880A7F80090D9
:1089C00035494FF440500880D8F800000672BDE8E1
:1089D000F08770B5264D2868017844784A0606D09D
:1089E00001F07F00012828D002282BD035E0092C87
:1089F00006D0052C07D0032C0ED0012C14D02CE06F
:108A0000FFF74DFE28E0C1787F292ED8817861BB21
:108A1000818851BB807A27E0C17801291DD18088E7
:108A2000D8B9FFF76EFF17E0C178012915D1818809
:108A300099B9407A80060AD40FE00B2C0DD1FFF7CC
:108A400052FE09E0012C02D0032C03D005E0FFF711
:108A5000A9FE01E0FFF71AFF48B10849204609685E
:108A600049698847032819D008B1082024E017E095
:108A7000941200209C120020541200209812002012
:108A80008E1200200050004004120020A41200208A
:108A9000505C004000600040A212002009200BE062
:108AA000DE4A062000211268DD4B120403EBD232AD
:108AB0005160DC4A302111802968087270BDF8B518
:108AC000D94CDA4D09262068002729684278062A01
:108AD00005D0AAB1082A4ED00A2A52D06EE00278F8
:108AE00052066BD18078012804D0022804D00328D4
:108AF00004D063E0C96959E0096A57E0496A55E062
:108B00004288BABBC288022A58D1027992BB027845
:108B1000530601D1838833B102F07F02012A05D0C8
:108B2000022A0DD04AE0AFF205413FE08A69407960
:108B300000219047F0B92068807A0028F3D13DE009
:108B4000417901F00F0001F070020B06B84901EB0A
:108B50008001D1F8001C03D5C1F30111090102E025
:108B6000C1F301310903B34B1B78834226D90AB9FB
:108B70000029D8D122E0007840061FD1AFF2FF4192
:108B800014E0027802F07F02012A17D1827AAAB19A
:108B900042889AB902798AB9C288012A0ED18A69B3
:108BA00040790021904748B9AFF2E34131B12068E4
:108BB0004782816100208847002006E029682068FC
:108BC000096940788847032813D021680A8AA2F5EA
:108BD0007F43FF3B0BD002280ED06AB10878000615
:108BE00025D5C888009082420AD9088218E00E7202
:108BF000F8BD20680672F8BD4FF008000872F8BD95
:108C00000ED228688C4B90F82C00824201D21F7043
:108C100006E0B2FBF0F400FB142008B90120187044
:108C2000286890F82C008882BDE8F84082E603208E
:108C30000872824900030880F8BD814810B590F899
:108C40002C10002000F0FDFB77480068007A08280F
:108C500002D0092809D006E078494FF480500880F6
:108C6000704910200880002010BD012010BD70B593
:108C70006A4800686C4D0004C10B694801440989C9
:108C800089B200EB41042868017A09290FD02178C4
:108C9000017061784170A08800F03CFD296848802F
:108CA000208900F037FD29688880A089C88028685D
:108CB00001210172C08820B1FFF701FFBDE87040BB
:108CC000BBE7FFF786FEF9E7F0B55A49584D48F67D
:108CD0008F770B78002148F2800C0BE0CEB205EBC9
:108CE0008604D4F8002C3A40324342EA0C02C4F81D
:108CF000002C491C9942F1D3484940F08000091FDB
:108D00000860F0BD10B5484C2068017A022904D0F3
:108D1000042902D0062905D015E0FFF70BFE2068D4
:108D2000007A11E04178052909D10178490606D178
:108D3000C078FFF7C9FF43480068006A80473B4896
:108D4000006880688047082021680872BDE81040EC
:108D500073E710B5344C2068007A022811D004283B
:108D60000FD0032804D0052802D0072805D008E03A
:108D700000F00EF82068007A04E02C480068C06813
:108D80008047082021680872BDE8104055E7704709
:108D90002DE9F047244EDFF88C803027356835F810
:108DA000100FA968A9B100B3AC88844200D9044669
:108DB0002046884781462888001B288068882044F0
:108DC0006880002000F013FB01462246484600F070
:108DD00044F9288848B119494FF4405008800021CF
:108DE000084600F010FBA8F800702888A98888427F
:108DF00001D3032001E018B1052031680872E6E5CF
:108E0000316806200872054900200968044A0904EF
:108E100002EBD1314860A8F80070D8E5505C004002
:108E200000600040A412002094120020981200203C
:108E300000500040541200208C120020A21200208A
:108E4000041200209C1200200648054902220160FD
:108E50000A72064A0449C0E9011208680047000086
:108E600038370020941200200412002058120020ED
:108E70002DE9F84F0020ADF80000DFF89CA14BF67B
:108E8000BF7648F28007644D644C40F68F7848F610
:108E90000F7BDFF88C910AF1440A31E00888614ABF
:108EA00010F00F00107034D05F4901EB8001D1F851
:108EB000002CADF80020BDF8002012040BD5D1F82D
:108EC000002C02EA0802C1F8002C584901EB80008E
:108ED00050F8040C8047BDF80000000610D551483A
:108EE0005149007801EB8001D1F8002C02EA0B0215
:108EF000C1F8002C4E4901EB800050F8040C80476B
:108F0000DAF800004946A9F800000004C6D4BDE81C
:108F1000F88F28682080208800F03000608020884A
:108F200000F4405020802868304080F4005080F0E9
:108F30002000384328600888C006286815D400EA55
:108F40000B002860FFF7DEFE26E02188890401D5AA
:108F500080F400506188C90626D46188890601D54D
:108F600080F0200038432860D1E7ADF80000BDF85C
:108F70000000000506D5286800EA08002860FFF711
:108F800076FE09E0BDF800000004B9D5286800EAC3
:108F900008002860FFF7DDFE286821883040C904FA
:108FA000D3D580F48050D0E780F01000D5E72DE9CC
:108FB000F041194C1B4E1C4F4434194D26E000BFA4
:108FC00047F6FF702060288800F00F0107EB810052
:108FD0003170D0F8002C92B2130408D5D0F8002CD0
:108FE00040F68F731A40C0F8002C104809E01206B2
:108FF0000CD5D0F8002C48F60F731A40C0F8002C9E
:109000000B4800EB810050F8040C80472068288052
:109010000004D5D4BDE8F081005C0040A21200201D
:10902000A61100209012002000500040CC1100201A
:10903000B0110020104B10B5521C520803EB410137
:109040000AD000BF10F8013B521E10F8014B43EA52
:10905000042321F8043BF5D110BD074B521C5208E4
:1090600003EB410106D000BF31F8043B20F8023B7E
:10907000521EF9D17047000000600040FC490860B2
:109080007047FB48006880B27047F949091D0860C5
:109090007047F748001D006880B27047F4480830F8
:1090A000006880B27047F2490C3108607047F048A0
:1090B0000C30006880B27047ED4920F00700103195
:1090C00008607047EA481030006880B27047E94A8B
:1090D00002EB8000C0F8001C7047E64901EB8000FD
:1090E000D0F8000C80B270478200E2480244D2F807
:1090F000000C48F68F1318400843C2F8000C704764
:10910000DC4901EB8000D0F8000CC0F341204002A4
:1091100070478200D7480244D2F8000C48F6BF736B
:109120001840CB0601D580F01000890601D580F0EB
:10913000200048F280010843C2F8000C704782000A
:10914000CC480244D2F8000C4BF68F731840CB0485
:1091500001D580F48050890401D580F4005048F294
:1091600080010843C2F8000C704700B50A46034668
:10917000FFF7B3FF9900BF4B012A194407D0022A19
:1091800004D120F0100000BFC1F8000C00BD20F495
:109190008050F9E7B74901EB8000D0F8000CC0F32C
:1091A000011000017047B34901EB8000D0F8000CBA
:1091B000C0F30130000370478100AE480144D1F88C
:1091C000000C48F6BF72104080F0300048F2800278
:1091D0001043C1F8000C70478100A6480144D1F843
:1091E000000C4BF68F72104080F4405048F2800221
:1091F0001043C1F8000C704781009E480144D1F82B
:10920000000C48F68F72104048F280121043C1F8EB
:10921000000C7047810097480144D1F8000C48F6D3
:109220008F62104048F280021043C1F8000C704772
:10923000810090480144D1F8000C48F68F6210403C
:1092400048F280021043C1F8000C70478100894841
:109250000144D1F8000C48F68F72104048F2801299
:109260001043C1F8000C7047810082480144D1F8D6
:10927000000C48F68F72104048F280121043C1F87B
:10928000000C704781007B480144D1F8000C48F67F
:109290008F62104048F280021043C1F8000C704702
:1092A000744901EB8000D0F8000CC0F301100128D4
:1092B00000D0002070476F4901EB8000D0F8000C0F
:1092C000C0F30130012800D00020704781006948B8
:1092D0000844D0F8001C40F68F721140C0F8001C02
:1092E0007047810063480844D0F8001C48F60F72AC
:1092F0001140C0F8001C704781005E480144D1F85D
:10930000000C48F68F7210404CF280021043C1F8F6
:10931000000C7047810057480144D1F8000C48F612
:109320008F72104048F2C0021043C1F8000C704721
:10933000810050480844D0F8001C490409D5D0F8F1
:10934000001C48F68F7211404CF280021143C0F8A5
:10935000001C7047810047480844D0F8001C4906AB
:1093600009D5D0F8001C48F68F72114048F2C002AF
:109370001143C0F8001C704782003E481044D0F8EA
:10938000002C48F68F731A400A4348F280010A43C2
:10939000C0F8002C7047374901EB8000D0F8000C72
:1093A00000F00F007047324A21F0010110321268BC
:1093B00092B202EBC000304A42F8101070472C4ABB
:1093C00021F001011032126892B202EBC0002A4A69
:1093D00002EB40008160704725491031096889B26D
:1093E00001EBC000244931F8100080B270472049D9
:1093F0001031096889B201EBC0001F4901EB400040
:10940000008980B270471A4A1032126892B202EB99
:10941000C000194A02EB4000416070473E2909D95B
:109420004A09C90601D1521E92B24FF4004141EAE5
:10943000822104E04A08C90700D0521C9102016051
:1094400070470B4A1032126892B202EBC0000A4A0F
:109450000C3202EB40023E2910D94809C90601D15D
:10946000401E80B24FF4004141EA80200BE0000032
:10947000405C004000500040006000404808C907C0
:1094800000D0401C800210607047A549096889B26D
:1094900001EBC000A34901EB40008088C0F3090044
:1094A00070479F49096889B201EBC0009D4901EBF3
:1094B00040008089C0F30900704730B521F00104F5
:1094C00097490B6822F001029BB203EBC0035D00D9
:1094D000944BEC50096889B201EBC00003EB4000EB
:1094E000826030BD8E4A21F00101126892B202EB17
:1094F000C0008C4A42F810107047894A21F00101DF
:10950000126892B202EBC000864A02EB4000816012
:1095100070478349096889B201EBC000814931F87D
:10952000100080B270477E49096889B201EBC00023
:109530007C4901EB4000008980B270472DE9F0437F
:10954000774D012912D002290ED1296889B201EB89
:10955000C0014B0073490B445A602B689BB203EB6C
:10956000C00001EB4000C260BDE8F08329686D4B8C
:1095700089B201EBC0011B1D03EB410C53095108DB
:109580005E1E4C1C4FF400493E2A07D91F465FEA75
:10959000C26800D1B7B249EA872705E00F465FEA03
:1095A000C27800D02746BF02CCF800702D68ADB25B
:1095B00005EBC0005B4D0C3505EB40003E2A05D99C
:1095C000D10600D1B3B249EA832103E0D20700D02B
:1095D000214689020160C7E7514B01290AD00229BF
:1095E00007D1196889B201EBC0004E4901EB400078
:1095F00042607047196889B201EBC0004949091DF2
:1096000001EB40013E2A09D95009D20601D1401E82
:1096100080B24FF4004242EA802004E05008D207B2
:1096200000D0401C8002086070473D4B01290AD0E1
:10963000022907D1196889B201EBC000394901EB51
:109640004000C2607047196889B201EBC00035491B
:109650000C3101EB40013E2A09D95009D20601D153
:10966000401E80B24FF4004242EA802004E05008DD
:10967000D20700D0401C8002086070472849096862
:1096800089B201EBC000274901EB40008088C0F39C
:10969000090070472249096889B201EBC0002149DD
:1096A00001EB40008089C0F3090070471C4A116833
:1096B00089B201EBC0014B001A490B449B8913F49A
:1096C0007C4F01D001207047126892B202EBC000BB
:1096D00001EB400080888005F5D002207047124BD6
:1096E00048F68F7203EB800001290AD0022907D1C6
:1096F000D0F8001C11404CF280021143C0F8001C4D
:109700007047D0F8001C114048F2C002F5E741EA6A
:1097100000207047C1B2000A40EA012070470000F3
:10972000505C00400060004000500040184900209C
:10973000086018494FF43F4008801549091F086028
:109740000020704770B500F07F0514460E4628468D
:10975000FFF742FE0146A2B23046FFF76BFCA1B212
:109760002846FFF750FE002070BD70B500F07F0660
:109770000D463046FFF795FE04463046FFF737FEAC
:10978000014622462846FFF768FC204670BD0000CF
:10979000445C0040A01200202DE9F04788461D4699
:1097A00016468146012102F0B7F9E94F6424394693
:1097B000484602F066FA10B9641EA4B2F7D200223D
:1097C0004146484602F0EFF914B9E249002008602A
:1097D000E14F64243946484602F053FA10B9641E3A
:1097E000A4B2F7D23146484602F0D8F9DA4E6424E2
:1097F000B61C3146484602F044FA10B9641EA4B2C1
:10980000F7D22946484602F0C9F964243146484651
:1098100002F037FA10B9641EA4B2F7D2012148460B
:1098200002F084F9CD4D64242946484602F03CFA02
:1098300010B1641EA4B2F7D20021484602F080F9AC
:109840005020F8F7B9FF0020BDE8F08710B50B46AF
:1098500002463221C248FFF79FFF002010BD10B51D
:1098600037212020FFF7F2FF03212120FFF7EEFF31
:10987000C0212220FFF7EAFF88212320FFF7E6FF1F
:109880007F213020FFF7E2FF02213220FFF7DEFFC9
:1098900003213320FFF7DAFF5F21BDE810402020CD
:1098A000D4E72DE9F05F322688468346AC4F642426
:1098B0004FF0FF3A4FF4003500E0641E2946384669
:1098C00002F0F2F910B1002CF7D194E0002C1AD07C
:1098D0000121384602F020F9A04D64240F3D00E03C
:1098E000641E2946384602F0DFF950B1002C0AD038
:1098F00000223146384602F056F96424DFF85892C7
:1099000003E0002CECD176E0641E4946384602F0B4
:10991000B8F958B1002C6ED05946384602F03EF9DD
:10992000DFF83492642409F1020903E0002CEBD142
:1099300061E0641E4946384602F0A3F930B144B3F1
:109940000121384602F0E8F8642403E0002CF0D14D
:1099500051E0641E2946384602F0A6F948B1C4B168
:1099600001223146384602F01EF9794D64246D1CFF
:1099700003E0002CEDD13EE0641E2946384602F09B
:1099800080F920B12CB1724D64243F3503E0002CE6
:10999000F2D130E0641E2946384602F072F9A0B1D7
:1099A0004CB3384602F0FCF805464FF2FF713846DA
:1099B00002F010F90021384602F0C2F801213846C1
:1099C00002F0B4F86424654E03E0002CE2D112E00A
:1099D000641E3146384602F067F910B1002CF7D109
:1099E00009E044B10021384602F0AAF888F8005096
:1099F0000020BDE8F09F5046FBE72DE9FC5F824662
:109A00000020009004466D46019004F128002919B9
:109A1000C0B2FFF746FF18B14FF0FF30BDE8FC9F22
:109A2000641CE4B2062CF0D3BDF90000001103F071
:109A300006FF0646BDF90200001103F000FF0446D0
:109A4000BDF90400001103F0FAFE0546304603F0AC
:109A5000FAFF02460B4643A0F8F760FF204603F0EA
:109A6000F2FF02460B4642A0F8F758FF284603F0E3
:109A7000EAFF02460B4641A0F8F750FF304603F0DC
:109A800040FF002800DA404203F0D9FE834620461A
:109A900003F037FF002800DA404203F0D0FE04460E
:109AA000284603F02EFF002800DA404203F0C7FEEC
:109AB000814603F0C8FF4FF080480022434605F07E
:109AC00073FE05460E46204603F0BDFF00224346C6
:109AD00005F06AFE07460C46584603F0B4FF002224
:109AE000434605F061FE3A46234603F009FD2A4647
:109AF000334603F005FD06F043FB03F0E7FF0446A1
:109B00000146484603F0FEFF00D2A14621464846E2
:109B100003F0ACFC03F097FF05F088FA012203F094
:109B200077FE194A194B03F004FE0022184B03F08C
:109B30008EFD03F0CBFF0146164803F05FFC10F1E9
:109B4000FF4F00D30020CAF80000002066E70000A5
:109B500001000300A812002082000700100000107E
:109B6000005800406163635F783A25660D0A000083
:109B70006163635F793A25660D0A00006163635F84
:109B80007A3A25660D0A00001F85EB51B81E094080
:109B9000008056400000B44230B5E748A1B01C46F2
:109BA000C168269D491CC160052091FBF0F200FBB5
:109BB0001210002829D14021684603F054FB2046AA
:109BC00003F041FF0022DD4B03F0B3FD02460B46DC
:109BD000DBA1684604F0E6FC042102236A4608463D
:109BE000FDF7D8FE402110A803F03DFB284603F006
:109BF0002AFF02460B46D6A110A804F0D3FC02238C
:109C000010AA06210420FDF7C5FE21B030BD38B5ED
:109C10004FF0FF3200214420FBF7BBFAC64C002274
:109C200004F1380120788870A069C4F84200E06926
:109C3000C4F846001220FCF7F5F801220021142098
:109C4000FCF717F940F2B220FCF73AFF4FF4967098
:109C5000FDF784F90520FDF796F90220FDF7A7F836
:109C6000BF4D00214420FBF776FA28426060F8D00F
:109C70002078401C2070A088400432D54FF48142E7
:109C800000214420FBF785FA6846FCF7B3F9002869
:109C900026D000214C20FBF75EFA00F07F01282936
:109CA00003D80022AF48FCF710F9A3490A224A3131
:109CB000AC4803F0FCFA002812D1AA499E480822B9
:109CC0000A31183003F0F3FA002809D1012060703E
:109CD0000020A060A348418A6180A3A0F8F71EFE7F
:109CE00038BDA8A0F8F71AFEBDE838400021AC4AFC
:109CF0004420FBF74EBAF8B54FF0FF320021442064
:109D0000FBF747FA8C4C002204F15E012078887042
:109D10006088A4F868000C20FCF784F80122002178
:109D20000E20FCF7A6F80220FDF741F88C4D00212B
:109D30004420FBF710FA28426060F8D02078401CDD
:109D40002070A08840047DD54FF48142002144203A
:109D5000FBF71FFA6846FCF74DF9002877D0002181
:109D60004C20FBF7F8F900F07F01282903D80022E6
:109D70007C48FCF7AAF87B4E6F490027B7700A228F
:109D80006A31304603F093FA002860D16A49022212
:109D9000891C06F10B0003F08AFA002857D100F065
:109DA000C8FFC4E9080100F0D9FF7E4AC4E90A01EE
:109DB000801841F10001050A45EA01652846FCF7D3
:109DC000F1FF25F00100010E000244F201028018AB
:109DD00041F10001C4E90C015748D4E9082381305E
:109DE00000F0DFFF5448D4E90A23853000F0D9FFA2
:109DF0005148D4E90C23893000F0D3FF4E49207834
:109E00007731002288701620FCF70CF8012200211F
:109E10001820FCF72EF80120FCF7C9FF002816D106
:109E200000214420FBF797F90006F9D58022002194
:109E30004420FBF7AEF9A7602078401C207056F84C
:109E40000D0F01E004E002E0206170686061F8BD80
:109E5000BDE8F8400021524A4420FBF79AB9F9F7CF
:109E600019F8FAF791FA04464FA0F8F757FDFAF7F8
:109E7000A5F9FAF757F90220FAF749F9FCF743FE7A
:109E80000028FBD00020FBF740FA401C0BD0092033
:109E900084F86F0004F16400FBF708FE38B145A0B8
:109EA000F8F73CFDFEE748A0F8F738FDFEE794F828
:109EB000640009283AD04948FBF764FC44F20104E5
:109EC0002046FBF7A4FF2046FBF7A7FF40F2B22095
:109ED000FCF7F6FD4FF49670FDF740F80520FDF70E
:109EE00052F80320FCF722FFFBF7ECFB05460026A7
:109EF000FBF7E4FB3218104C75412946C4E90625EE
:109F000037A0F8F70BFD4FF4FA7760780A2578B19F
:109F1000FFF7F1FEA068411CA160322800DD6670E9
:109F20002846FAF7F4F8F7F7C6F8EEE73248C3E741
:109F3000FFF76DFE3D46F3E7B012002000005940E8
:109F40002044203A2025332E3266206D2020200028
:109F50002041203A2025332E3166202020000000A9
:109F600000D0272454370020B1EAC7A94944A3BA36
:109F700025303458BCD3C8EBCDF8C2E7B3C9B9A675
:109F80000A000000BCD3C8EBCDF8C2E7B3ACCAB13D
:109F9000BBF2D5DFBDD3CAD5B4EDCEF30A000000C5
:109FA0000090272460015A03B1EAC7A92076312E18
:109FB00030000000434F4E464947204641494C453A
:109FC0004420202020200000494E49542046414989
:109FD0004C454420202020200000000038100020A4
:109FE000B1EAC7A9C5E4D6C3B3C9B9A6202530389C
:109FF00078253038580A00004410002030B5FF485A
:10A00000A1B01C468168269D491C8160052091FBFA
:10A01000F0F200FB1210002829D14021684603F01D
:10A0200022F9204603F00FFD0022F54B03F081FBDF
:10A0300002460B46F3A1684604F0B4FA0421022359
:10A040006A460846FDF7A6FC402110A803F00BF96C
:10A05000284603F0F8FC02460B46EEA110A804F0D7
:10A06000A1FA022310AA06210420FDF793FC21B0D7
:10A0700030BD2DE9F043DFF8AC830C46054685B0D2
:10A08000C068414603F0F2F981462146A86803F012
:10A09000B5F9E549E54C884202D9214603F05CF95F
:10A0A000E349884202DD214603F0A8F9E14903F0C3
:10A0B000ABF90646E048006890F8390090B11422E8
:10A0C000DE49684603F0B6F8009801246F46314631
:10A0D00003F09AF957F8241003F03EF9641C052C9C
:10A0E000F5DB0646D649304603F0C0F94FF07E57FF
:10A0F0000446B84201DD3C4603E0D248844200D920
:10A1000004464FF0FF31304603F0EEF9494603F0C4
:10A1100078F90646214603F077F9CB4903F01CF99C
:10A12000414603F071F921462861084603F06CF9B5
:10A13000394603F066F903F086FC06F021F8044680
:10A140000F46304603F07FFC22463B4603F07FFA81
:10A150000022AB4B03F07BFA03F0B8FC686105B05A
:10A16000BDE8F0832DE9F047924689460646D14581
:10A1700042DA4C4606EBC4005546D0E900708046F2
:10A180002CE06D1EAC4208DA06EBC5013A46D1E977
:10A190000001434603F082FCF3D3AC4208DA06EB3D
:10A1A000C50006EBC402D0E90010C2E90010641C2F
:10A1B000AC4208DA06EBC4013A46D1E90001434655
:10A1C00003F054FCF3D3AC4208DA06EBC40106EB0F
:10A1D000C502D1E90001C2E900016D1EAC42D1DB2C
:10A1E00006EBC401621EC1E9007849463046FFF71C
:10A1F000B9FF04F10109BAE7BDE8F0872DE9F041A4
:10A20000ADF5347D0F468046012A6ED88A48006835
:10A21000B0F84400002868D05B208C4E02FB00F5AB
:10A2200006EBC50460681E280BDB03F02CFB002244
:10A23000874B05F095F903F091FB6060012006F86B
:10A240003500D8F8000003F0FEFB626804EBC202A0
:10A25000C2E90201386803F0F6FB626804EBC2024F
:10A26000C2E93E016068401C606016F835000028B5
:10A270003BD004F10801F022684602F0DBFF04F154
:10A28000F801F0223CA802F0D5FF04F5F471F022A9
:10A2900078A802F0CFFF1D2200216846FFF762FF79
:10A2A000DDE91E01DDE91C2303F02AF94FF0FF343C
:10A2B000224603F0ADFA03F009FCC8F800001D22A5
:10A2C00000213CA8FFF74EFFDDE95A01DDE95823E4
:10A2D00003F016F9224603F09BFA03F0F7FB38600F
:10A2E0001D22002178A8FFF73DFF0DF5347DBDE864
:10A2F000F08170B550F80A4F45682046294600F0B5
:10A3000086FDB8B33D4942684A6582688A654088DF
:10A31000A1F85C0000F022FD4E4A801841F10001D6
:10A32000000A40EA0160FCF73DFD344900224A3151
:10A330001420FBF777FD012200211620FBF799FD81
:10A340000120FCF734FD20B1BDE8704042A0F8F7D1
:10A35000E5BA00214420FAF7FEFE0006F9D54FF4D5
:10A36000814200214420FAF714FFBDE87040052027
:10A37000F9F7CDBE2046294600F0F4FD002805D0AF
:10A3800020462946BDE8704000F07CBA70BD2DE93A
:10A39000F04F97B000270646ADF800704089ADF841
:10A3A000000000F053FD05007DD000F0D7FC134CF9
:10A3B000284AC4E90601801841F10001000A40EA78
:10A3C0000160FCF7EFFC40F29E20FCF779FB4FF4B4
:10A3D0009670FCF7C3FD04F16A01207888706888E4
:10A3E000A4F87500E068C4F877002069C4F87B0021
:10A3F00000221520FBF716FD012233E04013002058
:10A40000000059402044203A2025332E3366206D29
:10A41000202020002041203A2025332E31662020A4
:10A42000200000000000C842000034C30000B44314
:10A4300000003443AF4C0639341000208C0B010867
:10A44000C364AA3C000080BFC3642A3C803900205A
:10A4500000003E4068816D03B7A2CBCDCAA7B0DC37
:10A460000A00000000211720FBF703FD0520FCF780
:10A470008AFD0320FCF79BFC401C14D0DFF890837E
:10A4800000214420FAF767FE10EA080F6060F7D059
:10A490002078401C2070A08840047CD500214FF417
:10A4A0008142442000E077E0FAF773FE14A8FBF73E
:10A4B000A1FD002870D000214C20FAF74CFEC0F31B
:10A4C0000901B1F5007F03D800223046FBF7FDFCFF
:10A4D0000020B0700A22CF49304602F0E8FE002882
:10A4E0005AD100F026FCC4E9080100F037FCC4E9A9
:10A4F0000A0112A906F10A0000F045FC13A906F1B1
:10A500000E0000F040FC10A906F1120000F03BFC28
:10A51000D4F81880A76A266A139812990190401AF5
:10A5200003F0C2F98146B81B059103F0BDF98246DC
:10A530008B4610990198081A03F0B6F90746A6EB66
:10A540000800019103F0B0F900900E4652465B46B8
:10A550004846059902F0D4FF3A46019B02F0D0FF2D
:10A560003346009A02F0CCFF0991DDE900218046D4
:10A570003346384603F06BF806460F4652465B46B4
:10A580004846059903F063F832463B4603F059F814
:10A590004246099B01E09AE090E003F0CAF803F01C
:10A5A00015FA03F08EF99C4A9C4B03F050F84FF0DB
:10A5B00098529B4BC4E90C0103F049F803F086FA6A
:10A5C000E060FCF76CF803F03AF96FF00A0102F072
:10A5D0008BFF944902F018FF934902F047FF0646AB
:10A5E000282106A802F03FFE904F08963946E06801
:10A5F00002F00AFF8E4E09903068B0F9320003F085
:10A600001EF9014606A8FFF734FD0AA82A880BA9FF
:10A610008046FFF7F3FD6888ADF8180060788DF884
:10A620001A00401C6070F9F767FD0790DDE90A0128
:10A6300002F01CFF03F007FA04F030FE00227D4B0D
:10A6400003F005F84FF0C0427B4B03F072F803F0C3
:10A650003DFA0C9000200D903168BDF838204B8EEB
:10A660007BB3002342EAC332ADF83820898E49B368
:10A670005FF0000142EA8131ADF83810ADF83C00DE
:10A68000ADF83A00ADF83E0018224146684602F0A7
:10A69000D1FD06AD95E80F0000F06CF91822414697
:10A6A000684602F0C7FD95E80F00FFF7A7FC0C987D
:10A6B00020613946099802F0D9FEE06017B0BDE884
:10A6C000F08F00E001E00123CCE70121D2E717B0D1
:10A6D0000021BDE8F04F594A4420FAF75ABD08B5A9
:10A6E000F8F7D8FBF9F750FE0446F9F767FDF9F7DC
:10A6F00019FD0220F9F70BFDFCF705FA0028FBD045
:10A700000020FAF702FE401C0ED0032084F87100EE
:10A71000092084F86F0004F16400FBF7C7F938B131
:10A7200047A0F8F7FBF8FEE74AA0F8F7F7F8FEE7CE
:10A7300094F86400092821D04B4800BFFBF722F8A9
:10A7400044F201042046FBF762FB2046FBF765FB61
:10A750000320FCF7EBFA0320FAF788FF43A0F8F791
:10A76000DDF82C4C2A4D7F3C0020FCF70CFC00202F
:10A77000FCF7F4FB0020FCF7ADFB03E03F48DDE70E
:10A78000F6F799FC00214420FAF7E5FC28426060C6
:10A79000F6D0A088400433D54FF4804200214420F5
:10A7A000FAF7F7FC6846FBF725FC18B300214C20AC
:10A7B000FAF7D1FCC0F30906B6F5007F04D831469C
:10A7C00000222F48FBF781FB2D4900200A228870C8
:10A7D00010492B48473902F06AFD38B10D490A2269
:10A7E0002139274802F063FD28B10EE031462448A4
:10A7F000FFF77FFD09E031462148FFF7C8FD04E07F
:10A800000E4A00214420FAF7C4FCF6F754FCABE7EB
:10A8100000D02724BF130020FA48CE3B1835B13DA5
:10A8200019DDB14100003443DB0F49400000C8424C
:10A830003410002000806640FB210940009027244E
:10A84000434F4E464947204641494C45442020202D
:10A8500020200000494E4954204641494C4544209F
:10A86000202020200000000038100020BBF9D5BEB9
:10A87000C5E4D6C3B3C9B9A60A000000441000203D
:10A8800080370020F0B5A9B005460E46A0216846E5
:10A8900002F0E9FC45F65A2280A1684603F082FEE8
:10A8A0000746684602F0FCFC6C4620442B463246C4
:10A8B0007CA103F077FE684602F0F2FCC21B7FA188
:10A8C000A01C03F06FFE7B20E055684602F0E8FC18
:10A8D00020447CA103F066FE684602F0E1FC81B2F0
:10A8E0006846F6F74AFD29B0F0BD70B5AEB02A2231
:10A8F000DDE936568DF814201B228DF81520020C48
:10A9000034998DF81620ADF817001C46084602F061
:10A91000F8FFCDF81900204602F0F3FFCDF81D0036
:10A92000ADF821500020CDF82300CDF82700280CE9
:10A93000ADF82B00ADF82D60300CADF82F002320C2
:10A940008DF832000DA804900F2209A9684602F084
:10A9500071FC0DF1140C9CE80F00F6F772FD044633
:10A96000C1B20DA8F6F714FDE1B20DA8F6F712FD7D
:10A970002EB070BD0FB44FF480712DE9F043C7B015
:10A9800006A802F070FC50480068B0F8460080B19C
:10A99000012809D1182252A9684602F04BFC4EAC9E
:10A9A00094E80F00FFF7A1FF47B0BDE8F0035DF8A2
:10A9B00014FB45F65A2239A106A803F0F3FD05461B
:10A9C00006A802F06DFC06AC204440A103F0EAFDAD
:10A9D00006A802F065FC4F99009120449DF83A3199
:10A9E000BDF838213CA103F0DDFD539802F089FF4A
:10A9F0008146529802F085FF8046509802F081FF10
:10AA00000746519802F07DFF064606A802F048FC72
:10AA100020443B46324638A1CDE9008903F0C2FD0F
:10AA2000559802F06EFF064606A802F039FCBDF903
:10AA30005A11BDF95E31BDF95C218DE80E0020444C
:10AA4000BDF85831324635A103F0ACFD06A802F03E
:10AA500027FC20443AA103F0A5FD06A802F020FC43
:10AA6000421B16A1A01C03F09DFD7B20605506A88B
:10AA700002F016FC204413A103F094FD06A802F096
:10AA80000FFCC1B206A8F6F783FC06A802F008FC8A
:10AA9000C1B206A8F6F77EFC86E700004A532530CF
:10AAA000345800007B224E6577546167223A222594
:10AAB00030386C582530386C58227D002530345899
:10AAC000000000000D0A0000341000207B225457C3
:10AAD00052223A20000000007B22613136223A22C5
:10AAE00025303458222C2252223A25642C2254221A
:10AAF0003A25642C000000002244223A25642C22CE
:10AB000050223A25642C2258636D223A25642C2267
:10AB100059636D223A25642C00000000224F223A2E
:10AB200025642C2256223A25642C2258223A256488
:10AB30002C2259223A25642C225A223A25647D007F
:10AB40007D00000038B50C460021ADF8001041042E
:10AB500002D4A16A491CA162C10302D56168491CE3
:10AB60006160C10402D5A168491CA160810202D5BF
:10AB70002169491C2161810002D5216A491C216299
:10AB8000810404D5410402D42168491C216010F4D9
:10AB9000081F02D06169491C6161410102D5E16869
:10ABA000491CE160C00035D5606B0021401C60632A
:10ABB0006846FBF733FABDF80000C10502D5A16B6A
:10ABC000491CA163010602D5E16B491CE163410602
:10ABD00002D5216C491C2164810602D5616C491C97
:10ABE0006164C10602D5A16C491CA164010702D5AC
:10ABF000E16C491CE164410702D5216D491C2165C6
:10AC0000810702D5616D491C6165C00702D0A06D46
:10AC1000401CA06538BD7249002049780E2909D230
:10AC2000DFE801F008080C1508080F0808071208EB
:10AC30000809802070474FF4C07070474FF460706F
:10AC400070474FF4B06070474FF4F06070474FF4B6
:10AC500078607047624900208979002900D1C820B6
:10AC600070474A780E2A1ED2DFE802F01D09151B34
:10AC7000070D180B1D0F1B1D1D12203813E0403847
:10AC800011E048380FE080380DE0A0F580700AE050
:10AC9000A0F5007007E0A0F5806004E0A0F5C060BA
:10ACA00001E0A0F50060097B0822891C8A4010445D
:10ACB0004FF69A114843000AFCF774B810B50B46DA
:10ACC0000246FFF7C7FF8418FFF7A5FF197B204452
:10ACD00000F5FA70072909D2DFE801F00808080436
:10ACE000040404000822891C8A401044BDE8104076
:10ACF000FCF734B93A4910B50A7B0821921C9140FF
:10AD000001EBD17100EB610200213648FAF741FAFC
:10AD1000BDE81040FAF7A5BD10B500220A60835CBB
:10AD2000D400A3400C68521C23440B60042AF6DBB9
:10AD300010BD7CB5002425466846FBF7A2FC042024
:10AD400069462D0245EA146522020C5C401E14433C
:10AD500040B20028F5DA204629467CBD7CB50024A7
:10AD600025466846FBF7C4FC042069462D0245EAE7
:10AD7000146522020C5C401E144340B20028F5DA30
:10AD8000204629467CBD10B500220A60835CD400B1
:10AD9000A3400C68521C2344D2B20B60042AF5D3A2
:10ADA00010BD10B500214254120A42EA0362491C48
:10ADB0001B0AC9B20429F6D310BD2DE9F04115468E
:10ADC0001E4607460024E2002846314602F01CFADF
:10ADD0003855641CE4B2042CF5D3BDE8F0810000C2
:10ADE000501000201C0002006B4800687230704751
:10ADF000694900200968B1F87210002900D00120CB
:10AE00007047654813210068723002F02CBAF0B523
:10AE1000614A01271368002213F1720302EB420416
:10AE200004EB0214E6187468B56844404D402C43A6
:10AE300007D134882CB102EB420000EB0210184419
:10AE4000F0BD521CBA42E9DB0020F0BD30B55249DA
:10AE500001230A680021723201EB410404EB011462
:10AE600014446588854207D124882CB101EB410048
:10AE700000EB0110104430BD491C9942ECDB00206E
:10AE800030BD4548012201680020723100EB4003CB
:10AE900003EB00130B4400F101001B8823B100B247
:10AEA0009042F3DB0020704780B270472DE9F043F9
:10AEB000164607468C46FFF7AAFF04002FD1DFF89D
:10AEC000D890D9F8000000F17208FFF7DAFF05B258
:10AED000002D24DD012D02DD21E0761CB6B23046C6
:10AEE000FFF7B4FF0028F8D105EB450000EB051192
:10AEF00001EB080424F8135D66806760C4F808C09D
:10AF0000D9F80010B1F85E10A181D9F80010B1F89D
:10AF10006010E181D9F80000B0F86200208220467C
:10AF2000BDE8F08310B5FFF791FF002804D0BDE81D
:10AF30001040132102F097B910BD10B5FFF767FF5D
:10AF4000002804D0BDE81040132102F08CB910BDD8
:10AF5000124A0020D2E90012114300D001207047AC
:10AF60000E487047F0B50D4C0125D4E9002382EA64
:10AF7000000683EA01073E4302D01A4302D003E0F1
:10AF8000002501E0C4E900012846F0BD0348002186
:10AF9000016041607047000034100020D813002089
:10AFA0002849084328490860704770B50F23C478C2
:10AFB00001780122F4B1244C2468457804F4E0645B
:10AFC000C4F5E064240AC4F10406E3408478B54083
:10AFD0001C402C4301F1E021230181F8003400786A
:10AFE00000F01F018A404009800000F1E020C0F815
:10AFF000002170BD01F01F0082404809800000F16F
:10B00000E020C0F8802170BD104A114001430E4875
:10B01000001F016070470C4A121D0029116801D001
:10B02000014300E08143116070474FF0E0210428A4
:10B03000086903D020F004000861704740F0040064
:10B04000FAE700000000FA050CED00E080FFFF1FAA
:10B0500001684FF6FE7211400160002101604160FD
:10B060008160C1606A496A4A0839904203D14868E0
:10B0700040F00F0006E0664A1432904204D148685E
:10B0800040F0F00048607047614A2832904203D196
:10B09000486840F47060F5E75D4A3C32904203D165
:10B0A000486840F47040EDE7594A5032904203D16D
:10B0B000486840F47020E5E7554A6432904203D175
:10B0C000486840F47000DDE7514A7832904203D17D
:10B0D000486840F07060D5E74E4A111F904203D196
:10B0E000086840F00F0006E04A4A1432904204D14A
:10B0F000086840F0F00008607047464A28329042E5
:10B1000003D1086840F47060F5E7424A3C3290424F
:10B1100003D1086840F47040EDE73E4A5032904257
:10B12000EAD1086840F47020E5E730B5036847F6D7
:10B13000F07293430C6A8A682243D1E904452C4398
:10B1400022438C692243CC6922434C6A22438C6A95
:10B1500022431A430260CA6842600A6882604968F2
:10B16000C16030BD0021016041608160C16001614A
:10B1700041618161C1610162416281627047002960
:10B18000016802D041F0010102E04FF6FE72114069
:10B1900001607047002A026801D00A4300E08A4338
:10B1A0000260704741607047406880B27047014656
:10B1B0000020CA0002D5174A083A01E0144A083AAA
:10B1C00012680A4200D001207047C10003D511491E
:10B1D000091F086070470E490839486070470146EA
:10B1E0000020CA0002D50B4A083A01E0084A083A92
:10B1F00012680A4200D001207047C10003D50549FA
:10B20000091F08607047024908394860704700000C
:10B210000800024008040240374900200860091D68
:10B220000860091D0860091D08603349334814315E
:10B230000860704730B530498379026853B30B68B2
:10B2400093430B600A1D13680468A34313600279DB
:10B250000A441368046823431360274A08321368BA
:10B260000468A3431360131D1C680568AC431C608D
:10B270004479102C05D021440A68006802430A6012
:10B2800030BD1168046821431160196800680143EA
:10B29000196030BD0079084401689143016030BDF8
:10B2A0000021016001710C224271817170471249C5
:10B2B00010310A6802430A60704701460E4A0020B6
:10B2C000143212680A4200D0012070470A49143132
:10B2D00008607047084A014600201268064B0A4081
:10B2E00014331B680B4202D0002A00D001207047A3
:10B2F000014914310860704700040140FFFF0F004E
:10B30000FC4A116801F03801014311607047F949A6
:10B310000A6822F008020A600A6802430A6070475D
:10B32000F4490A6822F010020A600A6802430A60BF
:10B330007047F048F0494160F04941607047ED487E
:10B34000ED494160ED4941607047EA48016941F0CB
:10B35000800101617047E748016941F080010161A6
:10B360007047E4490420CA68D20701D00120704721
:10B37000CA68520701D502207047C968C906FBD5C3
:10B380000320704700B50346FFF7EBFF03E000BF63
:10B39000FFF7E7FF5B1E012803D0002B00D105203B
:10B3A00000BD002BF4D1FAE770B505464FF4302606
:10B3B0003046FFF7E7FF042811D1CE4C206940F05A
:10B3C000020020616561206940F040002061304644
:10B3D000FFF7D8FF216941F6FD721140216170BD70
:10B3E00030B54FF430252846FFF7CCFF042810D1A4
:10B3F000C04C206940F004002061206940F040000A
:10B4000020612846FFF7BEFF216941F6FB7211401B
:10B41000216130BD00B50346FFF7A3FF03E000BF85
:10B42000FFF79FFF5B1E012803D0002B00D10520F2
:10B4300000BD002BF4D1FAE730B54FF43025284693
:10B44000FFF7E8FF042810D1AA4C206940F004005F
:10B450002061206940F0400020612846FFF7DAFFB4
:10B46000216941F6FB721140216130BDA1490020E4
:10B47000C969890700D50120704770B5A525FFF778
:10B48000F5FF00B100254FF430263046FFF77AFF74
:10B49000042827D1974C9848A0609848A06020695C
:10B4A00040F020002061206940F0400020613046DB
:10B4B000FFF768FF41F6EF7604280ED1206941F6C8
:10B4C000DF7108402061206940F0100020618C4845
:10B4D00005804FF40050FFF755FF052802D0216981
:10B4E0003140216170BDF8B5064600204FF4005C84
:10B4F00000900D466046FFF745FF042816D17D4CAD
:10B50000206940F00100206135806046FFF73AFF76
:10B5100041F6FE77042806D1B61C280C0096308030
:10B520006046FFF72FFF216939402161F8BDF0B572
:10B5300006464FF400570D463846FFF723FF042810
:10B540000CD16C4C206940F00100206135803846F8
:10B55000FFF718FF2169BA1E11402161F0BDF0B557
:10B5600006464FF400570D463846FFF70BFF0428F8
:10B5700013D1604C6048A0606048A060206940F032
:10B580001000206135803846FFF7FCFE052804D006
:10B59000216941F6EF7211402161F0BD2DE9F041C2
:10B5A000C04300F0FF0CC0F30727C0F30746050EA9
:10B5B0004FF400584046FFF7E5FE042837D14D4CC4
:10B5C0004D49A1604D49A160216941F010012161FF
:10B5D000BCF1FF0F08D04A480830A0F800C0404630
:10B5E000FFF7D0FE04281BD1FF2F07D044480A30B4
:10B5F00007804046FFF7C6FE042811D1FF2E07D072
:10B600003F480C3006804046FFF7BCFE042807D1B7
:10B61000FF2D07D03A480E3005804046FFF7B2FEB6
:10B62000052804D0216941F6EF7211402161BDE87F
:10B63000F08170B505464FF430263046FFF7A2FE84
:10B64000042818D12B4C2C48A0602C48A0602069FD
:10B6500040F020002061206940F040002061304629
:10B66000FFF790FE41F6DF71042805D0052802D0CF
:10B6700022690A40226170BD20690840206120696A
:10B6800040F0100020611E480DB1002100E0A5210E
:10B6900001803046FFF776FE0528ECD0216941F69F
:10B6A000EF721140216170BDF0B5124C074612488F
:10B6B00016460D46A0601148A0604FF4005C60463D
:10B6C000FFF760FE042814D1206940F010002061CB
:10B6D00035430B493D43891C45F0F800088060461E
:10B6E000FFF750FE052804D0216941F6EF721140A2
:10B6F0002161F0BD0020024023016745AB89EFCDF9
:10B7000000F8FF1F1C48C069800870471A48006A8B
:10B710007047194900200968890600D50120704743
:10B72000154A0029116901D0014300E081431161EC
:10B73000704701460020104A012903D0D2680A420E
:10B7400003D17047D169C907FBD0012070470A496E
:10B75000C860704708490420CA68D20701D0012098
:10B760007047CA68520701D502207047C968C906E8
:10B77000FBD503207047000000200240914910B51E
:10B78000884206D10121042000F0FDFB00210420A5
:10B790003BE08D49884206D10121082000F0F3FBEF
:10B7A0000021082031E08949884206D1012110207A
:10B7B00000F0E9FB0021102027E08549884206D1EE
:10B7C0000121202000F0DFFB002120201DE0814925
:10B7D000884206D10121402000F0D5FB0021402005
:10B7E00013E07D49884206D10121802000F0CBFB87
:10B7F0000021802009E0794988420AD1841501217D
:10B80000204600F0C0FB00212046BDE8104000F0BB
:10B81000BABB10BD10B50121084600F0B4FB0021F1
:10B82000BDE81040012000F0AEBBF0B5CA7800259D
:10B8300002F00F03D20601D58A7813430A784FF03D
:10B840000F0E12F0FF0F4FF001021DD0D0F8004094
:10B850000F8802FA05F63740B74211D14FEA850C3E
:10B860000EFA0CF724EA070703FA0CF43C43CF78EE
:10B87000282F02D0482F02D002E0466100E0066186
:10B880006D1C082DE4D304600C88FF2C1ED944687D
:10B890005FF0000606F1080702FA07F50F882F404F
:10B8A000AF420FD14FEA860C0EFA0CF7BC4303FAF5
:10B8B0000CF73C43CF78282F00D14561CF78482F33
:10B8C00000D10561761C082EE4D34460F0BD4FF62C
:10B8D000FF710180022181700421C170704702460E
:10B8E000002092680A4200D001207047806880B230
:10B8F000704702460020D2680A4200D001207047FB
:10B90000C06880B2704701617047416170470AB1F9
:10B910000161704741617047C160704741F48032F6
:10B920008261816182618169806970472C4B10B5A9
:10B930001A684FF68074224042EA001008431860EB
:10B9400010BD2849C8617047F0B5254C002801DAC0
:10B95000E36900E06368420D120185B2C0F301574C
:10B960009540C0F30346032F05D0C2020AD5032237
:10B97000B240934307E023F07062636823F0706382
:10B98000636002E0AB4343F0706201B12A430028D8
:10B9900001DAE261F0BD6260F0BD10B58A0721F006
:10B9A00003040F49130F21440F228C689A409443DB
:10B9B0008C608A68984002438A6010BD0949C1F8CA
:10B9C000DC00704700080140000C014000100140FD
:10B9D0000014014000180140001C014000200140FB
:10B9E0000000014000002042C64910B588424FF0D7
:10B9F000010101D14C0501E04FF48004204600F024
:10BA0000CBFA2046BDE81040002100F0C5BA70B561
:10BA10000446808886B00D4620F03F06684600F058
:10BA200057FAB9490298B0FBF1F189B20E43A680EA
:10BA3000228822F001022280B44B2A689A421CD844
:10BA40005200B0FBF2F080B2042800D20420491C5E
:10BA50002184A083208840F00100208021884FF6B7
:10BA6000F5300140A8886A89104308432080A889DE
:10BA700029890843208106B070BDEB88A3F53F46B5
:10BA8000FF3E0BD002EBC20303EB0212B0FBF2F05D
:10BA900080B240F48040020506D007E002EB42028B
:10BAA000B0FBF2F080B2F6E740F001004FF496727E
:10BAB00051434FF47A72B1FBF2F140F40040C6E713
:10BAC00041F288310160002181804BF6FF72C28013
:10BAD000018141814FF480418181704700290188B3
:10BAE00002D041F0010101E021F001010180704725
:10BAF0000029818802D041F4006101E021F4006155
:10BB0000818070470029818802D041F4805101E092
:10BB100021F48051818070470029018802D041F4CE
:10BB2000807101E021F48071018070470029018853
:10BB300002D041F4007101E021F4007101807047EE
:10BB40000029018802D041F4806101E021F4806184
:10BB500001807047828901F0FE0122F0FE0211434C
:10BB6000818170470029818902D041F0010101E003
:10BB700021F00101818170470029018802D041F044
:10BB8000400101E021F0400101807047002A8288D5
:10BB900001D00A4300E08A438280704701827047E7
:10BBA000008AC0B2704712B141F0010101E001F01A
:10BBB000FE010182704708B508440090008808BD66
:10BBC0000029018802D041F4004101E0C1F30E01D7
:10BBD00001807047B1F5006F018803D021F4006146
:10BBE0000180704741F40061FAE7B1F5005F018818
:10BBF00003D021F400510180704741F40051FAE76D
:10BC00000029018802D041F4805101E021F48051E3
:10BC100001807047B1F5006F018803D021F4006105
:10BC20000180704741F40061FAE70029018802D0E1
:10BC300041F0200101E021F0200101807047008BDC
:10BC4000000A70470029018802D041F0100101E08C
:10BC500021F01001018070470029018803D021F0F4
:10BC600080010180704741F08001FAE7B1F5804F13
:10BC7000818B02D021F4804101E041F48041818335
:10BC8000704702460020938A128B43EA024323F056
:10BC90007F42914300D101207047818A008B41EAA5
:10BCA000004121F07F4070470CB502460020009211
:10BCB0000A0F21F07F41019202D0009A143202E073
:10BCC000009A090C1832009212680A4200D0012032
:10BCD0000CBDC9438182704710B5034600209A8885
:10BCE0004FF4E06404EA11449B8A224021F07F4132
:10BCF0000B4202D0002A00D0012010BDC94381822E
:10BD0000704700000054004040420F00A086010030
:10BD10000D49086070470C49486070470A498860BF
:10BD2000704709494AF6AA200860704706494CF650
:10BD3000CC4008607047044A01460020D2680A429D
:10BD400000D001207047000000300040A448016886
:10BD500041F0010101604168A24A1140416001685F
:10BD6000A14A11400160016821F48021016041680D
:10BD700021F4FE0141604FF41F0181607047984932
:10BD80000A6822F480320A600A6822F480220A607B
:10BD9000B0F5803F07D0B0F5802F03D1086840F49C
:10BDA000A02008607047086840F48030F9E7024638
:10BDB000002053098A49012B0AD0022B0AD0496A74
:10BDC00002F01F02012393400B4200D00120704774
:10BDD0000968F5E7096AF3E718B500204FF4A06495
:10BDE00000903120FFF7E3FF0099491C0091A14228
:10BDF00001D00028F5D03120FFF7D9FF002800D06E
:10BE0000012018BD76490A6822F0F80242EAC00013
:10BE100008607047754908607047714A5368084365
:10BE200023F47C13184350607047704908667047CC
:10BE30006B4A516821F00301014351607047684823
:10BE4000406800F00C007047654A516821F0F0012D
:10BE5000014351607047624A516821F4E061014337
:10BE6000516070475E494A6822F4605242EAC0005D
:10BE7000486070475A4A0029517A01D0014300E0D6
:10BE80008143517270475949C1F8D8007047544AEC
:10BE9000516821F4404101435160704750490022EC
:10BEA00081F8202081F82020012802D0042802D126
:10BEB000052081F8200070474D49086070474849C7
:10BEC0000A6A02430A627047494944390860704768
:10BED00030B543494A6812F00C03464A03D0042B9C
:10BEE00001D0082B21D002604A680F23424C03EA9C
:10BEF0001212A35C0268DA4042604B68072505EA2B
:10BF00001323E35C22FA03F383604B6805EAD3232F
:10BF1000E35CDA40C2604968032303EA9131231FDE
:10BF2000595CB2FBF1F1016130BD4A684B6802F423
:10BF300070124FF0020413F4803F04EB924202D0DF
:10BF40004B689B0301D52D4B00E02A4B5A43CAE7AF
:10BF5000234A0029516901D0014300E08143516126
:10BF600070471F4A0029916901D0014300E08143D5
:10BF7000916170471A4A0029D16901D0014300E05C
:10BF80008143D1617047164A0029D16801D001432D
:10BF900000E08143D1607047114A0029116901D046
:10BFA000014300E081431161704711494039086045
:10BFB00070470E49C86470470949C87170470848FE
:10BFC000416A41F0807141627047054A0146002094
:10BFD00092680A4200D00120704701498872704778
:10BFE000001002400000FFF8FFFFF6FE0000424292
:10BFF0008004424200127A00E413002000093D0050
:10C00000994910B588420AD1841401212046FFF7CE
:10C01000BAFF2046BDE810400021FFF7B4BF9349A6
:10C02000884202D10121041404E0914988420AD1D6
:10C030000121C4132046FFF7AFFF2046BDE81040A2
:10C040000021FFF7A9BF10BD30B502884C8802F46B
:10C0500041530A88CD8822438C882C4322430C8983
:10C0600022434C8922438C892243CC8922431A43A0
:10C070000280828B22F400628283098A018230BDB1
:10C08000F0B505460C4602200021AA8B85B001269A
:10C090004FF240031A40AA832884AF8BA268022A79
:10C0A00027D0A08800B102266846FFF711FFE1887B
:10C0B0000098B1F5007F2DD07101B0FBF1F000BF09
:10C0C00000EB8000A1684000B0FBF1F0401D80B2A1
:10C0D0000A21B0FBF1F000F00101401A4FF6FF72A7
:10C0E000C0F34F0002EA0121821EFE2A01D3022082
:10C0F0000021E288084302432A8420886188A289BB
:10C100000843A18811430843384340F40060A883E2
:10C1100005B0F0BD000AD3E7002101804180818095
:10C12000C180018141818181C181072101827047E4
:10C130000021018041808180C18002228260818152
:10C1400070470029018802D041F0400101E021F050
:10C150004001018070470029818B02D041F4806149
:10C1600001E021F4806181837047090901238B403C
:10C17000002A828899B201D00A4300E08A43828073
:10C180007047002A828801D00A4300E08A438280F7
:10C1900070478181704780897047A1F57E42018890
:10C1A000FF3A02D041F4807101E021F480710180F6
:10C1B00070470029818802D041F0040101E021F09C
:10C1C000040181807047028822F4006202800288A4
:10C1D0000A4302807047018841F480510180704712
:10C1E0000029018802D041F4005101E021F40051FE
:10C1F00001807047012901D0008B7047808A704709
:10C20000008A7047B1F5804F018803D021F4804146
:10C210000180704741F48041FAE70246002012890C
:10C220000A4200D001207047C9430181704710B510
:10C2300001F00F040122034602FA04F40020090968
:10C240008A4091B29A88A4B20A401989214202D048
:10C25000002A00D0012010BD01F00F020121914001
:10C26000C9430181704700000030014000380040A0
:10C27000003C0040F94910B5884202D10121C414A4
:10C2800086E0B0F1804F09D0F54988420DD10121F7
:10C290000220FFF781FE0021022064E00121084610
:10C2A000FFF77AFE002101205DE0EE49884206D1C9
:10C2B00001210420FFF770FE0021042053E0EA4929
:10C2C000884206D101210820FFF766FE00210820E0
:10C2D00049E0E649884206D101211020FFF75CFEC3
:10C2E000002110203FE0E249884206D101212020B0
:10C2F000FFF752FE0021202035E0DE49884202D1BE
:10C300000121441444E0DC49884202D10121CC04DB
:10C310003EE0DA49884202D101210C0538E0D849D3
:10C32000884202D101214C0532E0D649884206D12B
:10C3300001214020FFF730FE0021402013E0D249C8
:10C34000884206D101218020FFF726FE00218020AF
:10C3500009E0CE4988420AD1841501212046FFF721
:10C360001BFE00212046BDE81040FFF715BEC8495E
:10C37000884202D101210C040AE0C649884202D158
:10C3800001214C0404E0C44988420AD101218C04F3
:10C390002046FFF7F8FD2046BDE810400021FFF7DA
:10C3A000F2BD10BD30B50288AC4BB24C98420DD0F6
:10C3B000A0420BD0B0F1804F08D0A94DA84205D0C3
:10C3C000A84DA84202D0A84DA84203D122F0700582
:10C3D0004A882A43A54DA84206D0A54DA84203D0BD
:10C3E00022F44075CA882A4302808A8882850A8896
:10C3F000028598420AD0A04208D0A54A904205D0B2
:10C40000A44A904202D0A44A904201D1097A0186FE
:10C410000121818230BD30B5028C22F001020284FC
:10C42000028C8388048B22F0020224F073050C88AE
:10C430002C430D8915434A882A43884DA8420BD0C6
:10C440008C4DA84208D0924DA84205D0914DA842EB
:10C4500002D0914DA8420DD122F008054A8923F45B
:10C4600040732A4322F004058A882A438D891D439C
:10C47000CB892B4383800483C9888186028430BDA5
:10C4800070B5028C22F010020284028C8488038B27
:10C490000D8823F4E6464FF6FF7303EA052535437E
:10C4A0000E8922F0200203EA061616434A8803EAA0
:10C4B00002123243694EB04202D06E4EB04215D1E4
:10C4C00022F080064A8924F4406403EA02123243CF
:10C4D00022F040068A8803EA021232438E8903EA78
:10C4E00086062643CC8903EA84043443848005838A
:10C4F000C9880187028470BD70B5028C22F48072F5
:10C500000284028C8488838B0D8823F073031D437F
:10C5100022F400730E894FF6FF7202EA06261E43CC
:10C520004B8802EA032333434C4EB04202D0514EB3
:10C53000B04215D123F400664B8924F4405402EA3A
:10C540000323334323F480668B8802EA03233343B7
:10C550008E8902EA06162643CC8902EA0414344383
:10C5600084808583C9888187038470BD70B5028CFF
:10C5700022F480520284048C8288838B0D8823F4F9
:10C58000E6464FF6FF7303EA0525354324F40056CB
:10C590000C8903EA043434434E8803EA0636264302
:10C5A0002E4CA04202D0334CA04205D122F480444C
:10C5B0008A8903EA8212224382808583C988A0F88F
:10C5C0004010068470BD828B22F440628283828B8D
:10C5D0004FF6FF7303EA01210A4382837047828B7F
:10C5E00022F00C028283828B0A4382837047028B83
:10C5F00022F440620283028B4FF6FF7303EA0121AB
:10C600000A4302837047F0B5048C24F010040484BC
:10C61000078B048C4FF6FF7527F4734705EA033345
:10C620003B4305EA02221A430C4B05EA01169842E5
:10C630000ED0104B98420BD0B0F1804F08D0084B71
:10C64000984205D0074B984202D0074B984225D11B
:10C6500024F02001314341F0100124E0002C01407E
:10C660000004004000080040000C004000100040A2
:10C670000014004000340140004C014000500140D3
:10C680000054014000180040001C00400020004001
:10C6900000400140004401400048014024F0A00354
:10C6A0000B4343F0100102830184F0BD028B22F0A2
:10C6B0000C020283028B0A430283704770B5048C1C
:10C6C00024F001040484058B048C4FF6FF7606EAFF
:10C6D0000313134325F0F305F94A2B4390420ED080
:10C6E000F84A90420BD0B0F1804F08D0F64A904201
:10C6F00005D0F64A904202D0F54A904202D124F089
:10C70000020201E024F00A020A4342F0010103831D
:10C71000018470BD2DE9F05F0D4604460888E84F9E
:10C72000DFF8A0C3DFF8A0834988AA882B894FF0DF
:10C73000804960B3042832D04FF6FF7E082836D0F7
:10C74000208C9B4620F480502084A38B268C70463E
:10C7500000EA022223F473431A4300EA0B30104329
:10C760000EEA013EBC420BD0644509D04C4507D0CF
:10C77000444505D0D54A944202D0D54B9C4245D180
:10C7800026F4005141EA0E0141F4805143E0204675
:10C79000FFF794FFE9882046BDE8F05F86E7204672
:10C7A000FFF731FFE9882046BDE8F05F1FE7208CE6
:10C7B00020F480702084B4F81CA0208C0EEA0313AF
:10C7C00013432AF0F30A0EEA012B43EA0A03BC42A0
:10C7D0000BD0644509D04C4507D0444505D0BB4A31
:10C7E000944202D0BA4A944204D120F4007040EA44
:10C7F0000B0002E020F42060084340F48070A38323
:10C800002084E9882046BDE8F05FE8E626F402428D
:10C810000A4342F48051A08320462184E988BDE880
:10C82000F05FD0E62DE9F0410C4600264988074626
:10C83000012501B90226A288012A00D102252088FB
:10C8400023890028384610D0FFF7DDFEE1883846FE
:10C85000FFF7CDFE23892A4631463846FFF72EFFE3
:10C86000E1883846BDE8F04120E7FFF727FFE1887F
:10C870003846FFF71BFF23892A4631463846FFF723
:10C88000C2FEE1883846BDE8F041B0E610B50A883E
:10C890004B88CC881A438B8823431A430B891A434D
:10C8A0004B8989891A430A43A0F8442010BD4FF6EA
:10C8B000FF71818000210180C18041800172704739
:10C8C0000021018041808180C1800181418181817D
:10C8D000C181704700210180418001228280C18096
:10C8E000018170470021018041808180C1800181E8
:10C8F0004181818170470029018802D041F0010106
:10C9000001E021F0010101807047002930F8441F47
:10C9100002D041F4004101E0C1F30E0101807047F3
:10C92000002A828901D00A4300E08A43828170474D
:10C93000818270471143A0F848107047002A82890D
:10C9400001D00A4300E08A4382817047018921F0C7
:10C95000070101817047028922F070020A430281B7
:10C96000704700B50346FFF7F6FF188940F007004F
:10C97000188100BD70B516460D46602904464FF07B
:10C98000010231460AD0FFF799FE29462046FFF7FB
:10C99000E2FF208940F00700208170BDFFF733FEE1
:10C9A000F3E730B504894FF6FF7505EA0323134317
:10C9B000E4B20B432343038130BD10B50446FFF7B7
:10C9C000F0FF208940F07700208110BD10B50446AB
:10C9D000FFF7E7FF208940F48040208110BD0185EA
:10C9E00082827047028822F070020A4302807047F8
:10C9F00070B50589048B068C25F007050D434FF6AD
:10CA0000FC410C4040F201110C434FF6FF7101EA6A
:10CA1000031126F02206114331430581048301846A
:10CA200070BD028B22F070020A4302837047028BB2
:10CA30004FF6FF7322F4E04203EA01211143018320
:10CA40007047828B22F070020A4382837047828B88
:10CA50004FF6FF7322F4E04203EA01211143818380
:10CA600070470029018802D041F0800101E021F0E7
:10CA70008001018070470029818802D041F00401C3
:10CA800001E021F00401818070470029818802D0F3
:10CA900041F0080101E021F0080181807047002980
:10CAA000818802D041F0010101E021F00101818083
:10CAB0007047028B22F008020A430283704700008D
:10CAC000002C0140003401400004004000080040F8
:10CAD000000C0040028B4FF6FF7322F4006203EA61
:10CAE000012111430183E9E7828B22F008020A4306
:10CAF0008283E3E7828B4FF6FF7322F4006203EA3E
:10CB0000012111438183D9E7028B22F004020A43F9
:10CB10000283D3E7028B4FF6FF7322F4806203EAAD
:10CB2000012111430183C9E7828B22F004020A43E9
:10CB30008283C3E7828B4FF6FF7322F4806203EA9D
:10CB4000012111438183B9E7028B22F080020A435D
:10CB50000283B3E7028B4FF6FF73C2F30E0203EAC0
:10CB6000012111430183A9E7828B22F080020A434D
:10CB70008283A3E7828B4FF6FF73C2F30E0203EAB0
:10CB800001211143818399E7028C22F002020A43BA
:10CB9000028493E7028C22F008020A4302848DE7A4
:10CBA000028C4FF6FF7322F0200203EA01111143B9
:10CBB000018483E7028C4FF6FF7322F0800203EAC0
:10CBC00001111143018479E7028C4FF6FF7322F4BF
:10CBD000007203EA0121114301846FE7028C4FF6D2
:10CBE000FF7322F4006203EA01211143018465E727
:10CBF000028C4FF6FF7322F4005203EA0131114315
:10CC000001845BE710B50123048C8B409C430484B2
:10CC1000038C8A401343038410BD10B50423048C95
:10CC20008B409C430484038C8A401343038410BDCF
:10CC300030B50124058C00F118038C40A543058410
:10CC400089B108290FD0091FC1F34E0018440168AB
:10CC500021F4E041016001684FF6FF7303EA02220C
:10CC60001143016030BD03EB5100016821F07001F8
:10CC700001600168F4E70029018802D041F0020157
:10CC800001E021F00201018018E70029018802D0AB
:10CC900041F0040101E021F0040101800EE70029C8
:10CCA000818802D041F0800101E021F08001818083
:10CCB00004E7028822F00802028002880A43028008
:10CCC000FCE6828822F07002828082880A43828099
:10CCD000F4E6028922F00702028102890A430281F6
:10CCE000ECE6028922F08002028102890A43028175
:10CCF000E4E68184E2E68185E0E68186DEE601877E
:10CD0000DCE68187DAE6A0F84010D7E6028822F454
:10CD10004072028002880A430280CFE6808ECDE610
:10CD2000008FCBE6808FC9E6B0F84000C6E6808C65
:10CD3000C4E6008DC2E602460020128A0A4200D0F4
:10CD40000120BBE6C9430182B8E602460020138AEF
:10CD500092890B4202EA010202D0002A00D001208F
:10CD6000ACE6C9430182A9E6C44910B588420AD19C
:10CD700001218C032046FFF706F92046BDE810404C
:10CD80000021FFF700B9BE49884202D101214C04BD
:10CD900010E0BC49884202D101218C040AE0BA4962
:10CDA000884202D10121CC0404E0B84988420AD16A
:10CDB00001210C052046FFF7EFF82046BDE81040A2
:10CDC0000021FFF7E9B810BD30B50446008A85B0F0
:10CDD0000D464CF6FF710840E98801432182A18984
:10CDE0004EF6F3100140A8882A8910436A890A4345
:10CDF0001043A081A08A4FF6FF410840A989014352
:10CE0000A1826846FFF764F89C48844201D10398E8
:10CE100000E00298A189090400EBC00101EB0010B9
:10CE2000296801D5490000E08900B0FBF1F06422D7
:10CE3000B0FBF2F109010B096FF018056B4300EB31
:10CE40008300A3891D044FF0320306D503EBC00015
:10CE5000B0FBF2F000F0070005E003EB0010B0FBC0
:10CE6000F2F000F00F000843208105B030BD4FF410
:10CE70001651016000218180C18001810C22428114
:10CE80008181704710B5038A4FF2FF0213400A8870
:10CE90004C8822438C88C9880C4322431A4302825F
:10CEA00010BD0021018041808180C1807047002930
:10CEB000818902D041F4005101E021F400518181C7
:10CEC000704710B5C1F3421301F01F040121A140C6
:10CED000012B07D0022B07D01430002A026805D09E
:10CEE0000A4304E00C30F8E71030F6E78A430260AA
:10CEF00010BD002A828A01D00A4300E08A43828260
:10CF00007047028A22F00F020282028A0A430282DA
:10CF10007047828922F40062828182890A43828179
:10CF200070470029818902D041F0020101E021F01F
:10CF3000020181817047028A22F020020282028A65
:10CF40000A43028270470029018A02D041F48041DD
:10CF500001E021F4804101827047C1F30801818022
:10CF600070478088C0F308007047818941F0010153
:10CF700081817047028BD2B20283028B42EA012187
:10CF800001837047028B02F47F420283028B0A43C3
:10CF9000028370470029818A02D041F0200101E01C
:10CFA00021F02001818270470029818A02D041F05E
:10CFB000100101E021F01001818270470029818A6F
:10CFC00002D041F0080101E021F0080181827047A0
:10CFD0000029818902D041F4004101E0C1F30E0132
:10CFE000818170470029818A02D041F4006101E00B
:10CFF00021F4006181827047828A22F004028282D9
:10D00000828A0A43828270470029818A02D041F0D5
:10D01000020101E021F002018182704702460020F6
:10D0200012880A4200D001207047C943018070472E
:10D0300030B501F01F0201240025C1F3421304FAA8
:10D0400002F2012B0FD0022B0FD0838A4FEA11215D
:10D050000088134204FA01F400EA040001D000B190
:10D060000125284630BD8389F0E7038AEEE70A0AE6
:10D0700001219140C9430180704700000038014000
:10D080000044004000480040004C00400050004078
:10D090000648804706480047FEE7FEE7FEE7FEE752
:10D0A000FEE7FEE7FEE7FEE7FEE7FEE755D10008F4
:10D0B000ED0000080CB500214B4801910091026879
:10D0C00042F4803202604FF4A063026802F400323E
:10D0D0000092019A521C0192009A12B9019A9A4246
:10D0E000F3D10268920333D5012100913F490A68C8
:10D0F00042F010020A600A6822F007020A600A6819
:10D1000042F002020A604168416041684160416842
:10D1100041F480614160416821F47C1141604168C3
:10D1200041F4E8114160016841F0807101600168DB
:10D130008901FCD5416821F003014160416841F05B
:10D14000020141604168C1F381010229FAD10CBD9D
:10D1500000910CBD244810B5016841F00101016047
:10D160004168234A114041600168224A1140016030
:10D17000016821F480210160416821F4FE014160D1
:10D180004FF41F018160FFF795FF1B494FF00060CE
:10D19000086010BD144910B54868184A10F00C0317
:10D1A000174803D0042B01D0082B0AD0026049682D
:10D1B000134AC1F30311121D515C0268CA40026098
:10D1C00010BD4A684B6802F470124FF0020413F469
:10D1D000803F04EB924202D04B689B0301D5094B80
:10D1E00000E0064B5A43E1E70010024000200240F5
:10D1F0000000FFF8FFFFF6FE08ED00E000127A00E5
:10D20000F413002000093D00202A04DB203A21FA13
:10D2100002F00021704721FA02F3D040C2F120024F
:10D220009140084319467047A0F16101192900D8BF
:10D230002038704740EA01039B0703D009E008C982
:10D24000121F08C0042AFAD203E011F8013B00F8CB
:10D25000013B521EF9D27047D2B201E000F8012B17
:10D26000491EFBD270470022F6E710B513460A4666
:10D2700004461946FFF7F0FF204610BD30B50546BD
:10D280002A460B4612F8010B13F8014B08B1A042D5
:10D29000F8D01CB1002802D06D1CF1E7284630BD43
:10D2A000421C10F8011B0029FBD1801A704730B5D1
:10D2B00004460020034600E05B1C934203D2E05C7E
:10D2C000CD5C401BF8D030BD2DE9F05F93460F4692
:10D2D00080460446002601F0A7F9D0F80090824667
:10D2E00014F8015B2DB100F07FFC0068405DC007C1
:10D2F000F6D12B2D02D02D2D1AD0641E0021CAF894
:10D3000000105A463946204600F07BFC014627B102
:10D310003868A04201D1C7F80080DAF8000002287E
:10D3200009D0CAF80090700505D54842BDE8F09FC5
:10D3300046F48066E2E70846F8E700F037BD70B5CE
:10D34000064601F071F9046805460A2200213046BC
:10D3500000F0F4FC2C6070BDF0B480EA0102D40F40
:10D360004200B2EB410F02D20246084611464A0083
:10D3700042D0C30DDDB2C1F3C752AD1A202D35DA4C
:10D38000C1F3160141F4000204B15242C5F1200676
:10D3900002FA06F12A411044B3EBD05F23D0C4B1A6
:10D3A000012DA0EBC35009DCF0BC4FF0004202EAB3
:10D3B000C352DBB200F5000000F03FBD400000F1B9
:10D3C000807000EBC350A0F1807040EAD17049003A
:10D3D00009E0490841EAC071A0EBC35000F5000024
:10D3E000400800EBC350F0BC00F01EBD61420122BA
:10D3F00002EB4101001BF6E7F0BC704781F00041F1
:10D40000AAE780F00040A7E780EA010210B502F029
:10D410000043400022D04A001FD0010E01EB1261F0
:10D42000C0F35600C2F3560240F4000042F400027A
:10D43000A0FB022000047F39140400D0401C50EAF5
:10D44000124001D44000491EC2B20C0604EBD010B9
:10D45000401C4008802A02D003E0002010BD20F0CC
:10D460000100002900DA0020184310BD30B480EA22
:10D47000010202F0004530F0004221F0004013D0DC
:10D4800090B1C30DD40DC2F31601C0F31600E41A17
:10D4900041F4000140F400027D34914201D3641C48
:10D4A00000E04900002C02DA30BC002070474FF445
:10D4B00000000023914201D3891A034340084FEA38
:10D4C0004101F7D151B1914202D14FF0004105E045
:10D4D00002D24FF0010101E06FF0010103EBC450F3
:10D4E000284430BC00F0A0BC420005D0C0F3C752B5
:10D4F0005242914201DC0020704700EBC15070475E
:10D500002DE9FE4F804681EA0300C00F0C460090D3
:10D5100021F0004123F00045B8EB0200A94105D2FB
:10D520004046214690461C460B46024623F00040EA
:10D53000104347D0270DC7F30A00C3F30A510290E6
:10D54000401A019040286BDAC3F3130040F4801BAB
:10D550000098924620B10023D2EB030A63EB0B0B39
:10D5600001985946C0F14002504600F01CFB0646A7
:10D570000D4650465946019A00F024FB10EB080076
:10D580006141002487EA115284EAE7731A4340D0CC
:10D59000009A62B3019A012A4FEA075215DC001B78
:10D5A00061EB02014FF0004202EA0752CDE900426E
:10D5B000001C41F5801132462B4600F07BFC03B085
:10D5C000BDE8F08F40462146F9E7001B61EB020100
:10D5D000001C41F5801300185B412018A2F50017CC
:10D5E00047EB030140EAD570B6196D4111E06D08B3
:10D5F0004FEA360645EAC0754FEA0752001B61EB59
:10D600000201001C41F5801149084FEA3000001961
:10D61000514132462B4603B0BDE8F04F00F03BBC11
:10D620000098012240000023D0EB020263EBE0737C
:10D63000009821464FEAE074B8EB000061EB04016A
:10D64000E9E783F000435BE781F0004158E72DE90B
:10D65000FE4F81EA030404F0004421F000410094ED
:10D660004FF0000B23F0004350EA01045ED052EA71
:10D6700003045BD0C3F30A54C1F30A552C44A4F24B
:10D68000F3340194A0FB0254C1F3130141F480115F
:10D69000C3F3130343F4801301FB024400FB034E66
:10D6A000840A970A44EA815447EA8357A4FB07682F
:10D6B00002958D0A05FB07854FEA932C04FB0C5459
:10D6C0002705029D4FEA065847EA1637B5EB0805CD
:10D6D0006EEB070C870E920E47EA811742EA83121F
:10D6E000A7FB0201B6EB0B0164EB00042B0D43EA30
:10D6F0000C335E1844EB1C50DA465146E7FB02013E
:10D70000C5F313044FEA0B3343EA14534FEA0432D0
:10D71000019C43EA0603A4F10C040294009CCDE9A9
:10D7200000B400F0C7FB03B0BDE8F08F0020014655
:10D73000F9E72DE9F04D81EA030404F0004B21F0F4
:10D74000004514464FF0000A23F0004150EA05025C
:10D7500020D054EA01021DD0C5F30A570246C5F392
:10D760001303C1F31300C1F30A5640F4801543F4C8
:10D770008013A7EB0608101BD64608F2FD3873EBA2
:10D78000050002D308F1010801E092185B41B8F1ED
:10D79000000F03DA00200146BDE8F08D00204FF4B1
:10D7A0008011064684460EE0171B73EB050705D370
:10D7B000121B63EB050306434CEA010C49084FEAD0
:10D7C000300092185B4150EA0107EDD152EA0300A4
:10D7D00012D082EA040083EA0501084305D0101B39
:10D7E000AB4106D20122002306E000224FF00043A5
:10D7F00002E06FF0010253101AEB06004CEB0851E7
:10D8000010EB0A0041EB0B01BDE8F04D00F043BB0B
:10D8100070B521F0004303430CD0C1F30A55002436
:10D82000D5EB040564EB0403D617AD1AB34102DB54
:10D830000020014670BD201841EB025170BDC10FA0
:10D8400080EAE0700844CA079623002100F0F5BA88
:10D8500096230022114600F0F0BAF0B4CA17CB0F9D
:10D8600050405140C61841F100054FEAC37231469D
:10D8700028004FF0960303D0B623F0BC00F0DDBAC9
:10D8800030460021F9E70EB5C10F80EAE070084488
:10D89000CA07002140F233438DE80E000A460B46CA
:10D8A00000F008FB03B000BD0EB540F23341029119
:10D8B0000021CDE900110A460B4600F0FBFA03B047
:10D8C00000BD3EB5CA17CB0F002450405140C018D0
:10D8D0006141DA0740F233430094CDE90123224647
:10D8E000234600F0E7FA03B030BD0EB540F23342F4
:10D8F00002920022CDE90022134600F0DBFA03B0C9
:10D9000000BD00F0004220F00040C10DC0F3160041
:10D9100040F400007F2901DA00207047962903DCDB
:10D92000C1F19601C84001E096398840002AF4D040
:10D930004042704720F00040C10DC0F3160040F493
:10D9400000007F2901DA00207047962903DCC1F12D
:10D950009601C840704796398840704770B5C1F34A
:10D960000A5201F000450024C1F3130140F2FF33D5
:10D9700041F480119A4201DA002070BD40F2334335
:10D980009A42A2F2334203DC5242FFF73DFC00E030
:10D9900090402C43F1D0404270BDC1F30A5210B503
:10D9A000C1F3130140F2FF3341F480119A4201DACE
:10D9B000002010BD40F233439A42A2F2334203DC0E
:10D9C0005242FFF721FC10BD904010BD70B5C1F36D
:10D9D0000A5201F000450024C1F3130140F2FF3365
:10D9E00041F480119A4202DA0020014670BD40F2F3
:10D9F00033439A42A2F2334203DC5242FFF704FC63
:10DA000001E000F0D0F82C43F0D00023D0EB03006D
:10DA100063EB010170BDC1F30A52C1F3130140F27F
:10DA2000FF3341F480119A4202DA00200146704728
:10DA300040F233439A42A2F2334202DC5242FFF7F1
:10DA4000E3BB00F0B0B800F0004230F000400AD074
:10DA5000C10D01F56071C0F3160042EA0151C20820
:10DA600040071143704700200146704730B5041E3F
:10DA700071F1000404DB4FF00044404264EB01010B
:10DA8000141E73F1000405DB1C464FF000435242A4
:10DA900063EB04038B4208BF824230BD30B5041EE5
:10DAA00071F1000404DB4FF00044404264EB0101DB
:10DAB000141E73F1000405DB1C464FF00043524274
:10DAC00063EB0403994208BF904230BD01F000436C
:10DAD00030B421F0004150EA010206D00A0DA2F54F
:10DAE0006072C1F31301002A02DC30BC00207047D1
:10DAF000440F44EAC104C100E01830BC00EBC2503E
:10DB000000F092B9002801DBC0F10040002901DBE0
:10DB1000C1F100418842704730B50B4601460020F4
:10DB20002022012409E021FA02F59D4205D303FADF
:10DB300002F5491B04FA02F52844151EA2F1010260
:10DB4000F1DC30BD2DE9F05F0546002092469B4692
:10DB500088460646814640241BE028464146474603
:10DB60002246FFF751FB53465A46C01A914110D343
:10DB700011461846224600F016F82D1A67EB0108E8
:10DB80004F4622460120002100F00DF817EB000956
:10DB90004E41201EA4F10104DFDC484631462A46EE
:10DBA0004346BDE8F09F202A04DB203A00FA02F148
:10DBB000002070479140C2F1200320FA03F319437B
:10DBC00090407047202A06DBCB17203A41FA02F03A
:10DBD00043EAE07306E041FA02F3D040C2F12002CA
:10DBE000914008431946704700487047DC0D010812
:10DBF00010B50446FFF7F8FF0068005D00F0010073
:10DC000010BD2DE9F05F82460078002715468B464F
:10DC10000AF10104B946302801D09DB113E014F88F
:10DC2000010B0127782803D0582801D045B10AE01C
:10DC30000DB1102D07D10027102514F8010B02E0BB
:10DC4000082500E00A250026B0460EE005FB080086
:10DC500005FB06F1012701EB10461FFA80F8B6F527
:10DC6000803F00D3B94614F8010B294600F016FA9C
:10DC70000028EBDABBF1000F05D00FB1641E00E005
:10DC80005446CBF80040B9F1000F06D000F0CCFCB0
:10DC900002210160C81EBDE8F09F48EA0640FAE78D
:10DCA0000FB4002300B589B00CA900910B996FF057
:10DCB0000042CB601E4B06931E4B07930423CDE915
:10DCC00001321D4A089202466B46002000F088FA95
:10DCD00009B05DF814FB70B586B006464FF0FF3012
:10DCE0000091CDE90101002015460C460490324612
:10DCF000694604A8FFF7D4FF02460498211825B10D
:10DD000008B1084600E020462860049800280DD09D
:10DD1000002A02DD0098884208D0081B0094CDE953
:10DD200001043246694604A8FFF7BAFF06B070BD89
:10DD300019E4000837E40008F1DB00082DE9F0479A
:10DD400091460F4680460446002614F8015B2DB12B
:10DD5000FFF74AFF0068405DC007F6D12B2D02D0C7
:10DD60002D2D18D0641E4A4639462046FFF749FF3C
:10DD700027B13968A14201D1C7F8008071054FF081
:10DD800002040BD54042002803DD00F04DFC046086
:10DD9000A007BDE8F08746F48066E4E70028F8DADB
:10DDA00000F042FC04606FF00040F2E72DE9F05F04
:10DDB00093460F4680460446002600F035FCD0F816
:10DDC0000090824614F8015B2DB1FFF70DFF00684B
:10DDD000405DC007F6D12B2D02D02D2D1FD0641E23
:10DDE0000021CAF800105A463946204600F034FB9C
:10DDF000024627B13868A04201D1C7F80080DAF89E
:10DE0000000002280ED0CAF8009070050AD5002044
:10DE10000346D2EB000063EB0101BDE8F09F46F43E
:10DE20008066DDE71046F8E70029A8BF7047401C70
:10DE3000490008BF20F00100704710B4B0FA80FC20
:10DE400000FA0CF050EA010404BF10BC704749B15D
:10DE5000CCF1200421FA04F411FA0CF118BF0121CD
:10DE600021430843A3EB0C01CB1D4FEA00614FEAAD
:10DE7000102042BF002010BC704700EBC35010447C
:10DE80000029A4BF10BC7047401C490008BF20F007
:10DE9000010010BC704710B5141E73F1000408DABD
:10DEA000401C41F1000192185B411A4301D120F05E
:10DEB000010010BD2DE9F04D92469B4611B1B1FA1B
:10DEC00081F202E0B0FA80F220329046FFF76BFE5A
:10DED00004460F4640EA0A0041EA0B0153465A46FF
:10DEE000084313D0114653EA010019D0C8F140028B
:10DEF0005046FFF789F905460E46504659464246B8
:10DF0000FFF751FE084305D0012004E020463946C2
:10DF1000BDE8F08D0020054346EAE0762C43374308
:10DF20000A986305E40AA0EB08000022FD0A44EA0F
:10DF300047540A3002D500200146E9E701051019CF
:10DF40006941DDE9084500196941BDE8F04DA2E7E6
:10DF50002DE9F04D00231A461B1A8A4103DB0020ED
:10DF60000146BDE8F08DC1F30A52C1F3130141F43B
:10DF700080154FF0000BD10702D100186D41521EE1
:10DF80000027044640F2FF11384601EB620A3E4684
:10DF90008046024600204FF48011FFF735F9C21980
:10DFA0007141BB1846EB0100B4EB030C75EB000CA0
:10DFB00004D3E41A65EB000517460E46241908F150
:10DFC00001006D4180463428E3DDF91946EB060077
:10DFD000091BA84103D24FF0FF32134601E0002293
:10DFE00013461BEB070046EB0A51BDE8F04DFFF767
:10DFF00052BF2DE9FE4FC3F30A5701F0004500243C
:10E00000C1F30A56C3F31303C1F3130143F480139E
:10E0100012EB020AA64641F48011009543EB030C73
:10E02000A7F1010B16E0B0EB0A0061EB0C01071E33
:10E0300071F1000707DA4FF00008D0EB080085F017
:10E04000004568EB0101171A73EB0107EBD3761E4D
:10E05000001849415E45F6DA50EA010209D0CDE9DF
:10E0600000E5002213460296FFF724FF03B0BDE847
:10E07000F08F20460099F9E7064C074D06E0E0686E
:10E0800040F0010394E8070098471034AC42F6D3FF
:10E09000F2F730F8C4120108E41201083A2800D25D
:10E0A000303820F02002412A01D3A2F13700884203
:10E0B00001D34FF0FF3070472DE9FF4F087883B050
:10E0C0009946FF2805D0491C2D2804D000240020A3
:10E0D00008E000200BE00124F9E700EB800003EBEF
:10E0E0004000491C0B78FF2BF7D104B140420023BC
:10E0F0000293147819461D462D2C01D02B2C04D1E7
:10E10000521C2D2C13D000240294AA461478FF2C04
:10E110000FD00A25A3FB057801FB05814FF0000C09
:10E1200003FB0C11521CE3194AEB0101EEE7012439
:10E13000EAE7814453EA010002D019F5C87F06DA04
:10E1400003980021C0E9001107B0BDE8F08F002559
:10E15000AE4E2F46DFF8B8821846FFF7C6FBCDE972
:10E160000001B9F1000002DAC9F1000400E0044640
:10E170000023A74A1AEB030B42EB045A12E0E00714
:10E1800007D02A46334638464146FFF760FA07462D
:10E1900088462A46334610461946FFF758FA054680
:10E1A0000E466410002CEAD1DDE90001B9F1000F40
:10E1B0005A46534606DAFFF7BCFA3A464346FFF79B
:10E1C000B8FA05E0FFF743FA3A464346FFF73FFA4D
:10E1D000029A0AB181F00041039AC2E90001B3E753
:10E1E0002DE9FF4F1F468DB0D7E901464FF0FF38AC
:10E1F0002E2045464FF000090B90B9696D1C0E9812
:10E200008847396A824688470028F6D1BAF1FF3F2D
:10E210000AD024F4D064002E11DDBAF12B0F08D0FF
:10E22000BAF12D0F0BD102E0404611B08DE744F456
:10E230008064B9696D1C0E9888478246761E6946CF
:10E24000600501D52D2000E02B208DF8000001F1A4
:10E25000010B0DF1200809E0B9696D1C0E98884783
:10E2600082460F9844F40074761E0560002E02DD8D
:10E27000BAF1300FF0D00B998A453ED144F08004BA
:10E2800006E00F99681CA9F1010944F400740860C4
:10E29000B9696D1C761E0E98884782463028F0D0EA
:10E2A0002BE00B998A4505D1200603D444F0800465
:10E2B000761E18E0504600F01DFB08B30DF1130167
:10E2C000761E44F400748B4508D2AAF130000BF896
:10E2D000010B200607D5A9F1010003E0200602D4B6
:10E2E00009F101008146A00502D50F99681C08605C
:10E2F000B9696D1C0E9888478246002ED1DC53E028
:10E30000002E51DDBAF1650F02D0BAF1450F4BD1A5
:10E31000A00549D5B9696D1C24F44074761E0E9889
:10E3200088478246002E0CDD2B2804D0BAF12D0F31
:10E3300007D144F48074B9696D1C0E9888478246F1
:10E34000761EE00501D52D2100E02B2108F8011BE8
:10E35000CDF82C8021E00DF12901761E44F40074E3
:10E3600088450CD2AAF1300010F0FF0088F80000B8
:10E3700002D10B99884509D908F1010806E0E005AA
:10E3800001D5244801E042F20F708146B9696D1C45
:10E390000E98884782460F980560002E04DD50468F
:10E3A00000F0A8FA0028D6D1F9690E988847FF2016
:10E3B0008BF8000088F800000020069007904B467C
:10E3C0006A4608A906A8FFF777FEA00502D46FF0F9
:10E3D00001002AE714F0240F0AD0E00714D1DDE988
:10E3E00006123868031D3B600068C0E900120BE0AC
:10E3F000DDE90601FFF76AFB0146E00704D1386852
:10E40000021D3A600068016028460EE700001440D3
:10E410000000F03FF1D8FFFF426842B1016811F8F7
:10E42000013B23B1521EC0E900121846704701217A
:10E43000C160881E704742685AB1C368016843B919
:10E4400083688B4205D0491E521CC0E9001200208F
:10E4500070474FF0FF3070472DE9F74F4FF000093C
:10E46000009C1546CA4614F8010B302801D0ADB106
:10E4700015E014F8010B4FF00109782803D0582853
:10E4800001D04DB10BE00DB1102D08D14FF00009B6
:10E49000102514F8010B02E0082500E00A250027EA
:10E4A0003E46B8464FEAE57B16E0A5FB07230BFB8B
:10E4B000073105FB080005FB0616010C571846F14D
:10E4C00000061FFA80F8381E4FF0010976F58030FB
:10E4D00000D3CA4614F8010B2946FFF7DFFD0028D8
:10E4E000E3DA019838B1B9F1000F01D0641E00E001
:10E4F000009C01980460BAF1000F08D000F094F875
:10E5000002210160C81E014603B0BDE8F08F31044E
:10E5100041EA174148EA0740F6E770B58C1810F851
:10E52000015B15F0070301D110F8013B2A1106D158
:10E5300010F8012B03E010F8016B01F8016B5B1E72
:10E54000F9D12B0705D40023521E0DD401F8013B4D
:10E55000FAE710F8013BCB1A921C03E013F8015BB9
:10E5600001F8015B521EF9D5A142D8D3002070BD3D
:10E570000FB47CB50C0009AD01D0611E00E0002194
:10E58000CDE90001064B6A462946089800F0BAF921
:10E59000002C02D0009A002111707CBC5DF814FBA5
:10E5A0000BF000080FB4084B10B504A902AA039899
:10E5B00000F0A8F9044602A9002000F031FD204631
:10E5C00010BC5DF814FB000021F000087CB50C00C5
:10E5D0001D461646014601D0601E00E00020CDE930
:10E5E0000010064B6A462946304600F08BF9002C95
:10E5F00002D0009A002111707CBD00000BF00008D1
:10E60000490050EAC12018BF04204A0D18BF40F04D
:10E61000010040F2FF72B2EB515F08BF40F0020010
:10E62000012808BF052070470048704708140020E3
:10E630002DE9F0414F1E00EBC7010446D1E900016E
:10E6400015461E4637F006020DD02A463346FEF721
:10E65000FEFF7F1E04EBC703D3E90023FEF750FF44
:10E6600037F00602F1D1022F25D0042F13D0062F48
:10E6700018BFBDE8F0812A463346FEF7E8FFD4E92B
:10E680000A23FEF73DFF2A463346FEF7E0FFD4E9B2
:10E690000823FEF735FF2A463346FEF7D8FFD4E9B4
:10E6A0000623FEF72DFF2A463346FEF7D0FFD4E9B6
:10E6B0000423FEF725FF2A463346FEF7C8FFD4E9B8
:10E6C0000223FEF71DFF2A463346FEF7C0FFD4E9BA
:10E6D0000023BDE8F041FEF713BF000000221346FF
:10E6E00010460149FFF725B80000F03F0122FFF76F
:10E6F0008FB8FEF705BF0022134610461146FFF7FC
:10E7000018B840F2013200204FF0E041FFF780B826
:10E71000024A00201107FFF77BB8000001FDFFFF50
:10E7200000214FF07E50FEF7A1BE0121FEF7DCBEB6
:10E7300000210846FEF79ABE0148006870470000B5
:10E740000814002002E008C8121F08C1002AFAD1EC
:10E7500070477047002001E001C1121F002AFBD161
:10E76000704700000149086070470000081400204D
:10E770002DE9FF5F82B00021DDE90430020DDDF8F4
:10E7800040B0034318D044F61050A2F2FF32424387
:10E790001514119801281FD0A5EB0B00401C5FEA4F
:10E7A000000A4FF000064E4FDFF83891B046504651
:10E7B00015D5CAF1000413E0119801244AA30128D9
:10E7C00001D16FEA0B010298119AC0E90031C0E94A
:10E7D000024206B0BDE8F09FCBF10000DFE704463F
:10E7E0000021404A491842EB0450CDE9001012E0E4
:10E7F000E00707D032463B4640464946FEF727FF32
:10E800008046894632463B4610461946FEF71FFFB2
:10E8100006460F466410002CEAD1DDE90401DDE96B
:10E820000023BAF1000F06DAFEF711FF42464B460D
:10E83000FEF70DFF05E0FEF77CFF42464B46FEF774
:10E8400078FF04460E460022284BFFF727F903D82D
:10E850004FF0FF30014607E00022254B20463146AD
:10E86000FEF74EFEFFF7D7F8102409E0002C0ADB74
:10E870000A220023FFF766F9039B30321A55641E03
:10E8800050EA0102F2D1641C039AC4F1110314444A
:10E89000119A012A03D0012208430DD10AE008434E
:10E8A00004D000204FF0110B119072E7A3EB0B0581
:10E8B0006D1E0DE05B4504DD4FF0000205F1010522
:10E8C00004E003DA4FF00002A5F10105002AECD0C4
:10E8D00002981199C0E90231C0E9004579E70000CA
:10E8E000000014400000F03F300000000000F04342
:10E8F0000000E03F30380A2801D201207047002094
:10E90000704700002DE9FF4F95B09A4688460646AD
:10E910000025EEE1252877D100242746F94A012178
:10E92000039400E0044316F8013F203B01FA03F092
:10E930001042F7D130782A2811D06FF02F033078A9
:10E94000A0F13002092A16D8039A44F0020402EB1F
:10E95000820203EB42021044761C0390EFE758F862
:10E96000042B0392002A03DA504244F4005403902B
:10E9700044F00204761C30782E2816D116F8010FC8
:10E9800044F004042A280DD06FF02F023078A0F153
:10E990003003092B09D807EB870302EB4303C718A1
:10E9A000761CF3E758F8047B761C30786C280FD07F
:10E9B00006DC4C2817D068280DD06A2814D104E052
:10E9C000742810D07A280FD10DE044F400140AE026
:10E9D00044F4801401E044F440147278824202D17D
:10E9E00004F58014761C761C307866280BD013DC76
:10E9F000582877D009DC002875D04528F6D046285D
:10EA0000F4D047281AD193E118E0632835D0642860
:10EA100079D0652812D18BE1702873D008DC672883
:10EA2000F1D069286FD06E280DD06F2806D1ACE0E8
:10EA300073282CD0752874D0782853D05246179953
:10EA400090476D1C54E1C4F30250022809D00328FA
:10EA50000DD0D8F8001004280DD00D6008F104087E
:10EA600046E1D8F80010EA17C1E90052F6E7D8F8F5
:10EA700000100D80F2E70D70F0E718F8041B8DF818
:10EA8000001000208DF80100EB46012003E058F84B
:10EA900004BB4FF0FF3061074FF0000102D40DE0DE
:10EAA00009F101018946B9420FDA8145F8DB1BF80B
:10EAB00009100029F4D108E009F1010189468142D9
:10EAC000FADB1BF809100029F6D103985346A0EB96
:10EAD000090721463846179A00F080FA284400EBCF
:10EAE000090507E044E008E10DE01BF8010B524680
:10EAF00017999047B9F10109F7D253462146384694
:10EB0000179AF2E039E00A21C4F302524FF0000BE9
:10EB10000091022A06D058F8040BC117032A09D025
:10EB20000AE023E008F1070020F00702F2E8020102
:10EB3000904605E000B2C117042A01D140B2C117C6
:10EB4000002906DA0A460021404261EB02012D222B
:10EB500002E0220504D52B228DF80420012203E0D7
:10EB6000E20701D02022F7E7914657E00A2100E0B2
:10EB700010214FF0000B00910BE010214FF0000B23
:10EB800044F004040827009103E008204FF0000B34
:10EB90000090C4F30252022A05D058F8040B002159
:10EBA000032A08D008E008F1070020F00702F2E885
:10EBB0000201904603E080B2042A00D1C0B24FF0B7
:10EBC000000922072AD53278702A07D0DDF800C064
:10EBD0008CF0100C5CEA0B0C05D00EE040228DF896
:10EBE0000420012208E050EA010306D030238DF80A
:10EBF00004308DF8052002229146009B83F0080323
:10EC000053EA0B030AD150EA010201D1620705D58C
:10EC100030228DF804204FF001097F1E3278582AE7
:10EC200004D039A20C920CAA02920BE03BA2F9E7A5
:10EC30005B46009AFEF786FF0C9B9B5C029A521E75
:10EC40000292137050EA0102F2D1029804A9081A44
:10EC500000F1200B600702D524F4803400E0012786
:10EC60005F4502DDA7EB0B0000E0002000EB0B018D
:10EC7000009003984944401A0390E00306D4534699
:10EC80002146179A039800F0A9F90544002706E0E9
:10EC900001A85246C05D179990476D1C7F1C4F45D7
:10ECA000F6DBE0030CD553462146179A039800F093
:10ECB00095F9054404E030205246179990476D1CA1
:10ECC0000099481E00900029F5DC08E0029802999E
:10ECD00052460078491C0291179990476D1CBBF170
:10ECE0000001ABF1010BF1DC5BE100F065F90544DB
:10ECF000761C307800287FF40DAE19B02846BDE8A8
:10ED0000F08F0000092801003031323334353637B6
:10ED10003839616263646566000000003031323367
:10ED20003435363738394142434445460000000007
:10ED3000600700D4062708F1070020F00700F0E87C
:10ED40000223804603F0004C5FEA0C0001D097A03C
:10ED500009E0200501D596A005E0E00701D095A0C7
:10ED600001E0AFF24C001390307823F000436528A7
:10ED70000CD006DC452809D046281DD047287FD175
:10ED80003BE0662818D067287AD136E00021112FA1
:10ED900001DB112000E0781CCDE9000104A90CA8DA
:10EDA000FFF7E6FCDDE90D010C9A4FF0000B07F1CF
:10EDB0000109109200914EE04FF000400097CDE91C
:10EDC000011004A90CA8FFF7D3FCDDE90D020C9B90
:10EDD0000F994FF0000B91461093009211B9791CD6
:10EDE00000EB0109B7EB090003D4C0F1FF3B07F1C9
:10EDF0000109A9EB0700019042E0012F00DA012789
:10EE00000021112F01DD112000E03846CDE900017D
:10EE100004A90CA8FFF7ACFCDDE90D010C9A0091E8
:10EE20004FF0000BB946109221070FD4009A4A45C3
:10EE300003DA914601E0A9F10109B9F1010F05DDFD
:10EE4000109AA9F10101515C3029F4D0B84202DADC
:10EE500010F1040F03DA0121CDE9011010E00028C0
:10EE600003DC8344A9EB000102E0411C494500DDBD
:10EE70008946A0EB0B00401C01904FF0004002902F
:10EE8000200705D40198484502DB4FF0FF30019080
:10EE900000208DF84B0002980DF14B07B0F1004FA8
:10EEA00025D002200C902B200D90029800280CDA1F
:10EEB000404202902D200D9007E00A210298FEF7B3
:10EEC0002BFE3031029007F8011D0C99481E0C9062
:10EED0000029F2DC02980028EFD1791E0D98087005
:10EEE000307800F0200040F0450007F8020D11A82E
:10EEF000C01BC01D02901398007800B1012000EBE8
:10EF00000901019801EBE071029801440398401A4D
:10EF1000401E0390E00306D453462146179A0398F7
:10EF200000F05CF805441398007818B15246179920
:10EF300090476D1CE00323D553462146179A03984A
:10EF400000F04CF805441BE0BBF1000F07DB009814
:10EF5000584504DD1098179910F80B0001E0179937
:10EF600030205246904701980BF1010B401E05F1ED
:10EF70000105019004D12E205246179990476D1C2F
:10EF8000B9F10001A9F10109DEDC05E017F8010B78
:10EF90005246179990476D1C0299481E029000290D
:10EFA000F4DC53462146179A03989EE62D00000094
:10EFB0002B000000200000002DE9F0410446002550
:10EFC0001E461746880404D405E039462020B04781
:10EFD0006D1C641EF9D52846BDE8F0812DE9F0418D
:10EFE000044600251E469046C80301D5302700E0A0
:10EFF0002027880404D505E041463846B0476D1CFB
:10F00000641EF9D52846BDE8F0814A68002A06D07A
:10F010000A68531C0B6010704868401E48607047B7
:10F020000A68531C0B601070704700002DE9F04D0A
:10F030008D4F21F0004A86B005460C46BA452ADBC2
:10F04000AAEB070028430AD08848824501DC1AD180
:10F05000CDB106B02846BDE8F04DFFF747BB844A66
:10F06000844B2846FEF7F3FA07460E46824A834B46
:10F0700028462146FEF7EBFA06B03A463346BDE88D
:10F08000F04DFEF73DBA0120FFF76CFB06B0BDE87E
:10F09000F04DFFF730BB7A48824542DABAF1795F2A
:10F0A0000BDA2846FFF7ACFA042808BFFFF730FB5D
:10F0B000284606B02146BDE8F08D2A460B4610468C
:10F0C000FEF7C5FA834602466E480E460B460621F9
:10F0D0007844FFF7ADFA5A463346FEF7B8FA804651
:10F0E00069488A465A46334604217844FFF7A0FA15
:10F0F0005A463346FEF7ABFA00223B46FEF700FACB
:10F1000002460B4640465146FEF713FB2A4623466D
:10F11000FEF79DFA06B02A462346BDE8F04DFEF7FD
:10F12000EFB9284624F0004100223D463B46FEF759
:10F130008BFA4FF0FF32FEF76BFB06460246534850
:10F140000F460B4606217844FFF772FA32463B46DB
:10F15000FEF77DFACDE900014D4832463B460421D9
:10F160007844FFF765FA32463B46FEF770FA002214
:10F170002B46FEF7C5F9834602913046394600F02A
:10F18000FFFF804643480D46504517DCDDE900018E
:10F190005A46029BFEF7CDFA42462B46FEF757FA37
:10F1A00042462B46FEF7ACF90122FEF731FB304A0E
:10F1B000304BFEF746FA304A304B4CE04FF0000A35
:10F1C00052460B464046FEF79BF9CDE903105246E6
:10F1D0002B4610461946FEF73AFA32463B46FEF7F2
:10F1E00033FADDE90332FEF7A4FA06460F46DDE9FD
:10F1F00000015A46029BFEF79CFA834600910122C9
:10F2000030463946FEF704FB194A1A4BFEF71CFA42
:10F2100006460F46012240462946FEF7F9FA5A46AD
:10F22000009BFEF714FA32463B46FEF70AFA064602
:10F230000F46012250462946FEF7EAFA0E4DDFF846
:10F2400058802A464346FEF7FFF932463B46FEF712
:10F25000FBF92A464346FEF7F7F9002CD8BF81F0A8
:10F26000004106B0BDE8F08D0000F03F0000F07FE7
:10F27000075C143326A6913C182D4454FB21F93F1A
:10F280000000E03FCC1A0000E21A0000561A00000D
:10F290006C1A00003333EF3FFB21E93F2DE9F84FB3
:10F2A00004460D4621F0004000917349814211DC73
:10F2B0007249884201DC06D12CB120462946BDE8BE
:10F2C000F84FFFF713BA6E48002DCCBF6D496E4959
:10F2D000BDE8F88F6D49814211DD6D498142D8BF8B
:10F2E0004FF0FF366DDD20462946FFF789F90428E7
:10F2F00008BFFFF70DFA20462946BDE8F88F65499B
:10F30000654F25F00045814233DD6449814219DDB6
:10F31000002632464FF0804320462946FEF7F0F89B
:10F3200080468A46012220462946FEF771FA0022CD
:10F330003B46FEF786F942465346FEF7FAF9044685
:10F340000D463EE001260022BA463B4620462946AD
:10F35000FEF7D6F880460F4600225346204629463F
:10F36000FEF76FF942463B46FEF7E3F904460D46C9
:10F3700027E04B4981421BDDDFF828A1022600224D
:10F38000534620462946FEF762F900223B46FEF727
:10F39000B7F880460F460022534620462946FEF71E
:10F3A00050F942463B46FEF7C4F904460D4608E0D4
:10F3B000032622462B4600203B49FEF7BAF90446B5
:10F3C0000D4622462B4610461946FEF740F98B465D
:10F3D000824602460B46FEF73AF907460246334894
:10F3E00088460B4606217844FFF722F952465B46D1
:10F3F000FEF72DF982462E488B463A4643460521B4
:10F400007844FFF715F93A464346FEF720F90246DD
:10F410000B46002E504659460CDAFEF771F822468C
:10F420002B46FEF714F901B022462B46BDE8F04FFB
:10F43000FEF70AB9FEF764F822462B46FEF707F9F5
:10F440001C4A7A4402EBC603D3E90023FEF7F9F81D
:10F4500022462B46FEF7F5F8174A7A4402EBC6031C
:10F46000D3E90023FEF7F0F8009A002AB8BF81F034
:10F470000041BDE8F88F0000000010440000F07F5C
:10F48000182D4454FB21F93FFB21F9BF0000DC3F5C
:10F490000000203E0000F33F0000F03F0000E63F88
:10F4A000008003400000F83F0000F0BF6E1800002D
:10F4B0002C180000CA1700009217000030B583B066
:10F4C0000446FFF739F905460020CDE90000024661
:10F4D00021466846FEF7FFFB2846FFF743F9DDE9C2
:10F4E000000103B030BD00002DE9F041C0F3C75169
:10F4F000A1F17F050446172DA8BFBDE8F0814FF0AC
:10F500007F471549002D0EDAFDF726FFB7EB400FB8
:10F510001ED300281CDD002CC8BF4FF07E54B8BF9E
:10F520004FF0004414E00D4A22FA05F6344208BFB9
:10F53000BDE8F081FDF710FFB7EB400F08D30028BE
:10F5400006DD002C03DD4FF40000E8400444B44322
:10F550002046BDE8F0810000CAF24971FFFF7F003C
:10F5600070B514461D460E46002814BF0121002127
:10F57000314321F00041C1F17F6101F1E041C90F48
:10F5800016D1002C14BF01210021294321F0004194
:10F59000C1F17F6101F1E041C90F09D11449B1EB1B
:10F5A000460F08BF00281CD0690008BF002C18D0E7
:10F5B0003146FEF71EFD024640F2FF7030EA115060
:10F5C0000DD0F017B0EBE17F09D0084665F31E00BF
:10F5D00084460B4620466146FEF736F80246104642
:10F5E00070BD0120FFF7BEF8BDE87040FFF783B89B
:10F5F0000000E0FF2DE9F0410026A0F50001B1F187
:10F60000FE4F7DD200F500226FF07E0101EBE2514A
:10F61000C2F3025477184FF07E52A0EBC15602EBB2
:10F62000045557EA040047D029463046FDF794FEBA
:10F63000804629463046FDF7E1FE4146FDF716FFBC
:10F6400005460146FDF7E0FE80464A49FDF7DCFE2F
:10F650004949FDF781FE064641462846FDF7D4FE9E
:10F660003146FDF7D1FE06463846FEF7E8F8074674
:10F670004249FDF7C9FE4249794451F82410FDF78B
:10F680006BFE3146FDF768FE06463E492846FDF70B
:10F69000BBFE3146FDF760FE054638463A49FDF7A8
:10F6A000B3FE3A49794451F82410FDF755FE294636
:10F6B000BDE8F041FDF750BE4FF07E513046FDF7FA
:10F6C0009DFE05463249FDF79FFE3249FDF744FE97
:10F6D0002946FDF799FE3049FDF73EFE2946FDF724
:10F6E00093FE2E49FDF738FE044629460846FDF7ED
:10F6F0008BFE2146FDF788FE04462949284600E096
:10F700000EE0FDF781FE2146FDF726FE0446254961
:10F710002846FDF779FE2146BDE8F041FDF71CBE05
:10F720004FF07F42B2EB400F03D2BDE8F041FEF74D
:10F73000FCBFB0F1FF4F08BFBDE8F081B0F1004F52
:10F7400006D90120FFF70EF8BDE8F041FEF7F0BF43
:10F7500030F0004105D06FF016061721FDF7C4FE0A
:10F7600050E70220FEF7FEFFFEF7DAFF80F00040D0
:10F77000BDE8F081DE02323E3B3D943EFC849A3689
:10F780002C160000D95B5E3F00209A3EE015000079
:10F79000924FA93D7279DEBD2D3E143ED85B5EBE10
:10F7A000157B4B3C0000D83E2DE9F04D1D460C4624
:10F7B00098B0174621F0004123F00043002814BF01
:10F7C0004FF0010C4FF0000C0CEB440CFE4A0CEB1C
:10F7D00002064FEA620C66452BD33E0018BF012695
:10F7E00006EB45061644F94A964222D3F84A53EAF4
:10F7F000070C02D0944205D148B918B00020114638
:10F80000BDE8F08D002808BF4FF0000C01D04FF08C
:10F81000010C0CEB440212F5001F0AD8002F14BF94
:10F820004FF0010C4FF0000C0CEB450212F5001FDD
:10F8300007D918B03A462B462146BDE8F04DFEF7F1
:10F8400058BF0022DFF88CA3002CB8BF534526DA3E
:10F85000DFF884C36345A8BF022220DADFF870C353
:10F860009C451CDCDFF874C30CEB235CBCF1140F6B
:10F8700008DDCCF1340627FA06FC0CFA06F6BE4287
:10F880000DD108E05FB9CCF1140623FA06FC0CFA9E
:10F8900006F69E4203D10CF00102C2F1020251EAC7
:10F8A000000C19D1002D17DA002C18BF022A01D044
:10F8B000012A07D00220FEF755FF18B0BDE8F04D31
:10F8C000FEF70CBF0220FEF74DFFFEF707FF18B052
:10F8D00081F00041BDE8F08DB7F1000C6CD15345CB
:10F8E00025D104F1804212F5801201BF00280020CA
:10F8F000B74918B008BFBDE8F08DB548884207DCAD
:10F90000002DA1BF6046294618B0BDE8F08D07E084
:10F91000281E05DA80F0004118B06046BDE8F08D81
:10F92000AF497944D1E9000118B0BDE8F08DDFF8A6
:10F93000A0C2634525D1002D1FDA19B1514512D15E
:10F94000D8B909E0002840F0EC82A24A214618B05C
:10F9500062F31E01BDE8F08D0020214618B060F36F
:10F960001E01BDE8F08D08DA18B02346BDE8F04D61
:10F97000024600206146FDF7DCBE18B02146BDE816
:10F98000F08D514518DAB5F1804F0DD0A5F1005C2E
:10F99000BCF1FF5C10D1B4F1000C0DDB18B0614676
:10F9A000BDE8F04D00F0ECBB234618B00246BDE8C0
:10F9B000F04D1946FDF74BBE060024F0004C3BD13C
:10F9C000D9B1514533D1002C06DD002DA1BF002057
:10F9D000514618B0BDE8F08D002C01DD002D1BDB79
:10F9E000002C13DA002D11DB012A4FF0000014BFA8
:10F9F00078497C4918B0BDE8F08D022A18BF002C68
:10FA00000AD0012A08D1002C06DA0AE0002CB8BF7F
:10FA1000002D11DA012A04D0002018B00146BDE8FB
:10FA2000F08D18B000204FF00041BDE8F08DA1F13D
:10FA30004050B0F17F601AD0012000EBE47050EA32
:10FA4000020421D0624C521E4FF0000B104304BF41
:10FA50004FF0000B644C654883427CDD644A654886
:10FA600093421FDD884217DB002D25DB37E0002C99
:10FA700000DA4AB1022A0CBF01204FF0FF3018B063
:10FA8000BDE8F04DFDF7FFBE0120FEF76BFE18B09C
:10FA9000BDE8F04DFEF72FBE4D4A8A4202DC002D34
:10FAA0000ADC1CE0814202DA002D18DA04E0484B3F
:10FAB000994220DD002D12DD0220FEF753FEFEF7F5
:10FAC00020FE05460E460022534658462146FDF7C5
:10FAD000BEFD18B066F31E012846BDE8F08D022079
:10FAE000FEF740FEFEF714FE0A46214618B062F308
:10FAF0001E01BDE8F08D002230466146FDF7A1FDF4
:10FB000080460E466FF00102FDF782FE4FF055323F
:10FB1000394BFDF799FD42463346FDF798FD00222B
:10FB2000364BFDF791FD824642463346049110461E
:10FB30001946FDF78CFD5246049BFDF788FD8A4669
:10FB400000904FF0C0422E4B40463146FDF77FFDFE
:10FB50002C4A2B4B00E027E0CDE9060151460098E6
:10FB6000FDF775FD82460191274A284B40463146F4
:10FB7000FDF76DFD5246019BFDF763FD82460B4686
:10FB800002460591DDE90601FDF7BAFCDDE9062331
:10FB9000002688463046FDF754FD5246059BFDF78A
:10FBA00053FD024600F07EB90020B1F5801F07DA50
:10FBB000352230466146FDF72BFE06466FF03400D5
:10FBC00000EB215024E00000FFFF1F00FFFF0F00AB
:10FBD0000000F03F0000F07F0000404301FCFFFF09
:10FBE0002A1400000000F0FF0000F0BF0000E04118
:10FBF0000000F043FFFFEF3F5555D53F0000E03FC9
:10FC00004715F73FFE822B6544DF5DF80BAE543E8F
:10FC1000A0F2FF300190C1F3130040F07F6141F08A
:10FC200040510291FE498842D8BF002004DDFD49C1
:10FC30008142C8BF012001DD0D9008E000200D9039
:10FC40000198401C01900298A0F580100290029942
:10FC5000F54878440B910D9900EBC100D0E90023E1
:10FC60000F9330460A920B99FDF7EBFCCDE90601A4
:10FC7000DDE90A2130460F9BFDF742FC02460B46A8
:10FC80000020EA49FDF755FD059102460B4600901C
:10FC9000DDE90601FDF7DBFC1490E5488A464FF0EC
:10FCA000000878440299006812904FF0005040EA32
:10FCB00061010D980F9B01EB804000F50021099137
:10FCC0000A9A1298FDF7BDFC32460B9BFDF7BCFC6F
:10FCD00042465346FDF7BBFC06460291404651465C
:10FCE000099B129AFDF7B3FCDDE90623FDF7ACFC96
:10FCF0003246029BFDF7A5FC059B009AFDF7A7FC89
:10FD00000091149A0490534610461946FDF79FFC43
:10FD100006460246C7480B46029106217844FEF784
:10FD200087FCCDE90510029B324610461946FDF7C7
:10FD30008EFCDDE90532FDF78AFC05910646534647
:10FD400040461946149AFDF7DBFB009B049AFDF729
:10FD50007EFC3246059BFDF7D3FBCDE905104246FC
:10FD6000534610461946FDF772FC0022B24B029131
:10FD70000A90FDF7C5FBDDE90532FDF7C1FB0E4634
:10FD80004246AD4B4046FDF75CFC029B0A9AFDF7EC
:10FD900058FCDDE90532FDF757FC424602910A9016
:10FDA000334610465146FDF752FCCDE90601534655
:10FDB000149A02990A98FDF74AFC8A460290334643
:10FDC000424600990498FDF742FC5346029AFDF71B
:10FDD00097FB82460B4602460591DDE90601FDF7D9
:10FDE0008FFBDDE90623002088460646FDF729FC47
:10FDF0005246059BFDF728FC824609914FF0604270
:10FE00008E4B30464146FDF722FC049006918C4A09
:10FE10008A4B50460999FDF71AFC82460291894A9D
:10FE2000894B30464146FDF712FC5246029BFDF7D6
:10FE300067FB864B7B440D9A03EBC203D3E9002397
:10FE4000FDF75EFB0E9007910198FDF71CFD0591F3
:10FE5000DDE9061382460E9A0498FDF751FB7C4AB1
:10FE60007A440D9B02EBC303D3E900230093029273
:10FE7000FDF746FB5246059BFDF742FB00268846F0
:10FE800052463046059BFDF7DCFB009B029AFDF7CE
:10FE9000D8FB069B049AFDF7D4FB079B0E9AFDF74F
:10FEA000D3FB024600200B46029038462946FDF758
:10FEB000CEFB824601912B4638461946029AFDF741
:10FEC000C0FB32464346FDF7C2FB5246019BFDF79D
:10FED00017FB07468A463246434629460298FDF7F5
:10FEE000B6FB05460E463A465346FDF709FB594A0E
:10FEF0008846914221DBA8EB020353EA000210D1AD
:10FF00002A463346FDF79DFBCDE90401524A534B87
:10FF100038465146FDF7F4FADDE90423FDF7BEFD4E
:10FF200021D20220FEF71EFCFEF7EBFB0A4621461B
:10FF300018B062F31E01BDE8F08D494B28F0004275
:10FF40009A4210D3474A08EB020353EA00027FF4B7
:10FF5000C6AD2A463346FDF774FB3A465346FDF7D5
:10FF60009DFD7FF6BCAD0022019228F000403E4985
:10FF70003E4A01EB2051824223DA481C4FF48011A3
:10FF800021FA00F040443A4AC0F30A517A44394B0E
:10FF9000A1F2FF31CB4020EA0303C0F3130040F489
:10FFA0008010C1F11401C84012680190B8F1000F2F
:10FFB000BCBF4042019028463146FDF742FB054652
:10FFC0000E462A46334638465146FDF799FA4FF019
:10FFD00000084246284B40460591FDF738FBCDE925
:10FFE0000601264A264B40460599FDF730FB009155
:10FFF00002902A46334640460599FDF722FB3A46D1
:020000040801F1
:100000005346FDF721FB1F4A1F4BFDF720FB009BCA
:10001000029AFDF775FA0746884602460B4635E018
:100020008E9803007AB60B00721000000000F03FBB
:10003000AA100000D80F00000000084009C7EE3FDA
:10004000FD033ADCF5015B14E02F3EBEB00E00006C
:10005000740E000000009040FE822B654715973C0F
:1000600000CC904000346F3F01FCFFFF0000E03FF8
:10007000C00D0000FFFF0F00432EE63F396CA80CB7
:10008000615C20BEEF39FAFE422EE63FDDE9060153
:10009000FDF736FADDE9062305460E46FDF7D1FAEF
:1000A0003A464346FDF7D0FA0F462A4633460090BB
:1000B00010461946FDF7CBFA824602462E4888467E
:1000C0000B4605217844FEF7B3FA52464346FDF746
:1000D000BEFA2A463346FDF7B7FA80468A463B46C3
:1000E00028463146009AFDF7B2FA3B46009AFDF7E2
:1000F00007FA0691009000224FF080434046514697
:10010000FDF79FFA0F460C9042465346284631466B
:10011000FDF79DFA3B460C9AFDF70BFB069B009AF8
:10012000FDF78FFA2A463346FDF78BFA0022134B70
:10013000FDF78AFA054601980E4601EB00510815B5
:10014000002810DC28463146019AFDF761FBFEF7D6
:1001500057FA042808BFFEF7DBFA28463146019A11
:10016000FDF756FB05460B4618B02A465846214671
:10017000BDE8F04DFDF76BBA600C00000000F03FE9
:100180002DE9F04106460F46FDF7E2FE041E0D463E
:1001900018BF0120284320F00040C0F17F6000F12B
:1001A000E040C00F0ED0301C18BF0120384320F0B3
:1001B0000040C0F17F6000F1E040C00F04BF0120AB
:1001C000FEF7D0FA20462946BDE8F081100F01085D
:1001D00041020008940E01086B020008300F01086C
:1001E000970200087C0E01087F020008CC0E01086F
:1001F0009B030008E80E0108A1020008540F010843
:1002000083050008600F0108830400083C0E010804
:10021000570400084C0E0108EF0300081C0F0108EA
:10022000F3050008F80D0108F9060008EC0D0108B7
:100230005D070008100E010881070008E00D0108A5
:10024000B30700083C0F010857080008480F0108D1
:10025000E3080008B40E01086F090008C00E010889
:10026000490A00089C0E0108E70A0008A80E0108C8
:10027000310C0008040F01084D0C0008F40E0108B1
:100280006B0C0008D80E0108250D0008880E010827
:100290007D0D0008040E01089B0D00081C0E0108CE
:1002A000FB0D00082C0E0108B90D00085C0E0108BA
:1002B000690E00086C0E0108270E00082C0F0108BB
:1002C000EF05000800000000000000000004A80581
:1002D0000008500B0010A1160020000000000000D4
:1002E0000000002F000000000700070000147F142A
:1002F0007F1400242A7F2A12006264081323003628
:100300004955225000000503000000001C22410056
:10031000000041221C000014083E08140008083E9A
:100320000808000000A06000000808080808000095
:1003300060600000002010080402003E5149453E64
:100340000000427F40000042615149460021414582
:100350004B31001814127F10002745454539003CE9
:100360004A494930000171090503003649494936B7
:1003700000064949291E00003636000000005636A6
:10038000000000081422410000141414141400008A
:100390004122140800020151090600324959513E18
:1003A000007C1211127C007F49494936003E4141D0
:1003B0004122007F4141221C007F49494941007F81
:1003C00009090901003E4149497A007F0808087F70
:1003D0000000417F4100002040413F01007F0814A0
:1003E0002241007F40404040007F020C027F007F9E
:1003F0000408107F003E4141413E007F0909090683
:10040000003E4151215E007F0919294600464949B5
:1004100049310001017F0101003F4040403F001F82
:100420002040201F003F4038403F00631408146301
:1004300000070870080700615149454300007F41EB
:10044000410000552A552A55000041417F00000413
:10045000020102040040404040400000010204004C
:10046000002054545478007F4844443800384444B1
:10047000442000384444487F00385454541800083D
:100480007E0901020018A4A4A47C007F080404785B
:100490000000447D4000004080847D00007F1028E3
:1004A00044000000417F4000007C04180478007C78
:1004B0000804047800384444443800FC24242418F8
:1004C0000018242418FC007C080404080048545434
:1004D000542000043F444020003C4040207C001C4D
:1004E0002040201C003C4030403C00442810284460
:1004F000001CA0A0A07C004464544C4414141414A8
:1005000014140000000000000000000000000000C3
:100510000000000000F80000000000000033300080
:10052000000000100C06100C060000000000000087
:10053000000040C07840C0784000043F04043F04FD
:100540000400007088FC08300000001820FF211E05
:100550000000F008F000E018000000211C031E213C
:100560001E0000F00888700000001E2123241927B7
:10057000211010160E000000000000000000000016
:100580000000000000E0180402000000000718202E
:10059000400000020418E00000000040201807009E
:1005A0000000404080F0804040000202010F010244
:1005B0000200000000F0000000000101011F010125
:1005C0000100000000000000000080B0700000008A
:1005D0000000000000000000000000010101010116
:1005E00001010000000000000000003030000000A9
:1005F0000000000000008060180400601806010080
:10060000000000E010080810E000000F102020108B
:100610000F00001010F8000000000020203F2020F4
:10062000000000700808088870000030282422218B
:100630003000003008888848300000182020201141
:100640000E000000C02010F8000000070424243F22
:10065000240000F8088888080800001921202011CB
:100660000E0000E0108888180000000F11202011F3
:100670000E0000380808C83808000000003F0000DD
:1006800000000070880808887000001C22212122C8
:100690001C0000E010080810E000000031222211C8
:1006A0000F00000000C0C00000000000003030005B
:1006B00000000000008000000000000080600000DA
:1006C0000000000080402010080000010204081013
:1006D0002000404040404040400004040404040422
:1006E00004000008102040800000002010080402D0
:1006F0000100007048080808F000000000303601D2
:100700000000C030C828E810E00007182724231490
:100710000B000000C038E0000000203C230202274C
:10072000382008F8888888700000203F2020201199
:100730000E00C030080808083800071820202010D4
:10074000080008F808080810E000203F20202010CA
:100750000F0008F88888E8081000203F2020232098
:10076000180008F88888E8081000203F20000300DF
:100770000000C03008080838000007182020221E9A
:10078000020008F808000008F808203F21010121B4
:100790003F20000808F8080800000020203F202023
:1007A000000000000808F8080800C08080807F0072
:1007B000000008F888C028180800203F20012638CB
:1007C000200008F8080000000000203F2020202022
:1007D000300008F8F800F8F80800203F003F003F1C
:1007E000200008F830C00008F808203F2000071853
:1007F0003F00E01008080810E0000F102020201033
:100800000F0008F808080808F000203F2101010146
:100810000000E01008080810E0000F1824243850E9
:100820004F0008F8888888887000203F2000030C5B
:100830003020007088080808380000382021212264
:100840001C00180808F8080818000000203F2000C5
:10085000000008F808000008F808001F20202020E9
:100860001F000878880000C83808000007380E010B
:100870000000F80800F80008F800033C0700073CF7
:100880000300081868808068180820302C03032CA7
:1008900030200838C800C83808000000203F200079
:1008A000000010080808C838080020382621202039
:1008B0001800000000FE020202000000007F40401D
:1008C0004000000C30C000000000000000010638AD
:1008D000C00000020202FE000000004040407F0015
:1008E00000000000040202020400000000000000FA
:1008F00000000000000000000000808080808080F8
:1009000080800002020400000000000000000000DF
:100910000000000080808080000000192422222234
:100920003F2008F8008080000000003F11202011C7
:100930000E000000008080800000000E11202020AA
:100940001100000000808088F800000E11202010A7
:100950003F200000808080800000001F2222222291
:100960001300008080F0888888180020203F202015
:1009700000000000808080808000006B949494933D
:10098000600008F8008080800000203F21000020E7
:100990003F2000809898000000000020203F202089
:1009A0000000000000809898000000C08080807FD8
:1009B000000008F8000080808000203F24022D30D5
:1009C0002000000808F8000000000020203F202040
:1009D00000008080808080808000203F20003F20B9
:1009E000003F8080008080800000203F21000020A8
:1009F0003F200000808080800000001F20202020F9
:100A00001F00808000808000000080FFA120201156
:100A10000E000000008080808000000E112020A0C9
:100A2000FF80808080008080800020203F21200087
:100A30000100000080808080800000332424242472
:100A40001900008080E0808000000000001F20204E
:100A500000008080000000808000001F2020201007
:100A60003F20808080000080808000010E300806DA
:100A7000010080800080008080800F300C030C30EB
:100A80000F0000808000808080000020312E0E3119
:100A90002000808080000080808080818E70180619
:100AA000010000808080808080000021302C222185
:100AB000300000000000807C020200000000003FC7
:100AC000404000000000FF00000000000000FF00A8
:100AD00000000002027C800000000040403F000057
:100AE00000000006010102020404000000000000F2
:100AF000000012010002020000408304405700027F
:100B00000102030109024300020100C0320904008E
:100B1000000102020100052400100105240100016A
:100B2000042402020524060001070582030800FFD1
:100B300009040100020A000000070503024000004A
:100B400007058102400000040309041803480069F6
:100B5000006B00650072002000730075006400697E
:100B6000006F002603560069007200740075006172
:100B7000006C00200043004F004D00200050006F2B
:100B800000720074002000200000000000F45DC628
:100B90000080D14348E19240A60A563F0000000081
:100BA000555555555555C53F7D6FEB0312D6D4BFEE
:100BB0005544880E55C1C93F3B8F68B52882A4BFF4
:100BC00088B20175E0EF493F09F7FD0DE13D023FB5
:100BD0004B2D8A1C273A03C0C88A599CE52A00403D
:100BE00059018D1B6C06E6BF82922EB1C5B8B33F8A
:100BF0004FBB610567ACDD3F182D4454FB21E93F35
:100C00009BF681D20B73EF3F182D4454FB21F93F23
:100C1000E2652F227F2B7A3C075C143326A6813CA9
:100C2000BDCBF07A8807703C075C143326A6913C54
:100C3000C4EB98999999C9BF711623FEC671BCBFC0
:100C40006D9A74AFF2B0B3BF9AFDDE522DDEADBF28
:100C50002F6C6A2C44B4A2BF0D5555555555D53F40
:100C6000FF8300922449C23F6E204CC5CD45B73F5B
:100C7000513DD0A0660DB13FEB0D76244B7BA93FD3
:100C800011DA22E33AAD903F000000000080513DB0
:100C90000070C63D00900D3E0050343E00E0573ECF
:100CA00000D0783E00C08B3E000000000AD6A93676
:100CB000431C8C37658F7338832DA236121D1F3865
:100CC000B3756F38D2535A38000000000000F03F6F
:100CD000000000000000F83F0000000000000000DD
:100CE0000000004003B8E23F0000000000000000E8
:100CF00006D0CF43EBFD4C3E033333333333E33F76
:100D0000FFAB6FDBB66DDB3F4D268F515555D53FA1
:100D100001411DA96074D13F65DBC9934A86CD3F6F
:100D2000EF4E454A287ECA3F3E5555555555C53F5D
:100D300093BDBE166CC166BF2CDE25AF6A56113F4F
:100D4000F16BD2C541BDBBBED0A4BE726937663E51
:100D500000000000000000000040404040404040D3
:100D6000404041414141414040404040404040407E
:100D70004040404040404040400502020202020222
:100D80000202020202020202022020202020202071
:100D90002020200202020202020290909090909085
:100DA0001010101010101010101010101010101043
:100DB00010101010020202020202888888888888B7
:100DC00008080808080808080808080808080808A3
:100DD000080808080202020240000000590D01083C
:100DE00041542B44454341240000000041542B54FE
:100DF0004553544F4C45440041542B544553544C97
:100E00004544000041542B555345525F434D440027
:100E100041542B44495354414E43450041542B47C0
:100E200045545557424D4F444500000041542B5303
:100E300045545557424D4F444500000041542B47FF
:100E40004554574F524B4D4F4445000041542B538E
:100E50004554574F524B4D4F4445000041542B478A
:100E600045544D43554D4F444500000041542B53CC
:100E700045544D43554D4F444500000041542B52BD
:100E80004553544F5245000041542B554152545242
:100E90004154450041542B534156450041542B5079
:100EA000444F414F4646000041542B524E474F4657
:100EB0004600000041542B41444454414700000087
:100EC00041542B44454C54414700000041542B47AA
:100ED000455443464700000041542B50444F41477E
:100EE000455443464700000041542B534554434664
:100EF0004700000041542B50444F41534554434652
:100F00004700000041542B46494C54455200000014
:100F100041542B47455456455200000041542B473D
:100F2000455453454E534F520000000041540000B9
:100F300041542B52455354415254000041542B47C5
:100F40004554444C4953540041542B4745544B4C51
:100F50004953540041542B47455444455600000022
:100F600041542B5345544445560000000D0A676513
:100F700074646576206361703A256420616E6E64E6
:100F8000656C61793A25642C206B616C6D616E5FD4
:100F9000656E61626C653A25642C206B616C6D61D5
:100FA0006E5F513A252E33662C206B616C6D616E3D
:100FB0005F523A252E33662C20706172615F613A70
:100FC000252E34662C20706172615F623A252E32C4
:100FD000662C20706F735F656E61626C653A256484
:100FE0002C20706F735F64696D656E3A25640D0A1D
:100FF000000000000D0A73657464657620636170FB
:101000003A256420616E6E64656C61793A25642CC2
:10101000206B616C6D616E5F656E61626C653A2517
:10102000642C206B616C6D616E5F513A252E3366C6
:101030002C206B616C6D616E5F523A252E33662CED
:1010400020706172615F613A252E34662C207061D8
:1010500072615F623A252E32662C20706F735F6575
:101060006E61626C653A25642C20706F735F6469F1
:101070006D656E3A25640D0A0000000067657463B3
:10108000666720446C6973743A2564204B4C69731D
:10109000743A2564204E65743A2530345820416EE8
:1010A0006349443A256420526174653A25642046B8
:1010B000696C7465723A25642055736572436D647A
:1010C0003A25642070646F614F66667365743A25D3
:1010D0006420726E674F66667365743A25640D0A04
:1010E000000000007B22736C6F74223A222530349A
:1010F00058222C22613634223A222530386C582569
:1011000030386C58222C22613136223A2225303474
:1011100058222C2246223A2225303458222C22539F
:10112000223A2225303458222C224D223A222530D0
:101130003458227D00000000202020555742204DC9
:101140006F64756C6520B4EDCEF3CEBB313A256487
:101150002C20B4EDCEF3CEBB323A25642C20B4ED76
:10116000CEF3CEBB333A25642C20B4EDCEF3CEBB08
:10117000343A25642C20B4EDCEF3CEBB353A256449
:101180000D0A0000202020555742204D6F64756CD9
:101190006520BBF9D5BECDF8C2E73A2530345820DA
:1011A000BBF9D5BEC8DDC1BF3A256420B1EAC7A9E5
:1011B000C8DDC1BF3A256420D7EEB4F3B1EAC7A9B0
:1011C000C8DDC1BF3A25640D0A000000202020556B
:1011D0005742204D6F64756C6520BEE0C0EBB2CE07
:1011E000CAFD3AC6F4B6AFC2CBB2A83A25642CBF4A
:1011F000A8B6FBC2FCB2CECAFD513A252E33662CEE
:1012000020BFA8B6FBC2FCB2CECAFD523A252E338F
:10121000662C20D0A3D5FDCFB5CAFD613A252E346A
:10122000662C20D0A3D5FDCFB5CAFD623A252E325B
:10123000662C20CCECCFDFD1D3B3D93A25640A0099
:1012400041542B5557424D414300000041542B520D
:101250005353490041542B56455253494F4E0000B9
:1012600041542B52465445535400000041542B47DF
:1012700050494F544553540041542B52535400008D
:10128000726E674F66667365745F6D6DA3BA256491
:101290002C70646F614F66667365745F6465672068
:1012A0003A25642C206D6F74696F6E66696C746585
:1012B000723A25642C20757365725F636D643A25FC
:1012C000640A0000E4120108000000200C14000071
:1012D0001AE50008CC1601080C140020243B00007D
:1012E00054E70008C116D03FD03F0A12646009E8F5
:1012F000039001C012FFFF14111101120A2009BC52
:1013000074933C1D5A243F1A80044165FFFF11115C
:101310001A01031E8813E803323A190C1114010153
:10132000642DED39CC4604295012141EC201C409A3
:10133000010A211305011C090901263A413801FF60
:1013400001FF01FF01FF01FF01FF01FF01FF01FF9D
:1013500001FF01FF0110021F0116D03FD03F0A120A
:10136000646009E8039001C012FFFF14111101121B
:101370000A2009BC74933C1D5A243F1A8004417D05
:10138000FFFF1111581F018813E803323A29641432
:101390000101642DED39CC4604295012141EC201FE
:1013A000C409010A211305011C090901260A20416B
:1013B0009009AAA83924DD0801400210DA0410AA15
:1013C0000810140C0140DA8010DA4010DA2010CA3C
:1013D0001010699C6960E910593F7910596F7910B4
:1013E000596F7910595F7960694069D8690CA91003
:1013F000DA0310DA05109A065069186970490999DC
:101400001059217910DA0410DA081059B1791059FD
:10141000B1791059E16980B9F019100A1180E0E939
:1014200010292CA9102993A910DA071059A3D11358
:10143000E00C1B20F00411120D1B2010041A2004D4
:101440001A30041A4004411A50081A60041A700431
:101450001A80041A90041AA0041AB0041AC0041ABC
:10146000D0041AE0042AF0306A0EE6211A100C1A91
:1014700020041A30041A40041A50041A60041A7026
:10148000041A80045A902C1AA0081AB0041AC00436
:101490001AD0041AE0041305051C090901DE1281A3
:1014A00024090303175412010835151B0878081A7C
:1014B00041081A6C0813EB1A1B08600813DF1C1B89
:1014C000084C0813D3201B0840081BA92110160E36
:1014D00001080D231B083C081A77081E2C0F010871
:1014E000A508211954B904A17A900FE32041E9100D
:1014F0006132341AFD01690C1AFE014113090D1CF9
:101500000A0A034D2B0102C25113382B1320011676
:101510003E22E2223E2BFE220113E20217203F2050
:101520001F11112B7F4401134740180D040404F4CC
:1015300084D4A5A6A4D484F40C1952300D0202124E
:101540003A1613121A3242827E16FC848484FC2AD4
:10155000100124FF10101A3F091A3F682D06408021
:101560007FA716102CE724243AF01E1AF018160153
:10157000017F21113008070202FF02020719552BD3
:10158000FF540125FF0406841010111189899593D9
:1015900091FD919B95C58919091F10D0121C10D07F
:1015A0005817FF0808088C08280A206027101C1309
:1015B00010FF41011BFF01791DD0FF9050AC1EC4EC
:1015C00044464460B0120312FF1C1108467D3402E9
:1015D0000C18180D1008078C54261428478C9406F4
:1015E000BFC01002028189B2828AB282C3A29881EE
:1015F00003011426035612691272127412751261D5
:10160000126C12201243124F1A4D0812503A6F18E2
:101610001A2002011613CD800C1C088F8D040B10AC
:10162000098114512AC287120836F20A01081236BB
:10163000040B01084313DD821B08F90413E1831B2B
:1016400008F104131B841B0865041AAD041A8304F3
:101650001A8B041A93044132401A473819E2111ABE
:101660004B0829FA1A630832261374112A20081A23
:10167000046729741AC94C0916A41AD91C41299265
:1016800001240926280118134188B808CADE5044ED
:101690006F4119120E116F41504420269A21209B50
:1016A000100219024723093D9008091F0102030493
:1016B000050607089845020406082931290419344B
:0C16C000120984A24A04791431000000D1
:04000005080000ED02
:00000001FF
